S01B00006275666665725F646973635F745F626F6172642E7372656353
S3150802000000000A201DBE0308254903082D490308D6
S31508020010354903083D490308454903086DBE0308E7
S315080200200000000000000000000000006DBE03088A
S315080200304D4903080000000035030208E1020208E0
S315080200406DBE03086DBE03086DBE03086DBE0308C8
S315080200506DBE03086DBE03086DBE03086DBE0308B8
S315080200606DBE03086DBE03086DBE03085B4903082F
S31508020070694903086DBE03086DBE03086DBE030811
S315080200806DBE03086DBE03086DBE03086DBE030888
S315080200906DBE03086DBE03086DBE03086DBE030878
S315080200A06DBE03086DBE03086DBE03086DBE030868
S315080200B06DBE03086DBE03086DBE03086DBE030858
S315080200C06DBE03086DBE03086DBE03086DBE030848
S315080200D0000000006DBE03086DBE030879490308D7
S315080200E06DBE03086DBE03086DBE03086DBE030828
S315080200F06DBE03086DBE03086DBE03086DBE030818
S315080201006DBE03088D4903086DBE03086DBE03085C
S315080201106DBE03086DBE03086DBE03086DBE0308F7
S315080201206DBE03086DBE0308A14903086DBE030828
S315080201306DBE03086DBE03086DBE03086DBE0308D7
S315080201406DBE03086DBE03086DBE03086DBE0308C7
S315080201506DBE03086DBE03086DBE03086DBE0308B7
S315080201606DBE0308B54903086DBE03086DBE0308D4
S315080201706DBE03086DBE03086DBE03086DBE030897
S315080201806DBE03086DBE03086DBE03086DBE030887
S315080201906DBE03086DBE03086DBE03086DBE030877
S315080201A06DBE03086DBE03086DBE03086DBE030867
S315080201B06DBE03086DBE03086DBE03086DBE030857
S315080201C06DBE03086DBE03086DBE03086DBE030847
S315080201D06DBE03086DBE03086DBE03086DBE030837
S315080201E06DBE03086DBE03086DBE03086DBE030827
S315080201F06DBE03086DBE03086DBE03086DBE030817
S315080202006DBE03086DBE03086DBE0308000000003C
S31508020210000000006DBE0308000000006DBE030862
S315080202206DBE03086DBE03086DBE03086DBE0308E6
S315080202306DBE03086DBE03086DBE03086DBE0308D6
S315080202406DBE03086DBE03086DBE030800000000FC
S3150802025010B5054C237833B9044B13B10448AFF3F0
S3150802026000800123237010BDF01400200000000056
S31508020270E496050808B5034B1BB103490348AFF3D7
S31508020280008008BD00000000F4140020E49605086A
S3150802029072B64FF0E0201749C0F8081D16480168E3
S315080202A041F00101016015481249096801604FF0E1
S315080202B0E020134941614FF0070101614FF0000147
S315080202C0C0F8181D4FF07F41C0F81C1D0D49C0F833
S315080202D0201D7047FFF7FEBF01B5BDE80140704714
S315080202E001B500F097F8BDE801407047FFF7FEBF79
S315080202F0FFF7FEBF00000208001000E0001102200E
S315080203008FD003000000FF404FF000002D4A106016
S31508020310EFF3148020F0040080F3148862B64FF0DD
S3150802032080504FF0E021C1F8040DBFF34F8FBFF3A1
S315080203306F8FFEE72448254A4FF00003016891B102
S315080203400360EFF3098C2CE9F00F1EF0100F01D1B0
S315080203502CED108A1E4C4CF804EDC1F808C025682D
S315080203600DB18D61236072B61168D1B1016062B6B2
S315080203704F68174C8D6907F101074F602560D1F860
S315080203800CC08CF30B88D1F808C05CF804EB1EF09D
S31508020390100F01D1BCEC108ABCE8F00F8CF3098867
S315080203A0704772B61168016009B962B6F9E74FF08B
S315080203B000674FF0E028C8F8047D62B6D8E700BFA8
S315080203C0704700009C110220041102200811022025
S315080203D008170220026922F00702A2F144026FF00E
S315080203E0430313604FF0000353609360D3601361B5
S315080203F053619361D361136253629362D362136347
S3150802040053634FF0FF339363D1634FF080731364E2
S31508020410826070472249086800F101000860214B92
S315080204201A683AB1A2F101021A601AB91E4B4FF0C4
S31508020430010018601D490868026822B11C4B4FF07A
S3150802044001021A6008E000F104001A4B1A68904289
S3150802045001D1194B18680860134B1A6812B9144966
S315080204600868C8B101B51249086808B129F0F2F955
S315080204700D4B1A6872B129F05FF91048016849B93B
S315080204800F4801680F4A13680F484FF08052994285
S3150802049000D00260BDE80140BFF34F8F70470000ED
S315080204A0A811022008170220AC11022038120220D5
S315080204B03C12022034120220301202209C11022021
S315080204C0041102200811022004ED00E0034613F885
S315080204D0012B002AFBD1181A0138704781F0004116
S315080204E002E000BF83F0004330B54FEA41044FEA09
S315080204F0430594EA050F08BF90EA020F1FBF54EAA4
S31508020500000C55EA020C7FEA645C7FEA655C00F03F
S31508020510E2804FEA5454D4EB5555B8BF6D420CDD10
S315080205202C4480EA020281EA030382EA000083EA93
S31508020530010180EA020281EA0303362D88BF30BD33
S3150802054011F0004F4FEA01314FF4801C4CEA113189
S3150802055002D0404261EB410113F0004F4FEA0333E8
S315080205604CEA133302D0524263EB430394EA050F73
S3150802057000F0A780A4F10104D5F1200E0DDB02FAE2
S315080205800EFC22FA05F2801841F1000103FA0EF276
S31508020590801843FA05F359410EE0A5F120050EF13C
S315080205A0200E012A03FA0EFC28BF4CF0020C43FA6D
S315080205B005F3C01851EBE37101F0004507D54FF07A
S315080205C0000EDCF1000C7EEB00006EEB0101B1F5CA
S315080205D0801F1BD3B1F5001F0CD349085FEA300010
S315080205E04FEA3C0C04F101044FEA445212F5800F1B
S315080205F080F09A80BCF1004F08BF5FEA500C50F1B8
S31508020600000041EB045141EA050130BD5FEA4C0C9A
S31508020610404141EB0101013C28BFB1F5801FE9D2F7
S3150802062091F0000F04BF01460020B1FA81F308BF1A
S315080206302033A3F10B03B3F120020CDA0C3208DDE6
S3150802064002F1140CC2F10C0201FA0CF021FA02F1C1
S315080206500CE002F11402D8BFC2F1200C01FA02F131
S3150802066020FA0CFCDCBF41EA0C019040E41AA2BF56
S3150802067001EB0451294330BD6FEA04041F3C1CDA1E
S315080206800C340EDC04F11404C4F1200220FA04F03E
S3150802069001FA02F340EA030021FA04F345EA0301E8
S315080206A030BDC4F10C04C4F1200220FA02F001FAAA
S315080206B004F340EA0300294630BD21FA04F029462C
S315080206C030BD94F0000F83F4801306BF81F48011C5
S315080206D00134013D4EE77FEA645C18BF7FEA655C38
S315080206E029D094EA050F08BF90EA020F05D054EA0A
S315080206F0000C04BF1946104630BD91EA030F1EBF0F
S315080207000021002030BD5FEA545C05D14000494112
S3150802071028BF41F0004130BD14F580043CBF01F505
S31508020720801130BD01F0004545F0FE4141F47001EB
S315080207304FF0000030BD7FEA645C1ABF19461046C6
S315080207407FEA655C1CBF0B46024650EA013406BFC7
S3150802075052EA033591EA030F41F4002130BD00BF86
S3150802076090F0000F04BF0021704730B54FF4806443
S3150802077004F132044FF000054FF0000150E700BFC4
S3150802078090F0000F04BF0021704730B54FF4806423
S3150802079004F1320410F0004548BF40424FF0000110
S315080207A03EE700BF42004FEAE2014FEA31014FEA53
S315080207B002701FBF12F07F4393F07F4F81F06051A2
S315080207C0704732F07F4208BF704793F07F4F04BFED
S315080207D041F40021704730B54FF4607401F00045CA
S315080207E021F000411CE700BF50EA010208BF70472A
S315080207F030B54FF000050AE050EA010208BF70471B
S3150802080030B511F0004502D5404261EB41014FF483
S31508020810806404F132045FEA915C3FF4D8AE4FF08B
S3150802082003025FEADC0C18BF03325FEADC0C18BF6E
S31508020830033202EBDC02C2F1200300FA03FC20FABF
S3150802084002F001FA03FE40EA0E0021FA02F114440C
S31508020850BDE600BF70B54FF0FF0C4CF4E06C1CEA25
S3150802086011541DBF1CEA135594EA0C0F95EA0C0F96
S3150802087000F0DEF82C4481EA030621EA4C5123EA09
S315080208804C5350EA013518BF52EA033541F4801138
S3150802089043F4801338D0A0FB02CE4FF00005E1FBEB
S315080208A002E506F00042E0FB03E54FF00006E1FB35
S315080208B003569CF0000F18BF4EF0010EA4F1FF0478
S315080208C0B6F5007F64F5407404D25FEA4E0E6D41B8
S315080208D046EB060642EAC62141EA55514FEAC520C9
S315080208E040EA5E504FEACE2EB4F1FD0C88BFBCF545
S315080208F0E06F1ED8BEF1004F08BF5FEA500E50F1F6
S31508020900000041EB045170BD06F0004646EA0101BB
S3150802091040EA020081EA0301B4EB5C04C2BFD4EBED
S315080209200C0541EA045170BD41F480114FF0000EE6
S31508020930013C00F3AB8014F1360FDEBF002001F054
S31508020940004170BDC4F10004203C35DA0C341BDCCE
S3150802095004F11404C4F1200500FA05F320FA04F0A0
S3150802096001FA05F240EA020001F0004221F00041D4
S3150802097010EBD37021FA04F642EB06015EEA430E47
S3150802098008BF20EAD37070BDC4F10C04C4F1200577
S3150802099000FA04F320FA05F001FA04F240EA02002A
S315080209A001F0004110EBD37041F100015EEA430EFB
S315080209B008BF20EAD37070BDC4F1200500FA05F21B
S315080209C04EEA020E20FA04F301FA05F243EA02039A
S315080209D021FA04F001F0004121FA04F220EA0200A9
S315080209E000EBD3705EEA430E08BF20EAD37070BDEF
S315080209F094F0000F0FD101F00046400041EB0101CF
S31508020A0011F4801F08BF013CF7D041EA060195F0B0
S31508020A10000F18BF704703F00046520043EB03036A
S31508020A2013F4801F08BF013DF7D043EA0603704757
S31508020A3094EA0C0F0CEA135518BF95EA0C0F0CD062
S31508020A4050EA410618BF52EA4306D1D181EA0301A8
S31508020A5001F000414FF0000070BD50EA410606BFA2
S31508020A601046194652EA430619D094EA0C0F02D1E7
S31508020A7050EA013613D195EA0C0F05D152EA03362C
S31508020A801CBF104619460AD181EA030101F000414A
S31508020A9041F0FE4141F470014FF0000070BD41F093
S31508020AA0FE4141F4780170BD70B54FF0FF0C4CF46D
S31508020AB0E06C1CEA11541DBF1CEA135594EA0C0F8C
S31508020AC095EA0C0F00F0A7F8A4EB050481EA030ED9
S31508020AD052EA03354FEA013100F088804FEA0333C0
S31508020AE04FF0805545EA131343EA12634FEA02228E
S31508020AF045EA111545EA10654FEA00260EF000414F
S31508020B009D4208BF964244F1FD0404F5407402D2A0
S31508020B105B084FEA3202B61A65EB03055B084FEA31
S31508020B2032024FF480104FF4002CB6EB020E75EB2E
S31508020B30030E22BFB61A754640EA0C005B084FEA56
S31508020B403202B6EB020E75EB030E22BFB61A7546D3
S31508020B5040EA5C005B084FEA3202B6EB020E75EB1E
S31508020B60030E22BFB61A754640EA9C005B084FEA96
S31508020B703202B6EB020E75EB030E22BFB61A7546A3
S31508020B8040EADC0055EA060E18D04FEA051545EA92
S31508020B9016754FEA06164FEAC30343EA52734FEA3B
S31508020BA0C2025FEA1C1CC0D111F4801F0BD141EAB4
S31508020BB000014FF000004FF0004CB6E711F4801F19
S31508020BC004BF01430020B4F1FD0C88BFBCF5E06FF9
S31508020BD03FF6AFAEB5EB030C04BFB6EB020C5FEA09
S31508020BE0500C50F1000041EB045170BD0EF0004E5E
S31508020BF04EEA113114EB5C04C2BFD4EB0C0541EA90
S31508020C00045170BD41F480114FF0000E013C90E68C
S31508020C1045EA060E8DE60CEA135594EA0C0F08BF50
S31508020C2095EA0C0F3FF43BAF94EA0C0F0AD150EA4F
S31508020C3001347FF434AF95EA0C0F7FF425AF1046E2
S31508020C4019462CE795EA0C0F06D152EA03353FF40A
S31508020C50FDAE1046194622E750EA410618BF52EA87
S31508020C6043067FF4C5AE50EA41047FF40DAF52EA5B
S31508020C7043057FF4EBAE12E74FF0FF3C06E000BFF8
S31508020C804FF0010C02E000BF4FF0010C4DF804CD05
S31508020C904FEA410C7FEA6C5C4FEA430C18BF7FEAC5
S31508020CA06C5C1BD001B050EA410C0CBF52EA430CF3
S31508020CB091EA030F02BF90EA020F0020704710F173
S31508020CC0000F91EA030F58BF994208BF90422CBF02
S31508020CD0D8176FEAE37040F0010070474FEA410CFB
S31508020CE07FEA6C5C02D150EA013C07D14FEA430C19
S31508020CF07FEA6C5CD6D152EA033CD3D05DF8040B8A
S31508020D00704700BF8446104662468C4619466346BB
S31508020D1000E000BF01B5FFF7B7FF002848BF10F192
S31508020D20000F01BD4DF808EDFFF7F4FF0CBF0120D7
S31508020D3000205DF808FB00BF4DF808EDFFF7EAFF53
S31508020D4034BF012000205DF808FB00BF4DF808ED0E
S31508020D50FFF7E0FF94BF012000205DF808FB00BF03
S31508020D604DF808EDFFF7CEFF94BF012000205DF88D
S31508020D7008FB00BF4DF808EDFFF7C4FF34BF01209A
S31508020D8000205DF808FB00BF4FEA410C7FEA6C5C65
S31508020D9002D150EA013C0AD14FEA430C7FEA6C5C65
S31508020DA002D152EA033C02D14FF0000070474FF0DD
S31508020DB0010070474FEA410212F5001215D211D509
S31508020DC06FF47873B3EB625212D94FEAC12343F038
S31508020DD0004343EA505311F0004F23FA02F018BFBA
S31508020DE0404270474FF00000704750EA013005D183
S31508020DF011F0004008BF6FF0004070474FF0000046
S31508020E00704700BF4A0011D212F5001211D20DD551
S31508020E106FF47873B3EB62520ED44FEAC12343F0F0
S31508020E20004343EA505323FA02F070474FF000009A
S31508020E30704750EA013002D14FF0FF3070474FF049
S31508020E40000070474FEA4102B2F1E04324BFB3F50E
S31508020E50001CDCF1FE5C0DD901F0004C4FEAC00221
S31508020E604CEA5070B2F1004F40EB830008BF20F005
S31508020E700100704711F0804F21D113F13872BCBFBF
S31508020E8001F00040704741F480114FEA5252C2F114
S31508020E901802C2F1200C10FA0CF320FA02F018BF5D
S31508020EA040F001004FEAC1234FEAD32303FA0CFCB0
S31508020EB040EA0C0023FA02F34FEA4303CCE77FEA3F
S31508020EC0625307D150EA01331EBF4FF0FE4040F489
S31508020ED04000704701F0004040F0FE4040F4000038
S31508020EE0704700BF53B94AB9002908BF00281CBF7A
S31508020EF04FF0FF314FF0FF3000F0B4B9ADF1080CF6
S31508020F006DE904CE00F03CF8DDF804E0DDE90223E1
S31508020F1004B0704738B50022002304460D46FFF791
S31508020F200BFF28B920462946BDE8384000F00AB822
S31508020F30204605F1004100F005F8404261EB410107
S31508020F4038BD00BFD0B500220B4B06460F46FFF749
S31508020F5081FCFFF757FF0446FFF702FC0022074B06
S31508020F60FFF778FC02460B4630463946FFF7BAFACF
S31508020F70FFF748FF2146D0BD0000F03D0000F041D2
S31508020F802DE9F04F099D0C46002B4DD18A420F469A
S31508020F9084469646B2FA82F360D94BB102FA03FE48
S31508020FA0C3F120029F4000FA03FC20FA02F217431B
S31508020FB04FEA1E461FFA8EF44FEA1C42B7FBF6F1B9
S31508020FC006FB117701FB04F042EA0742904208D970
S31508020FD01EEB020201F1FF3702D2904200F22D8186
S31508020FE03946121A1FFA8CFCB2FBF6F006FB1022DF
S31508020FF000FB04F44CEA024C644508D91EEB0C0CBF
S3150802100000F1FF3202D2644500F21A81104640EA24
S315080210100140ACEB040C002125B12CFA03F30022A3
S31508021020C5E90032BDE8F08F8B4205D90DB1C5E995
S31508021030000100210846F5E7B3FA83F100294DD1EC
S31508021040A342C0F0F280904280F0EF800646234623
S315080210500846002DE6D0C5E90063E3E7002B40F019
S31508021060A2808A1A4FEA1E471FFA8EF60121B2FBA0
S31508021070F7F407FB14204FEA1C4242EA004206FB39
S3150802108004F090420FD91EEB020204F1FF382CBF7E
S315080210904FF001094FF00009904203D9B9F1000F48
S315080210A000F0C8804446121A1FFA8CFCB2FBF7F00D
S315080210B007FB102200FB06F64CEA024C664508D9E5
S315080210C01EEB0C0C00F1FF3202D2664500F2BB8021
S315080210D01046ACEB060C40EA04409DE7C1F1200637
S315080210E08B4004FA01FE22FA06F720FA06FCF440BF
S315080210F08A401F434EEA0C0300FA01FE4FEA1748DC
S315080211004FEA13491FFA87FCB4FBF8F008FB1044B0
S3150802111049EA044400FB0CF9A1450ED93C1900F131
S31508021120FF3A2CBF4FF0010B4FF0000BA14503D934
S31508021130BBF1000F00F093805046A4EB09041FFA96
S3150802114083F9B4FBF8F308FB134403FB0CFC49EAE6
S315080211500444A44506D93C1903F1FF3801D2A44533
S315080211607AD8434643EA0040A4EB0C04A0FB029853
S315080211704445CC46434602D306D1CE4504D201386D
S31508021180B9EB020C68EB07035DB1BEEB0C0264EB2C
S31508021190030404FA06F622FA01F3CC401E43C5E913
S315080211A0006400213EE702FA03FEC3F1200104FAB5
S315080211B003F200FA03FCCC404FEA1E4720FA01F17B
S315080211C01FFA8EF6B4FBF7F00A4307FB1044110C1C
S315080211D041EA044100FB06F48C420ED91EEB0101DA
S315080211E000F1FF382CBF4FF001094FF000098C427D
S315080211F002D9B9F1000F2CD04046091B92B2B1FBB5
S31508021200F7F407FB141142EA014204FB06F1914284
S3150802121007D91EEB020204F1FF3801D2914215D812
S315080212204446521A44EA004121E7861A64EB03034C
S3150802123001200EE7023C724435E702397244D0E6D1
S31508021240F4440238E3E6F444023842E7023C7244C4
S31508021250E7E702387144D0E7023B3C4482E70238AA
S315080212603C446AE7704700BF80B586B002AF786033
S315080212700023FB60342300934FF4C8430B4A0C49FE
S315080212800C4828F091FD0346002B0AD1094BBB6096
S31508021290B86802F071FEF860FB68002B01D000BF47
S315080212A0FDE700BF1037BD4680BD00BF0C15002004
S315080212B0009705080C79002080B582B000AF7860E7
S315080212C014220021786834F049FF7B68134A1A60B1
S315080212D07B684FF448725A607B6800221A727B68F0
S315080212E003225A727B6800229A727B680022DA729B
S315080212F07B6801221A737B6801225A737B68012272
S315080213009A737B6800221A747B6800225A7478687A
S3150802131000F06EF800BF0837BD4680BD3530424D35
S3150802132080B588B000AFF860B9601346FB71002338
S31508021330FB6100233B61BB687B617B69BB61002360
S31508021340FB6110E0FA69FB681344184630F03AF973
S3150802135003463B613A69BB691A60BB690433BB61E0
S31508021360FB690433FB61FB79FA699A42EADB0123DA
S3150802137018462037BD4680BD80B588B000AF786074
S3150802138014220021786834F0E9FE07F10C031422CE
S315080213900021184634F0E2FE07F10C03142219461E
S315080213A00F48FFF7BDFFFB680E4A934207D07868DD
S315080213B0FFF782FF10210C481AF044FB0AE007F1F6
S315080213C00C0314221946786834F07FFF0F21074868
S315080213D01AF038FB002318462037BD4680BD00BFE9
S315080213E000C01F083530424D14970508289705088E
S315080213F090B589B000AF78600023FB617B68BB615A
S31508021400FE2030F00EF90023FB611FE007F1080306
S3150802141010220021184634F0A1FEBB6907F1080420
S31508021420186859689A68DB680FC4FB6903F1016397
S3150802143003F57C2307F108021146184630F0D6F860
S31508021440BB691033BB61FB691033FB61FB69132B64
S31508021450DCD9012318462437BD4690BD80B483B033
S3150802146000AF78607B685B6818460C37BD465DF846
S31508021470047B704780B483B000AF786039607B68BC
S315080214803A685A6000BF0C37BD465DF8047B704760
S3150802149080B483B000AF78607B681B7A18460C3735
S315080214A0BD465DF8047B704780B483B000AF7860B0
S315080214B00B46FB707B68FA781A7200BF0C37BD467A
S315080214C05DF8047B704780B483B000AF78600B4642
S315080214D0FB70FB78042B04D8FB787A6813449B7A52
S315080214E000E0002318460C37BD465DF8047B7047BA
S315080214F080B483B000AF78600B46FB701346BB70AE
S31508021500FB78042B0DD8BB78002B05D0FB787A68BC
S31508021510134401229A7204E0FB787A681344002283
S315080215209A7200BF0C37BD465DF8047B704780B4DB
S3150802153083B000AF78607B68DB7B18460C37BD4604
S315080215405DF8047B704780B483B000AF78607B682F
S315080215501B7C18460C37BD465DF8047B704780B481
S3150802156083B000AF78600B46FB707B68FA781A7412
S3150802157000BF0C37BD465DF8047B704780B483B064
S3150802158000AF78607B685B7C18460C37BD465DF811
S31508021590047B704780B483B000AF78600B46FB705B
S315080215A07B68FA785A74012318460C37BD465DF8EB
S315080215B0047B704780B483B000AF0346FB71044ACC
S315080215C0FB79137000BF0C37BD465DF8047B704784
S315080215D0218F002080B586B000AFF8600B467A608E
S315080215E0FB720023FB752D481AF068FA0023FB7577
S315080215F04CE0FB7D2A4A4FF48E7101FB03F3134438
S315080216001B78012B3FD1FB7D4FF48E7202FB03F34D
S31508021610234A13440233194622481AF04FFA22483B
S315080216201AF04CFAFB7D4FF48E7202FB03F3183361
S315080216301B4A1344043319461A481AF03FFA1B4840
S315080216401AF03CFAFB7D164A4FF48E7101FB03F33E
S3150802165013449C331B782D2B12D015481AF02EFAF8
S31508021660FB7D4FF48E7202FB03F398330C4A134444
S31508021670043319460B481AF021FA0C481AF01EFAD6
S315080216800A481AF01BFAFB7D0133FB75FB7D102B0A
S31508021690AFD900BF00BF1837BD4680BD38970508C9
S315080216A000000020609705086497050868970508F2
S315080216B06C97050880B584B000AFF8600B467A606F
S315080216C0FB7214F081FB0346184614F0C9FB00BFEF
S315080216D01037BD4680BD000080B586B000AFF86001
S315080216E00B467A60FB7200237B617B6803F5007305
S315080216F003224C49184634F039FD0346002B22D101
S315080217007B6803F500731846FEF7E0FE0346032BD3
S3150802171019D17B6803F58063184633F01DFC78619E
S315080217207B69002B07D014F04FFB034601211846AC
S3150802173014F029FF71E014F047FB0346012118460D
S3150802174014F03EFF69E07B6803F50073052236490B
S31508021750184634F00BFD0346002B22D17B6803F5AD
S3150802176000731846FEF7B2FE0346052B19D17B68AD
S3150802177003F58063184633F0EFFB78617B69002B2B
S3150802178007D014F021FB03460421184614F0FBFE89
S3150802179043E014F019FB03460421184614F010FF1F
S315080217A03BE07B6803F5007303222049184634F0B0
S315080217B0DDFC0346002B30D17B6803F5007318461F
S315080217C0FEF784FE0346032B27D17B6803F5806365
S315080217D0184633F0C1FB78617B69002B0ED014F0F2
S315080217E0F3FA03460121184614F0CDFE14F0ECFA7A
S315080217F003460421184614F0C6FE0EE014F0E4FA75
S3150802180003460121184614F0DBFE14F0DDFA0346FE
S315080218100421184614F0D4FEFFE700BF1837BD4668
S3150802182080BD00BF789705087C9705088497050848
S3150802183080B584B000AFF8600B467A60FB727B68AD
S3150802184003F500731A78B54B1B78D31A002B12D1FD
S315080218507B6803F500731846FEF738FE0346012B2C
S3150802186009D1AF481AF02AF9AE481AF027F9AE4854
S315080218701AF024F94FE27B6803F500730B22AB4991
S31508021880184634F073FC0346002B40F0C5817B688A
S3150802189003F500731846FEF719FE03460B2B40F0B4
S315080218A0BB817B6803F580630922A149184634F097
S315080218B05DFC0346002B6FD17B6803F580631846EF
S315080218C0FEF704FE0346092B66D17B6803F5C0635F
S315080218D01A78984B1B78D31A002B08D17B6803F524
S315080218E0C0631846FEF7F2FD0346012B13D07B6848
S315080218F003F5C06302229049184634F037FC0346C2
S31508021900002B13D17B6803F5C0631846FEF7DEFD8C
S315080219100346022B0AD114F057FA03460121184648
S3150802192014F070FE85481AF0C9F834E07B6803F5AE
S31508021930C0631A78824B1B78D31A002B08D17B68AE
S3150802194003F5C0631846FEF7C1FD0346012B13D003
S315080219507B6803F5C06303227A49184634F006FC0D
S315080219600346002B13D17B6803F5C0631846FEF7BE
S31508021970ADFD0346032B0AD114F026FA03460121CC
S31508021980184614F05CFE70481AF098F803E06F489F
S315080219901AF094F8BFE13EE17B6803F580630922F9
S315080219A06B49184634F0E2FB0346002B6FD17B687D
S315080219B003F580631846FEF789FD0346092B66D1AF
S315080219C07B6803F5C0631A785A4B1B78D31A002B27
S315080219D008D17B6803F5C0631846FEF777FD034610
S315080219E0012B13D07B6803F5C063022252491846BD
S315080219F034F0BCFB0346002B13D17B6803F5C063A6
S31508021A001846FEF763FD0346022B0AD114F0DCF9E9
S31508021A1003460221184614F0F5FD4E481AF04EF810
S31508021A2034E07B6803F5C0631A78454B1B78D31AF2
S31508021A30002B08D17B6803F5C0631846FEF746FDFE
S31508021A400346012B13D07B6803F5C06303223D4985
S31508021A50184634F08BFB0346002B13D17B6803F53B
S31508021A60C0631846FEF732FD0346032B0AD114F06B
S31508021A70ABF903460221184614F0E1FD36481AF07E
S31508021A801DF803E031481AF019F844E1C3E07B680F
S31508021A9003F5806309223149184634F067FB034689
S31508021AA0002B40F095807B6803F580631846FEF7A5
S31508021AB00DFD0346092B40F08B807B6803F5C06356
S31508021AC01A781C4B1B78D31A002B08D17B6803F5AE
S31508021AD0C0631846FEF7FAFC0346012B13D07B684F
S31508021AE003F5C06302221449184634F03FFB034645
S31508021AF0002B37D17B6803F5C0631846FEF7E6FC70
S31508021B000346022B2ED114F05FF903460421184628
S31508021B1014F078FD124819F0D1FF58E088970508A5
S31508021B208C970508A4970508E497050828980508D8
S31508021B303498050840980508449805084898050801
S31508021B40789805087C98050880980508B0980508CD
S31508021B50C4980508D098050800990508309905081B
S31508021B603C9905087B6803F5C0631A786B4B1B78AA
S31508021B70D31A002B08D17B6803F5C0631846FEF713
S31508021B80A5FC0346012B13D07B6803F5C063032229
S31508021B906349184634F0EAFA0346002B13D17B68E8
S31508021BA003F5C0631846FEF791FC0346032B0AD1D8
S31508021BB014F00AF903460421184614F040FD594860
S31508021BC019F07CFF03E0584819F078FFA3E022E0F9
S31508021BD07B6803F580631A78544B1B78D31A002B5B
S31508021BE015D17B6803F580631846FEF76FFC03463A
S31508021BF0012B0CD14E4819F061FF4E4819F05EFFD1
S31508021C004D4819F05BFF4D4819F058FF03E0464866
S31508021C1019F054FF7FE07EE07B6803F50073092222
S31508021C204749184634F0A2FA0346002B6FD17B685F
S31508021C3003F500731846FEF749FC0346092B66D1DD
S31508021C407B6803F580631A783E4B1B78D31A002B00
S31508021C5008D17B6803F580631846FEF737FC03460E
S31508021C60012B13D07B6803F5806302223649184696
S31508021C7034F07CFA0346002B13D17B6803F58063A4
S31508021C801846FEF723FC0346022B0AD114F09CF8E9
S31508021C9003460821184614F0B5FC2C4819F00EFF25
S31508021CA034E07B6803F580631A781C4B1B78D31AD9
S31508021CB0002B08D17B6803F580631846FEF706FCFD
S31508021CC00346012B13D07B6803F58063032214496C
S31508021CD0184634F04BFA0346002B13D17B6803F5FA
S31508021CE080631846FEF7F2FB0346032B0AD114F06B
S31508021CF06BF803460821184614F0A1FC144819F09B
S31508021D00DDFE03E0084819F0D9FE04E003E00648C0
S31508021D1019F0D4FE00BF1037BD4680BD7898050875
S31508021D207C9805086C990508B098050888970508EF
S31508021D309C990508C0990508F0990508209A05088E
S31508021D40509A050840980508449805085C9A0508BB
S31508021D50889A050890B59BB000AFF8600B467A6082
S31508021D60FB720023FB6500237B660023BB657B6849
S31508021D7003F500730522B249184634F0F7F903460B
S31508021D80002B12D17B6803F500731846FEF79EFBFB
S31508021D900346052B09D1AB4B01221A70AA4819F042
S31508021DA08DFE06F0B9FD00F051BC7B6803F50073A1
S31508021DB00522A649184634F0D9F90346002B12D152
S31508021DC07B6803F500731846FEF780FB0346052B6E
S31508021DD009D19C4B01221A709D4819F06FFE06F034
S31508021DE0E1FD00F033BC7B6803F5007305229949CF
S31508021DF0184634F0BBF90346002B12D17B6803F56B
S31508021E0000731846FEF762FB0346052B09D18D4B74
S31508021E1001221A70904819F051FE06F0AFFD00F043
S31508021E2015BC7B6803F5007305228C49184634F005
S31508021E309DF90346002B11D17B6803F500731846FA
S31508021E40FEF744FB0346052B08D17E4B01221A7086
S31508021E50834819F033FE06F0D7FDF7E37B6803F5EE
S31508021E60007308227F49184634F080F90346002B8E
S31508021E7010D17B6803F500731846FEF727FB034665
S31508021E80082B07D106F036FD53EC102B764819F0CD
S31508021E9015FEDBE37B6803F50073082273491846CF
S31508021EA034F064F90346002B26D17B6803F50073E8
S31508021EB01846FEF70BFB0346082B1DD1614B012280
S31508021EC01A707B6803F58063184633F045F8F8659F
S31508021ED0FB6D002B0CDBFB6D642B09DCF96D64488A
S31508021EE019F0ECFDFB6DDBB2184606F07DFCADE39E
S31508021EF0604819F0E3FDA9E37B6803F5007308223D
S31508021F005D49184634F032F90346002B13D17B6833
S31508021F1003F500731846FEF7D9FA0346082B0AD1C9
S31508021F20564819F0CBFD0CF0C9F90346FE211846AE
S31508021F300CF05BFA8AE3FB7A032B40F260837B6838
S31508021F4003F5007303224E49184634F00FF9034687
S31508021F50002B4CD17B6803F500731846FEF7B6FAD8
S31508021F600346032B43D17B6803F58063184632F098
S31508021F70F3FFF865FB7A032B07D97B6803F5C06381
S31508021F80184632F0E9FF786601E0FF237B66FB6DAF
S31508021F90002B27DBFB6D0F2B24DCF96D394819F072
S31508021FA08DFD0CF08BF90246FB6DDBB21946104625
S31508021FB00CF01BFA7B6E002B0CDB7B6E0F2B09DCFD
S31508021FC00CF07CF902467B6EDBB2194610460CF021
S31508021FD029FA0BE00CF072F90346FF2118460CF0B9
S31508021FE021FA03E0234819F069FD2FE32EE37B6803
S31508021FF003F5007306222449184634F0B7F8034657
S31508022000002B40F077827B6803F500731846FEF7CB
S315080220105DFA0346062B40F06D827B6803F5806302
S31508022020184632F099FFF865FB7A032B2ED97B689E
S3150802203003F5C063184632F08FFF786628E000BFC2
S31508022040B49A0508228F0020BC9A0508D09A05087A
S31508022050D89A0508EC9A0508F49A0508089B050813
S31508022060109B0508249B0508309B0508449B050818
S31508022070509B0508B0980508689B0508749B0508D7
S31508022080949B0508989B0508B49B0508FF237B6665
S31508022090FB6D002BC0F22982FB6D072B00F325820C
S315080220A0F96DC44819F00AFD7B6E002BC0F2148242
S315080220B07B6E0F2B00F310827B6E0C2B00F21482C0
S315080220C001A252F823F000BFFD200208E924020803
S315080220D0E9240208E9240208EF210208E924020891
S315080220E0E9240208E9240208E1220208E92402088E
S315080220F0E9240208E9240208D9230208FB6D002B09
S315080221000BD10CF0DBF8044607200CF06BFC0346F7
S31508022110194620460CF069F9D6E1FB6D012B0BD165
S315080221200CF0CCF8044607200CF0E6FC03461946E8
S3150802213020460CF05AF9C7E1FB6D022B0BD10CF0C5
S31508022140BDF8044607200CF035FD0346194620461D
S315080221500CF04BF9B8E1FB6D032B0BD10CF0AEF882
S31508022160044607200CF084FD0346194620460CF067
S315080221703CF9A9E1FB6D042B0BD10CF09FF8044640
S3150802218007200CF0D3FD0346194620460CF02DF91C
S315080221909AE1FB6D052B0BD10CF090F8044607204B
S315080221A00CF022FE0346194620460CF01EF98BE176
S315080221B0FB6D062B0BD10CF081F8044607200CF0B8
S315080221C071FE0346194620460CF00FF97CE1FB6DB9
S315080221D0072B40F079810CF071F8044607200CF0C1
S315080221E0BFFE0346194620460CF0FFF86CE1FB6D6C
S315080221F0002B0BD10CF062F8044605200CF0F2FB1A
S315080222000346194620460CF0F0F85FE1FB6D012BF8
S315080222100BD10CF053F8044605200CF06DFC03466E
S31508022220194620460CF0E1F850E1FB6D022B0BD162
S315080222300CF044F8044605200CF0BCFC034619468B
S3150802224020460CF0D2F841E1FB6D032B0BD10CF0C2
S3150802225035F8044605200CF00BFD034619462046C0
S315080222600CF0C3F832E1FB6D042B0BD10CF026F807
S31508022270044605200CF05AFD0346194620460CF082
S31508022280B4F823E1FB6D052B0BD10CF017F80446C5
S3150802229005200CF0A9FD0346194620460CF0A5F8C0
S315080222A014E1FB6D062B0BD10CF008F80446052049
S315080222B00CF0F8FD0346194620460CF096F805E19F
S315080222C0FB6D072B40F002810BF0F8FF0446052050
S315080222D00CF046FE0346194620460CF086F8F5E051
S315080222E0FB6D002B0BD10BF0E9FF044608200CF01E
S315080222F079FB0346194620460CF077F8E8E0FB6DB1
S31508022300012B0BD10BF0DAFF044608200CF0F4FB84
S315080223100346194620460CF068F8D9E0FB6D022BF5
S315080223200BD10BF0CBFF044608200CF043FC034606
S31508022330194620460CF059F8CAE0FB6D032B0BD15F
S315080223400BF0BCFF044608200CF092FC0346194623
S3150802235020460CF04AF8BBE0FB6D042B0BD10BF0C0
S31508022360ADFF044608200CF0E1FC03461946204658
S315080223700CF03BF8ACE0FB6D052B0BD10BF09EFF86
S31508022380044608200CF030FD0346194620460CF098
S315080223902CF89DE0FB6D062B0ED10BF08FFF044641
S315080223A008200CF07FFD0346194620460CF01DF85E
S315080223B08EE000BF989B0508FB6D072B40F08880CE
S315080223C00BF07CFF044608200CF0CAFD03461946AA
S315080223D020460CF00AF87BE0FB6D002B0BD10BF0C4
S315080223E06DFF044603200CF0FDFA03461946204603
S315080223F00BF0FBFF6EE0FB6D012B0BD10BF05EFFC2
S31508022400044603200CF078FB0346194620460BF0D7
S31508022410ECFF5FE0FB6D022B0BD10BF04FFF04467E
S3150802242003200CF0C7FB0346194620460BF0DDFFD6
S3150802243050E0FB6D032B0BD10BF040FF0446032043
S315080224400CF016FC0346194620460BF0CEFF41E077
S31508022450FB6D042B0BD10BF031FF044603200CF065
S3150802246065FC0346194620460BF0BFFF32E0FB6DBA
S31508022470052B0BD10BF022FF044603200CF0B4FC0B
S315080224800346194620460BF0B0FF23E0FB6D062BE8
S315080224900BD10BF013FF044603200CF003FD034691
S315080224A0194620460BF0A1FF14E0FB6D072B11D14C
S315080224B00BF004FF044603200CF052FD03461946AE
S315080224C020460BF092FF05E000BF0DE000BF0BE0CF
S315080224D000BF09E000BF07E00BF0F0FE0346FF214C
S315080224E018460BF09FFF04E003E05A4819F0E6FA93
S315080224F0ACE0ABE07B6803F5007303225649184645
S3150802250033F034FE0346002B75D17B6803F500735E
S315080225101846FDF7DBFF0346032B6CD17B6803F5F0
S31508022520806304224D49184633F020FE0346002BE9
S3150802253040F08B807B6803F580631846FDF7C6FF7B
S315080225400346042B40F081807B6803F5C063184676
S3150802255032F002FD78667B6803F50063184632F0AE
S31508022560FBFCB865BA6D796E3D4819F0A7FA07F112
S315080225705403012118462AF080F9002387F86330AC
S31508022580BB6DDAB27B6EDBB2D31ADBB20133DBB2D6
S3150802259087F8633097F96330002B05DC97F86330C8
S315080225A00833DBB287F8633097F8632007F15403E0
S315080225B0114618462AF07CF907F1540300211846F9
S315080225C02AF091F907F1100207F154031146184649
S315080225D02AF0D4FC07F1100318462AF000FC044638
S315080225E007F1100318462AF006FC03461946204648
S315080225F003F026FB29E0174819F060FA26E0FB7A71
S31508022600022B1ED17B6803F500730822154918466A
S3150802261033F0ACFD0346002B0FD17B6803F500733C
S315080226201846FDF753FF0346082B06D101200DF085
S315080226304DFC0D4819F042FA08E0064819F03EFA30
S3150802264004E0044819F03AFA00E000BF6C37BD46C8
S3150802265090BD00BFB0980508BC9B0508C09B05083D
S31508022660C89B0508F49B0508009C050880B584B03C
S3150802267000AFF8600B467A60FB7205F0C7FF0346A7
S31508022680184605F0FBFF0346012B03D12A4819F029
S3150802269015FA02E0294819F011FA05F0B7FF0346C0
S315080226A00021184606F011F80346012B03D12448E7
S315080226B019F004FA02E0234819F000FA05F0A6FF19
S315080226C003460121184606F000F80346012B03D1FA
S315080226D01D4819F0F3F902E01C4819F0EFF905F064
S315080226E095FF03460221184605F0EFFF0346012B24
S315080226F003D1174819F0E2F902E0164819F0DEF993
S3150802270005F084FF03460321184605F0DEFF03465B
S31508022710012B03D1104819F0D1F902E00F4819F03C
S31508022720CDF90BF08EFE034619460D4819F0C6F987
S3150802273000BF1037BD4680BD189C0508309C0508A9
S31508022740489C0508649C0508809C05089C9C05080D
S31508022750B89C0508D49C0508F09C05080C9D05083C
S31508022760289D050880B584B000AFF8600B467A60EC
S31508022770FB7205F04BFF03460021184605F0F3FFEE
S315080227800346012B03D1304819F098F902E02F4885
S3150802279019F094F905F03AFF03460121184605F0A7
S315080227A0E2FF0346012B03D1294819F087F902E013
S315080227B0284819F083F905F029FF0346022118462D
S315080227C005F0D1FF0346012B03D1234819F076F908
S315080227D002E0224819F072F905F018FF03460321B0
S315080227E0184605F0C0FF0346012B03D11C4819F011
S315080227F065F902E01B4819F061F905F007FF03467F
S315080228000421184605F0AFFF0346012B03D11648EB
S3150802281019F054F902E0154819F050F905F0F6FED8
S3150802282003460521184605F09EFF0346012B03D1F0
S315080228300F4819F043F903E00E4819F03FF900BFB3
S315080228401037BD4680BD00BF489D0508589D05083E
S31508022850689D0508789D0508889D0508989D0508C0
S31508022860A89D0508B89D0508C89D0508D89D0508B0
S31508022870E89D0508F89D05082DE9F0418EB002AFDE
S31508022880F8600B467A60FB7213F09EFA0346184606
S3150802289013F0CFFAF8620023BB6200237B6200239F
S315080228A03B620023FB610023BB6100237B617B68DB
S315080228B003F5007304227049184633F057FC0346A1
S315080228C0002B0FD17B6803F500731846FDF7FEFD52
S315080228D00346042B06D1694819F0F0F8F86AFEF7A0
S315080228E087FD07E27B6803F50073042264491846EC
S315080228F033F03CFC0346002B56D17B6803F5007384
S315080229001846FDF7E3FD0346042B4DD1F86AFEF798
S31508022910A5FD034619465B4819F0D0F8F86AFEF792
S31508022920B7FD03461946584819F0C8F80021F86A4F
S31508022930FEF7C9FD03461D460121F86AFEF7C3FDE7
S3150802294003461E460221F86AFEF7BDFD034698466F
S315080229500321F86AFEF7B7FD03461C460421F86A06
S31508022960FEF7B1FD034601930094434632462946D3
S31508022970464819F0A3F8F86AFEF7D9FD0346194640
S31508022980434819F09BF8F86AFEF7DDFD0346194637
S31508022990404819F093F8F86AFEF7F0FD034619461F
S315080229A03D4819F08BF8A5E17B6803F500731122FF
S315080229B03A49184633F0DAFB0346002B20D17B68E6
S315080229C003F500731846FDF781FD0346112B17D14F
S315080229D07B6803F58063184632F0BEFAB862B96AB4
S315080229E02F4819F06BF8BB6A002B05DDBB6A19463E
S315080229F0F86AFEF73FFD7DE12A4819F05FF879E1AA
S31508022A007B6803F500730E222749184633F0AEFB9E
S31508022A100346002B4ED17B6803F500731846FDF773
S31508022A2055FD03460E2B45D17B6803F58063184690
S31508022A3032F092FAB862BB6A002B0AD1B96A1B480D
S31508022A4019F03CF8BB6ADBB21946F86AFEF72CFDA8
S31508022A5050E1BB6A012B0AD1B96A154819F02EF85A
S31508022A60BB6ADBB21946F86AFEF71EFD42E10D485B
S31508022A7019F024F83EE100BF089E0508109E0508D5
S31508022A80249E05082C9E0508589E0508949E05084E
S31508022A90C49E0508F49E05083C9F05085C9F050828
S31508022AA0709F0508B0980508A09F0508B09F0508FD
S31508022AB0E89F05087B6803F500730A228F491846C2
S31508022AC033F054FB0346002B40F098807B6803F5ED
S31508022AD000731846FDF7FAFC03460A2B40F08E806F
S31508022AE07B6803F58063184632F036FA78627B68AB
S31508022AF003F5C063184632F02FFA38627B6803F58D
S31508022B000063184632F028FAF8617B6803F52063F9
S31508022B10184632F021FAB8617B6803F54063184615
S31508022B2032F01AFA78617B6A002B02D07B6A012B93
S31508022B3060D13B6A002B02D03B6A012B5AD1FB6952
S31508022B40002B02D0FB69012B54D1BB69002B02D0A2
S31508022B50BB69012B4ED17B69002B02D07B69012B05
S31508022B6048D17B6ADBB21A460021F86AFEF7C0FC36
S31508022B703B6ADBB21A460121F86AFEF7B9FCFB6921
S31508022B80DBB21A460221F86AFEF7B2FCBB69DBB26F
S31508022B901A460321F86AFEF7ABFC7B69DBB21A46D2
S31508022BA00421F86AFEF7A4FC0021F86AFEF78BFCFA
S31508022BB003461D460121F86AFEF785FC03461E46B2
S31508022BC00221F86AFEF77FFC034698460321F86A53
S31508022BD0FEF779FC03461C460421F86AFEF773FCE5
S31508022BE0034601930094434632462946444818F060
S31508022BF065FF7FE0434818F061FF7BE07B6803F5D9
S31508022C00007307224049184633F0B0FA0346002BF0
S31508022C1027D17B6803F500731846FDF757FC034670
S31508022C20072B1ED17B6803F58063184632F094F9A8
S31508022C30B862BB6A002B02D0BB6A002B0DDDBB6AE9
S31508022C40032B0ADCB96A314818F038FFBB6ADBB2D3
S31508022C501946F86AFEF783FC4CE02D4818F02EFF59
S31508022C6048E07B6803F5007304222A49184633F0C4
S31508022C707DFA0346002B1AD17B6803F500731846C2
S31508022C80FDF724FC0346042B11D17B6803F5806308
S31508022C90184632F061F9B862B96A1F4818F00EFF91
S31508022CA0BB6ADBB21946F86AFEF774FC22E07B6857
S31508022CB003F500731A78194B1B78D31A002B15D112
S31508022CC07B6803F500731846FDF700FC0346012BE3
S31508022CD00CD1134818F0F2FE124818F0EFFE12480B
S31508022CE018F0ECFE114818F0E9FE03E0054818F062
S31508022CF0E5FE00BF3037BD46BDE8F08120A00508D5
S31508022D002CA00508B098050858A0050860A0050873
S31508022D1084A00508A4A00508ACA00508889705089C
S31508022D20D0A00508ECA0050808A1050828A10508F1
S31508022D3090B589B000AFF8600B467A60FB72002343
S31508022D40FB610023BB6100237B617B6803F500738B
S31508022D501A78A34B1B78D31A002B0FD17B6803F57D
S31508022D6000731846FDF7B2FB0346012B06D19D48B0
S31508022D7018F0A4FE9C4818F0A1FE91E37B6803F5BF
S31508022D80007303229949184633F0F0F90346002BDB
S31508022D9008D17B6803F500731846FDF797FB0346CF
S31508022DA0032B15D07B6803F5007307229049184652
S31508022DB033F0DCF90346002B40F06F837B6803F59A
S31508022DC000731846FDF782FB0346072B40F065831E
S31508022DD07B6803F580631A78814B1B78D31A002B1C
S31508022DE027D17B6803F580631846FDF76FFB034618
S31508022DF0012B1ED17F4818F061FE7F4818F05EFE4F
S31508022E007E4818F05BFE7E4818F058FE7D4818F09A
S31508022E1055FE7D4818F052FE7C4818F04FFE7C4855
S31508022E2018F04CFE7B4818F049FE7B4818F046FE1F
S31508022E3036E37B6803F5806304227849184633F043
S31508022E4095F90346002B08D17B6803F5806318467B
S31508022E50FDF73CFB0346042B11D07B6803F5806320
S31508022E601A786F4B1B78D31A002B31D17B6803F57E
S31508022E7080631846FDF72AFB0346012B28D17B6897
S31508022E8003F5C063184632F067F8F861FB69002B50
S31508022E9002DDFB69082B03DD624818F00FFEFFE22C
S31508022EA027F0A8FA0346184627F016FB034601330D
S31508022EB0DBB219465C4827F07DFCFB69DBB2194692
S31508022EC0594827F092FC5949574828F023F8D6E280
S31508022ED07B6803F5806303225549184633F046F9A1
S31508022EE00346002B08D17B6803F580631846FDF775
S31508022EF0EDFA0346032B11D07B6803F580631A7833
S31508022F004C4B1B78D31A002B31D17B6803F58063AF
S31508022F101846FDF7DBFA0346012B28D17B6803F531
S31508022F20C063184632F018F8F861FB69002B02DD17
S31508022F30FB69082B03DD3B4818F0C0FDB0E227F019
S31508022F4059FA0346184627F0C7FA03460133DBB295
S31508022F501946394827F056FBFB69DBB2194636484B
S31508022F6027F06BFB3149344827F02BFF87E27B6851
S31508022F7003F5806309223149184633F0F7F8034608
S31508022F80002B08D17B6803F580631846FDF79EFA85
S31508022F900346092B11D07B6803F580631A78284B00
S31508022FA01B78D31A002B4FD17B6803F5806318462A
S31508022FB0FDF78CFA0346012B46D127F01BFA034686
S31508022FC0184627F089FA03460133DBB219461D482B
S31508022FD027F0C8FC15491B4828F045F84FE200BF00
S31508022FE08897050860A1050874A105088CA105083B
S31508022FF090A1050898A10508A8A10508C4A1050875
S31508023000DCA10508F0A1050810A2050828A20508F2
S3150802301054A2050880A20508BCA20508DCA2050878
S3150802302078980508E4A20508348F0020488F002006
S3150802303004A3050840980508388F002008A3050848
S3150802304014A305083C8F00207B6803F580630822D9
S315080230509D49184633F08AF80346002B08D17B6847
S3150802306003F580631846FDF731FA0346082B11D09B
S315080230707B6803F580631A78944B1B78D31A002B66
S3150802308031D17B6803F580631846FDF71FFA0346BC
S31508023090012B28D17B6803F5C063184631F05CFF23
S315080230A0F861FB69002B02DBFB690A2B03DD884802
S315080230B018F004FDF4E127F09DF90346184627F0B7
S315080230C00BFA03460133DBB21946824827F02EFA79
S315080230D0FB69DBB219467F4827F043FA7E497D48E9
S315080230E027F09EFDCBE17B6803F580630C227B49C2
S315080230F0184633F03BF80346002B08D17B6803F5E4
S3150802310080631846FDF7E2F903460C2B11D07B685B
S3150802311003F580631A78724B1B78D31A002B1AD1DF
S315080231207B6803F580631846FDF7D0F90346012B41
S3150802313011D127F05FF90346184627F0CDF9034661
S315080231400133DBB21946674827F026FA6249654811
S3150802315027F0C9FD93E17B6803F58063072262497C
S31508023160184633F003F80346002B08D17B6803F5AB
S3150802317080631846FDF7AAF90346072B11D07B6828
S3150802318003F580631A78594B1B78D31A002B3ED164
S315080231907B6803F580631846FDF798F90346012B09
S315080231A035D17B6803F5C063184631F0D5FEF86160
S315080231B07B6803F50063184631F0CEFEB861FB69F9
S315080231C0002B02DDFB69082B03DD494818F076FC63
S315080231D066E127F00FF90346184627F07DF90346FC
S315080231E00133DBB21946434800F0F0FFFB69DBB254
S315080231F01946404801F005F8BB69DBB219463D4855
S3150802320001F01AF834493B4801F085F937E17B6841
S3150802321003F580630A223849184632F0A7FF0346A7
S31508023220002B08D17B6803F580631846FDF74EF933
S3150802323003460A2B11D07B6803F580631A782F4B55
S315080232401B78D31A002B5FD17B6803F58063184677
S31508023250FDF73CF90346012B56D17B6803F5C0639B
S31508023260184631F079FEF8617B6803F50063184663
S3150802327031F072FEB861FB69002B02DBFB69022B97
S3150802328003DD1F4818F01AFC0AE127F0B3F80346D3
S31508023290184627F021F903460133DBB219461948C5
S315080232A000F0E5FFFB69DBB21946164800F0FAFFA3
S315080232B0BB69DBB21946134801F00FF806491148F3
S315080232C001F09FF9DBE000BFF49B050818A3050887
S315080232D01CA30508408F0020488F002040A305083C
S315080232E050A30508448F002054A305085CA30508CB
S315080232F0E4A20508248F002060A305086CA305082C
S3150802330070A30508288F00207B6803F580630D22C9
S315080233106549184632F02AFF0346002B08D17B6816
S3150802332003F580631846FDF7D1F803460D2B11D035
S315080233307B6803F580631A785C4B1B78D31A002BDB
S315080233404BD17B6803F580631846FDF7BFF8034641
S31508023350012B42D17B6803F5C063184631F0FCFDA8
S31508023360F8617B6803F50063184631F0F5FDB8612C
S315080233707B6803F52063184631F0EEFD7861FB6938
S31508023380002B02DDFB69022B03DD494818F096FB88
S3150802339086E027F02FF80346184627F09DF80346DD
S315080233A00133DBB21946434800F0B2FFFB69DBB2D0
S315080233B01946404800F0C7FFBB69DBB219463D48CB
S315080233C000F0DCFF7B69DBB219463A4800F0F1FFF0
S315080233D03949384801F08BF951E07B6803F5806377
S315080233E00B223649184632F0C1FE0346002B08D195
S315080233F07B6803F580631846FDF768F803460B2BCE
S3150802340011D07B6803F580631A782D4B1B78D31A83
S31508023410002B31D17B6803F580631846FDF756F811
S315080234200346012B28D17B6803F5C063184631F0A1
S3150802343093FDF861FB69002B02DBFB69012B03DDB7
S31508023440204818F03BFB2BE026F0D4FF034618462B
S3150802345027F042F803460133DBB219461A4800F050
S31508023460F9FFFB69DBB21946174801F00EF8124953
S31508023470154801F0D5F902E0144818F01FFB0E486A
S315080234802EF0A4F904460C482EF0ACF90346DBB23A
S315080234901946204606F0FEF902E00D4818F00EFB22
S315080234A02437BD4690BD00BF90A30508A0A3050812
S315080234B0A4A305082C8F0020488F0020C0A3050866
S315080234C0CCA30508D0A30508308F0020B0980508BC
S315080234D0F0A3050880B586B000AFF8600B467A609F
S315080234E0FB7200237B617B6803F500731A784C4BE9
S315080234F01B78D31A002B2AD17B6803F5007318466A
S31508023500FCF7E4FF0346012B21D17B6803F58063B0
S31508023510184631F021FD78617B69642B13DC414B37
S3150802352001221A707969404818F0C8FA3F4B1B689D
S315080235307A699A6304213D4820F014FD08213B4824
S3150802354020F070FE68E03A4818F0B8FA64E07B6842
S3150802355003F500731A78374B1B78D31A002B2AD136
S315080235607B6803F500731846FCF7B0FF0346012B88
S3150802357021D17B6803F58063184631F0EDFC78614A
S315080235807B69642B13DC274B01221A7079692A4856
S3150802359018F094FA254B1B687A69DA6304212348E2
S315080235A020F040FE0821214820F0DCFC34E02048C7
S315080235B018F084FA30E07B6803F500731A781F4B1B
S315080235C01B78D31A002B1CD17B6803F500731846A7
S315080235D0FCF77CFF0346012B13D1124B01221A700A
S315080235E0124B1B6863229A63104B1B686322DA63C9
S315080235F004210E4820F0B6FC08210C4820F0B2FC43
S315080236000AE0084B00221A700421084820F00AFE34
S315080236100821064820F006FE1837BD4680BD00BFC1
S3150802362008A40508C40402200CA405087005012094
S3150802363084A0050824A4050828A4050840A40508AA
S3150802364080B485B000AFF8600B467A60FB72044B13
S3150802365001221A7000BF1437BD465DF8047B704715
S31508023660C805022080B485B000AFF8600B467A60C0
S31508023670FB72044B01221A7000BF1437BD465DF86F
S31508023680047B7047C9050220B0B596B000AFF86052
S315080236900B467A60FB727B6803F5007304228B493A
S315080236A0184632F063FD0346002B08D17B6803F502
S315080236B000731846FCF70AFF0346042B13D07B68EF
S315080236C003F500731A78824B1B78D31A002B40F045
S315080236D0FA807B6803F500731846FCF7F7FE034683
S315080236E0012B40F0F0807B6803F580631A78794BEA
S315080236F01B78D31A002B0FD17B6803F58063184613
S31508023700FCF7E4FE0346012B06D1734818F0D6F9F6
S31508023710012387F85430B2E07B6803F580631A7890
S315080237206E4B1B78D31A002B0FD17B6803F5806387
S315080237301846FCF7CBFE0346012B06D1684818F05B
S31508023740BDF9022387F8543099E07B6803F5806354
S315080237501A78644B1B78D31A002B0FD17B6803F5B2
S3150802376080631846FCF7B2FE0346012B06D15E4873
S3150802377018F0A4F9032387F8543080E07B6803F530
S3150802378080631A78594B1B78D31A002B0FD17B68A2
S3150802379003F580631846FCF799FE0346012B06D10A
S315080237A0534818F08BF9042387F8543067E07B688E
S315080237B003F580631A784F4B1B78D31A002B0FD167
S315080237C07B6803F580631846FCF780FE0346012BE7
S315080237D006D1494818F072F9052387F854304EE0A5
S315080237E07B6803F580631A78444B1B78D31A002B3F
S315080237F00FD17B6803F580631846FCF767FE03461C
S31508023800012B06D13E4818F059F9062387F8543099
S3150802381035E07B6803F580631A783A4B1B78D31A2E
S31508023820002B0FD17B6803F580631846FCF74EFE22
S315080238300346012B06D1344818F040F9072387F8C6
S3150802384054301CE07B6803F580631A782F4B1B788B
S31508023850D31A002B0FD17B6803F580631846FCF751
S3150802386035FE0346012B06D1294818F027F9082305
S3150802387087F8543003E0274818F020F923E097F830
S315080238805430002B1FD097F85430082B1BD807F159
S31508023890100207F154031146184628F0E2FE29F0F1
S315080238A081FE044607F11003184628F07FFC0546F8
S315080238B007F11003184628F085FC03461A462946DE
S315080238C0204630F0B1FF5837BD46B0BDDCA2050828
S315080238D0789805084098050844A4050814A305081D
S315080238E068A4050818A305088CA4050850A30508AA
S315080238F0B0A405085CA30508D4A405086CA30508AA
S31508023900F8A40508A0A305081CA50508CCA3050864
S3150802391040A50508B098050880B584B000AFF860E0
S315080239200B467A60FB727B6803F500731A782E4B96
S315080239301B78D31A002B0FD17B6803F50073184640
S31508023940FCF7C4FD0346012B06D1284B1B6832221D
S31508023950DA6305F0B9F842E07B6803F500731A7872
S31508023960234B1B78D31A002B0FD17B6803F5007300
S315080239701846FCF7ABFD0346012B06D11B4B1B6809
S3150802398032221A6405F0AEF829E07B6803F5007363
S315080239901A78184B1B78D31A002B0BD17B6803F5C0
S315080239A000731846FCF792FD0346012B02D105F077
S315080239B0A7F814E07B6803F500731A780E4B1B7898
S315080239C0D31A002B0BD17B6803F500731846FCF754
S315080239D07DFD0346012B02D105F0A8F8FFE700BFDB
S315080239E01037BD4680BD00BF08A40508240501207E
S315080239F024A4050864A5050868A5050880B586B047
S31508023A0000AFF8600B467A60FB724FF496737B61DF
S31508023A107B6803F5007304224F49184632F0A6FB69
S31508023A200346002B2BD17B6803F500731846FCF777
S31508023A304DFD0346042B22D1484B1B686322DA63E9
S31508023A4005F090F809E0082145481AF025F80346DA
S31508023A50012B08D10A2025F09DFB7B695A1E7A6143
S31508023A60002BF0D100E000BF7B69002B02D13D4854
S31508023A7018F024F805F084F805F098F867E07B68F2
S31508023A8003F5007305223849184632F06FFB0346E0
S31508023A90002B2BD17B6803F500731846FCF716FD3D
S31508023AA00346052B22D12D4B1B6863221A6405F0A7
S31508023AB04BF809E004212A4819F0EEFF0346012BC8
S31508023AC008D10A2025F066FB7B695A1E7A61002B0B
S31508023AD0F0D100E000BF7B69002B02D1234817F022
S31508023AE0EDFF05F04DF805F061F830E07B6803F567
S31508023AF0007304221E49184632F038FB0346002B8F
S31508023B0025D17B6803F500731846FCF7DFFC0346EC
S31508023B10042B1CD10421124819F0BEFF0346012BBF
S31508023B2003D1144817F0CAFF02E0134817F0C6FF7C
S31508023B3008210B4819F0B0FF0346012B03D10F48A1
S31508023B4017F0BCFF03E00E4817F0B8FFFFE700BF07
S31508023B501837BD4680BD00BF6CA50508BC05012007
S31508023B600014024274A505088CA5050894A5050843
S31508023B70ACA50508B4A50508CCA50508E4A505085D
S31508023B80F8A5050880B586B000AFF8600B467A60DE
S31508023B90FB720023FB7500233B617B6803F5007308
S31508023BA01A78604B1B78D31A002B16D17B6803F55B
S31508023BB000731846FCF78AFC0346012B0DD15A4BB3
S31508023BC001221A70594B1B6863229A6304F0FCFFA0
S31508023BD03969574817F072FF99E07B6803F5007355
S31508023BE01A78544B1B78D31A002B16D17B6803F527
S31508023BF000731846FCF76AFC0346012B0DD14A4BA3
S31508023C0001221A70494B1B6863225A6304F0EAFFC1
S31508023C103969494817F052FF79E07B6803F5007362
S31508023C2004224649184632F0A1FA0346002B11D15E
S31508023C307B6803F500731846FCF748FC0346042B19
S31508023C4008D1394B01221A7004F0DAFF3C4817F002
S31508023C5035FF5CE07B6803F5007304223949184690
S31508023C6032F084FA0346002B11D17B6803F5007300
S31508023C701846FCF72BFC0346042B08D12A4B0122D3
S31508023C801A7004F0D3FF2E4817F018FF3FE07B683E
S31508023C9003F5007304222C49184632F067FA0346E4
S31508023CA0002B13D17B6803F500731846FCF70EFC4C
S31508023CB00346042B0AD109F0E9FF034602211846F6
S31508023CC00AF02EF8214817F0F9FE20E07B6803F582
S31508023CD0007302221E49184632F048FA0346002BA0
S31508023CE013D17B6803F500731846FCF7EFFB03460E
S31508023CF0022B0AD109F0CAFF0346032118460AF025
S31508023D000FF8144817F0DAFE01E00123FB75FB7D74
S31508023D10002B02D0104817F0D1FE00BF1837BD4657
S31508023D2080BD00BF08A405084A900020BC050120F2
S31508023D3010A6050824A405082CA6050848A6050801
S31508023D4050A6050870A6050878A6050880A60508DF
S31508023D509CA60508A0A60508B098050890B585B0E2
S31508023D6000AF78600023BB730023FB734FF4A052A5
S31508023D700021204832F0F2F907F10E030A221D4902
S31508023D80786827F075FC0346012B2ED10023FB73B6
S31508023D9028E0FB7B4FF48E7202FB03F3164A1344A8
S31508023DA09C1C1448FCF792FB03461A461149204606
S31508023DB032F0DCF90346002B11D1FB7B0E4A4FF495
S31508023DC08E7101FB03F3134418331B68B97B094A46
S31508023DD000209847094817F071FE012306E0FB7B8D
S31508023DE00133FB73FB7B102BD3D9002318461437F8
S31508023DF0BD4690BD4079002000000020689705085E
S31508023E0080B582B000AF0346FB71FB790D2B24D136
S31508023E104F4B00221A704F4817F050FE4E4B1B7834
S31508023E20002B16D04D48FFF799FF0346012B08D100
S31508023E30F02200214A4832F091F94849484832F0BE
S31508023E402EFA454B00221A70F0220021434832F01E
S31508023E5085F9444817F032FE76E0FB790A2B03D13E
S31508023E603B4B00221A706FE0FB791B2B03D1384BB0
S31508023E7001221A7068E0FB795B2B07D1344B1B7859
S31508023E80012B03D1324B02221A705DE0FB79412BDA
S31508023E901FD12F4B1B78022B1BD12D4B00221A70D8
S31508023EA02D4B1B78002B4FD12D492F4817F006FEB4
S31508023EB02B48FCF70BFB0346DAB2274B1A70F022A3
S31508023EC00021264832F04AF92549244832F0E7F912
S31508023ED03AE0FB79082B02D0FB797F2B16D11C4BD3
S31508023EE000221A701C4B1B78002B2DD01A4B1B78FC
S31508023EF0013BDAB2184B1A70174B1B781A46174B46
S31508023F0000219954194817F0D9FD1DE0124B1B7868
S31508023F105A1CD1B2104A11701946104AFB795354E9
S31508023F200D4B1A78124BA3FB0213D9090B461B0138
S31508023F305B1A1B01D31ADAB2074B1A70FB791946B8
S31508023F400C4817F0BBFDFFE700BF0837BD4680BD2A
S31508023F504B90002068970508208F0020308E00209D
S31508023F60408D0020BCA6050860970508C0A605086E
S31508023F7089888888C4A6050880B58EB008AF786097
S31508023F8000237B617B683B6106220E21554817F0A8
S31508023F9005FE07F10C0100234FF40062386925F08B
S31508023FA08FFE0346002B01D0022397E0FB68B0225E
S31508023FB0069201220592002204920A2203920A22FA
S31508023FC002924FF40062019200930023464A47493F
S31508023FD0474826F0BBF80346002B01D00E237DE0A6
S31508023FE0342300224349444825F07EFF0346002B2A
S31508023FF001D01C2372E0786817F042FB786817F044
S315080240009DFB786812F0DCFF786814F0D7F97868B7
S3150802401012F0B0FD342300223849394825F064FFEE
S315080240200346002B01D01C2358E0342300223549CD
S31508024030354825F059FF0346002B01D01C234DE0D5
S31508024040342300223149324825F04EFF0346002B1D
S3150802405001D01C2342E0342300222E492E4825F0A3
S3150802406043FF0346002B01D01C2337E034230022EA
S315080240702A492B4825F038FF0346002B01D01C237A
S315080240802CE0342300222749274825F02DFF034632
S31508024090002B01D01C2321E0342300222349244883
S315080240A025F022FF0346002B01D01C2316E03423F9
S315080240B000222049204825F017FF0346002B01D08D
S315080240C01C230BE0342300221C491D4825F00CFF53
S315080240D00346002B01D01C2300E07B6918461837DB
S315080240E0BD4680BDD0A6050845410208E0A60508DA
S315080240F04C900020F0A60508FC90002000A70508B1
S31508024100309100201CA705086491002034A70508F1
S315080241109891002048A70508CC91002060A70508B9
S315080241200092002074A705083492002098A7050873
S3150802413068920020B0A705089C920020C4A705082B
S31508024140D092002080B584B000AF78607B68BB60EF
S315080241500023FB73134B1B780133DAB2114B1A7027
S31508024160104B1B78092B13D90E4B00221A7017F025
S31508024170EDFDFB7B032B05D106F086FAFB7B0133AB
S31508024180FB7305E0FB7B032B02D8FB7B0133FB7336
S31508024190BB68DBB2184617F0ABFD642024F0FAFFC1
S315080241A0D8E700BF0493002080B500AF24F092F848
S315080241B000BF80BD80B483B000AF78607B681B788F
S315080241C018460C37BD465DF8047B704780B483B049
S315080241D000AF78600B46FB707B68FA781A7000BFEE
S315080241E00C37BD465DF8047B704780B483B000AFD8
S315080241F078607B685B7818460C37BD465DF8047BA9
S31508024200704780B483B000AF78600B46FB707B685A
S31508024210FA785A7000BF0C37BD465DF8047B7047C2
S3150802422080B483B000AF78607B689B7818460C37F9
S31508024230BD465DF8047B704780B483B000AF7860F2
S315080242400B46FB707B68FA789A7000BF0C37BD463E
S315080242505DF8047B704780B483B000AF78607B68F2
S315080242601B7818460C37BD465DF8047B704780B448
S3150802427083B000AF78600B46FB707B68FA781A70D9
S3150802428000BF0C37BD465DF8047B704780B483B027
S3150802429000AF78607B685B7818460C37BD465DF8D8
S315080242A0047B704780B483B000AF78600B46FB701E
S315080242B07B68FA785A7000BF0C37BD465DF8047BF6
S315080242C0704780B483B000AF78607B689B781846E5
S315080242D00C37BD465DF8047B704780B483B000AFE7
S315080242E078600B46FB707B68FA789A7000BF0C37C9
S315080242F0BD465DF8047B704780B483B000AF786032
S315080243007B681B7818460C37BD465DF8047B7047F8
S3150802431080B483B000AF78600B46FB707B68FA788E
S315080243201A7000BF0C37BD465DF8047B704780B42F
S3150802433083B000AF78607B685B7818460C37BD4659
S315080243405DF8047B704780B483B000AF78600B4693
S31508024350FB707B68FA785A7000BF0C37BD465DF869
S31508024360047B704780B483B000AF78607B689B7823
S3150802437018460C37BD465DF8047B704780B483B097
S3150802438000AF78600B46FB707B68FA789A7000BFBC
S315080243900C37BD465DF8047B704780B483B000AF26
S315080243A078607B68DB7818460C37BD465DF8047B77
S315080243B0704780B483B000AF78600B46FB707B68A9
S315080243C0FA78DA7000BF0C37BD465DF8047B704791
S315080243D080B483B000AF78607B681B7818460C37C8
S315080243E0BD465DF8047B704780B483B000AF786041
S315080243F00B46FB707B68FA781A7000BF0C37BD460D
S315080244005DF8047B704780B483B000AF78607B6840
S315080244105B7818460C37BD465DF8047B704780B456
S3150802442083B000AF78600B46FB707B68FA785A70E7
S3150802443000BF0C37BD465DF8047B704780B483B075
S3150802444000AF78607B681B7818460C37BD465DF866
S31508024450047B704780B483B000AF78600B46FB706C
S315080244607B68FA781A7000BF0C37BD465DF8047B84
S31508024470704780B483B000AF78607B685B78184673
S315080244800C37BD465DF8047B704780B483B000AF35
S3150802449078600B46FB707B68FA785A7000BF0C3757
S315080244A0BD465DF8047B704780B483B000AF786080
S315080244B07B681B7818460C37BD465DF8047B704747
S315080244C080B483B000AF78600B46FB707B68FA78DD
S315080244D01A7000BF0C37BD465DF8047B704780B47E
S315080244E083B000AF78600B46FB707B6802337A684C
S315080244F012881344FA781A707B681B8801339AB2B9
S315080245007B681A807B681B88DBB218460C37BD4667
S315080245105DF8047B704780B582B000AF7860396079
S315080245204FF481720021386831F018FE602138682C
S31508024530FFF7D5FF7868FFF73DFE03461946386848
S31508024540FFF7CDFF7868FFF750FE0346194638682D
S31508024550FFF7C5FF7868FFF763FE03461946386812
S31508024560FFF7BDFF3B681B88DBB218460837BD4616
S3150802457080BD80B584B000AF786039600023FB73D4
S3150802458003220021386831F0E9FDFB7B5A1CFA73D5
S315080245901A467B6813441B7819463868FFF716FED5
S315080245A0FB7B5A1CFA731A467B6813441B78194616
S315080245B03868FFF726FEFB7B5A1CFA731A467B6895
S315080245C013441B7819463868FFF736FEFB7B1846F4
S315080245D01037BD4680BD80B582B000AF78603960BD
S315080245E04FF481720021386831F0B8FD60213868CD
S315080245F0FFF775FF3B681B88DBB218460837BD46CE
S3150802460080BD80B582B000AF786039604FF48172A0
S315080246100021386831F0A2FD70213868FFF75FFF84
S315080246207868FFF718FE034619463868FFF757FFFA
S315080246307868FFF72BFE034619463868FFF74FFFDF
S315080246407868FFF73EFE034619463868FFF747FFC4
S315080246503B681B88DBB218460837BD4680BD80B565
S3150802466084B000AF786039600023FB73032200210F
S31508024670386831F073FDFB7B5A1CFA731A467B685D
S3150802468013441B7819463868FFF7F1FDFB7B5A1C61
S31508024690FA731A467B6813441B7819463868FFF77B
S315080246A001FEFB7B5A1CFA731A467B6813441B7875
S315080246B019463868FFF711FEFB7B18461037BD46C8
S315080246C080BD80B582B000AF786039604FF48172E0
S315080246D00021386831F042FD70213868FFF7FFFE85
S315080246E03B681B88DBB218460837BD4680BD80B5D5
S315080246F082B000AF786039604FF481720021386861
S3150802470031F02CFD71213868FFF7E9FE7868FFF76A
S31508024710F3FD034619463868FFF7E1FE7868FFF7A6
S3150802472006FE034619463868FFF7D9FE7868FFF78A
S3150802473019FE034619463868FFF7D1FE7868FFF76F
S315080247402CFE034619463868FFF7C9FE3B681B88E4
S31508024750DBB218460837BD4680BD80B584B000AFC7
S31508024760786039600023FB7303220021386831F030
S31508024770F5FCFB7B5A1CFA731A467B6813441B78B2
S3150802478019463868FFF7C4FDFB7B5A1CFA731A46AA
S315080247907B6813441B7819463868FFF7D4FDFB7B00
S315080247A05A1CFA731A467B6813441B7819463868EA
S315080247B0FFF7E4FDFB7B5A1CFA731A467B6813441F
S315080247C01B7819463868FFF7F4FDFB7B1846103745
S315080247D0BD4680BD80B582B000AF786039604FF4BF
S315080247E081720021386831F0B9FC71213868FFF707
S315080247F076FE7868FFF7ECFD034619463868FFF738
S315080248006EFE7868FFF7FFFD034619463868FFF71C
S3150802481066FE3B681B88DBB218460837BD4680BD74
S3150802482080B582B000AF786039604FF4817200219A
S31508024830386831F093FC72213868FFF750FE7868C1
S31508024840FFF7FCFD034619463868FFF748FE786805
S31508024850FFF70FFE034619463868FFF740FE3B6826
S315080248601B88DBB218460837BD4680BD80B584B0C2
S3150802487000AF786039600023FB7302220021386892
S3150802488031F06CFCFB7B5A1CFA731A467B6813449C
S315080248901B7819463868FFF7DDFDFB7B5A1CFA734D
S315080248A01A467B6813441B7819463868FFF7EDFDEC
S315080248B0FB7B18461037BD4680BD80B582B000AF77
S315080248C0786039604FF481720021386831F046FC0D
S315080248D072213868FFF703FE3B681B88DBB218466D
S315080248E00837BD4680BD80B584B000AF78603960B0
S315080248F00023FB7301220021386831F02FFCFB7B71
S315080249005A1CFA731A467B6813441B781946386888
S31508024910FFF7D6FDFB7B18461037BD4680BD80B52E
S3150802492082B000AF786039604FF48172002138682E
S3150802493031F014FC80213868FFF7D1FD3B681B88EB
S31508024940DBB218460837BD4680BD000080B400AF0A
S31508024950034B1B681846BD465DF8047B704700BFCB
S315080249600893002080B500AF4FF400620E490F4845
S3150802497026F0E8FE4FF400620D490E4826F0E2FEE4
S315080249804FF400720C490D4826F0DCFE4FF4006223
S315080249900B490C4826F0D6FE4FF400620A490B482A
S315080249A026F0D0FE00BF80BD1C9300200C93002089
S315080249B02C9B00201C9B002060A3002050A30020F3
S315080249C0A0A5002060A50020E0AD0020A0AD002033
S315080249D080B483B000AF78607B68002B01D10023D6
S315080249E046E07B68012B01D1012341E07B68022B5B
S315080249F001D102233CE07B68032B01D1032337E074
S31508024A007B68042B01D1042332E07B68052B01D194
S31508024A1005232DE07B68062B01D1062328E07B6857
S31508024A20072B01D1072323E07B68082B01D1082332
S31508024A301EE07B68092B01D80C2319E07B680A2B38
S31508024A4001D8102314E07B680B2B01D814230FE03E
S31508024A507B680C2B01D818230AE07B680D2B01D83A
S31508024A60202305E07B680E2B01D8302300E0402383
S31508024A7018460C37BD465DF8047B704780B483B090
S31508024A8000AF0346FB80FB88002B01D1002346E0DA
S31508024A90FB88012B01D1012341E0FB88022B01D1BE
S31508024AA002233CE0FB88032B01D1032337E0FB8872
S31508024AB0042B01D1042332E0FB88052B01D10523FF
S31508024AC02DE0FB88062B01D1062328E0FB88072B5D
S31508024AD001D1072323E0FB88082B01D108231EE016
S31508024AE0FB880C2B01D8092319E0FB88102B01D867
S31508024AF00A2314E0FB88142B01D80B230FE0FB884A
S31508024B00182B01D80C230AE0FB88202B01D80D2389
S31508024B1005E0FB88302B01D80E2300E00F23184648
S31508024B200C37BD465DF8047B7047000084B0B0B40C
S31508024B3000AF07F10C0484E80F00074B1D4607F186
S31508024B400C040FCC0FC50FCC0FC523682B6000BF12
S31508024B50BD46B0BC04B070472CA3002080B586B011
S31508024B6000AF78600B467B800023FB7500233B6110
S31508024B700023FB600023BB6000F0C2FD0346002B46
S31508024B800BD0444BD3F844323B61424BD3F8843AB8
S31508024B90FB607B681B68BB600AE03E4BD3F8443275
S31508024BA03B613C4BD3F8843AFB607B681B68BB606D
S31508024BB03A69BB689A4227D1364B93F86832002B7A
S31508024BC00AD1344BD3F850227B881344314AC2F8AF
S31508024BD050320123FB7558E02E4BB3F86C321A4655
S31508024BE07B881344B3F5006F0BDA2A4BB3F86C22B1
S31508024BF07B8813449AB2274BA3F86C220123FB75D0
S31508024C0043E00023FB7540E0FA68BB689A4227D165
S31508024C10204B93F8A83A002B0AD11E4BD3F8502200
S31508024C207B8813441B4AC2F850320223FB752CE0D8
S31508024C30184BB3F8AC3A1A467B881344B3F5006F9F
S31508024C400BDA144BB3F8AC2A7B8813449AB2114B8D
S31508024C50A3F8AC2A0223FB7517E00023FB7514E0C0
S31508024C603B69002B07D1242279680B4831F02DFBCA
S31508024C700123FB7509E0FB68002B06D1242279681B
S31508024C80064831F022FB0223FB75FB7D18461837CE
S31508024C90BD4680BD2CA3002070A50020B0AD002023
S31508024CA080B584B000AF03463960FB711346BB80FA
S31508024CB00023FB81FB79012B12D10023FB810AE039
S31508024CC0FB893A68134401221946124826F0E0FD88
S31508024CD0FB890133FB81FA89BB889A42F0D314E037
S31508024CE0FB79022B11D10023FB810AE0FB893A6882
S31508024CF0134401221946084826F0CAFDFB890133E6
S31508024D00FB81FA89BB889A42F0D300BF1037BD46A9
S31508024D1080BD00BF60A50020A0AD002080B582B08E
S31508024D2000AF0346FB71FB1D01221946034826F014
S31508024D30AFFD00BF0837BD4680BD00BF50A30020A7
S31508024D40F0B5C3B008AFF861B9617A61002387F894
S31508024D50E730F86917F0DBFCC7F8E000BF4B002222
S31508024D601A6084E0BD4B1B685A1CBC490A60B3F53D
S31508024D70FA7F7CD997F8E730013387F8E73007F1ED
S31508024D8068031946F86917F0F5FDBB6E3B61FA6EC2
S31508024D90FA60386FB8607B6FBA6FF96FD7F8800020
S31508024DA0D7F884407C60D7F88850D7F88C60D7F853
S31508024DB090400794069605957C68049403900291A0
S31508024DC001920093BB68FA683969A54816F076FE1F
S31508024DD0FB6F002B07D0FB691B689A69FB691B6886
S31508024DE022F001029A61F86917F091FCC7F8E0000F
S31508024DF0D7F8E010F86917F096FC984B00221A606B
S31508024E0010F0E2FF03460121184611F09FFB034604
S31508024E10002B02D0934816F051FE934B1B78022BB7
S31508024E202ED0914B01221A7007F1D8030221184697
S31508024E3027F033FF07F1940207F1D8031146184603
S31508024E4028F08DFA28F004FC044607F19403184664
S31508024E5027F0C5FF054607F19403184627F0CBFF4E
S31508024E6003461A46294620462FF0DEFC08E00721AB
S31508024E70F86917F0CFFD0346002B7FF473AF00E005
S31508024E8000BF7A69B969F86917F0FDFB0346002B7A
S31508024E903AD097F8E730013387F8E73010F094FFF5
S31508024EA003460121184611F051FB0346002B02D096
S31508024EB06E4816F003FE6C4B1B78012B24D06A4B06
S31508024EC001221A7007F1D8030121184627F0E5FED8
S31508024ED007F1940207F1D8031146184628F03FFA5B
S31508024EE028F0B6FB044607F19403184627F077FF25
S31508024EF0054607F19403184627F07DFF03461A462E
S31508024F00294620462FF090FC97F8E730002B28D147
S31508024F10554B1B78002B24D0534B00221A7007F1ED
S31508024F20D8030021184627F0B8FE07F1940207F1C4
S31508024F30D8031146184628F012FA28F089FB0446C7
S31508024F4007F19403184627F04AFF054607F194032A
S31508024F50184627F050FF03461A46294620462FF0E0
S31508024F6063FCF86900F026FB03461A46404B9A6032
S31508024F70F86900F0E9FA03463D4A1360F86900F059
S31508024F80FBFA03463A4A5360394B9B68002B1CD0FE
S31508024F9010F01AFF03460121184611F0D7FA034604
S31508024FA0002B0DD0324B1A68314B5B6807F1200093
S31508024FB0304931F03FF807F12003184616F07EFD16
S31508024FC02B4B9B68184600F03DFB0C2228492A48C1
S31508024FD031F0B4F80346002B36D0254B1B68DAB2FB
S31508024FE007F164031146184627F0DFFD204B5B687C
S31508024FF0DAB207F164031146184627F0F1FD1C4B95
S315080250009B68DAB207F164031146184627F003FED5
S3150802501007F1200207F164031146184628F049F9F8
S3150802502028F016FB044607F12003184627F0D7FE98
S31508025030054607F12003184627F0DDFE03461A4601
S31508025040294620462FF0F0FB0B4B094A07CA83E88C
S31508025050070000BFEC37BD46F0BD00BFFCB5002017
S31508025060ECA7050830A8050800B6002054A80508CC
S31508025070E0B5002078A80508ECB5002080B592B006
S3150802508000AF3B4640220021184631F067F800235C
S31508025090A7F8423000237B64B74826F0DDFB0346B7
S315080250A083F00103DBB2002B00F0E380B34B93F8E5
S315080250B06832002B5FD1B14BD3F850329AB2AF4B5C
S315080250C0A3F86C22AD4B0F22C3F8502210233B7073
S315080250D03B785AB2A94BB3F86C321B0A9BB25BB245
S315080250E003F00F035BB213435BB2DBB23B70A34B15
S315080250F0B3F86C32DBB27B703B4602333E2219466A
S315080251009D4826F000FC0346002B00F031814FF43F
S315080251107A719B4824F086FF0346002B0AD1FFF7D3
S3150802512015FC3B461A469749FFF70AFE944824F0AF
S31508025130D3FF02E0944816F0C1FC904BB3F86C32E8
S315080251403E3B9AB28D4BA3F86C228C4BB3F86A326B
S3150802515001339AB2894BA3F86A22884B012283F853
S315080251606822864BFF2283F86E22844B4FF4FA623A
S31508025170C3F87022FCE0814B93F86E32002B05D0FF
S315080251807E4B93F86E32012B40F0F2807B4BB3F8DC
S315080251906C323E2B02D940237B6404E0774BB3F88A
S315080251A06C3201337B6420233B703B785AB2734BD3
S315080251B0B3F86A325BB203F00F035BB213435BB216
S315080251C0DBB23B707B6C5A1E3B46013319466A4872
S315080251D026F099FB0346002B00F0CA804FF47A7139
S315080251E0674824F01FFF0346002B13D17B6C9BB242
S315080251F01846FFF743FC0346604AC2F85032FFF7E7
S31508025200A5FB3B461A465F49FFF79AFD5C4824F020
S3150802521063FF02E05C4816F051FC584BB3F86C2267
S315080252207B6C9BB2D31A9BB201339AB2534BA3F847
S315080252306C22524BB3F86A3201339AB24F4BA3F837
S315080252406A224E4BB3F86C32002B40F0918024222E
S3150802525000214C4830F082FF484B002283F868222E
S31508025260464B0022A3F86A22444BFF2283F86E2299
S315080252707EE0464826F0F0FA034683F00103DBB2E5
S31508025280002B75D03B4601221946404826F03BFBC7
S315080252900346002B69D03B781B09DBB2032B1FD1CF
S315080252A03B46013302221946384826F02CFB0346B0
S315080252B0002B5DD0314B0322DA604FF47A71304805
S315080252C024F0B0FE0346002B52D1FFF73FFB3B46C4
S315080252D01A462A49FFF734FD294824F0FDFE47E01D
S315080252E03B781B09DBB2002B42D13B460133012234
S315080252F01946264826F007FB0346002B37D03B788B
S315080253001B029BB203F47063A7F842307B781A46F5
S31508025310B7F842301343A7F84230B7F842203B4663
S3150802532002331946194826F0EEFA0346002B1FD017
S31508025330B7F8423002339BB21846FFF79FFB034683
S315080253400E4AD3604FF47A710D4824F06BFE034679
S31508025350002B0DD1FFF7FAFA3B461A460749FFF723
S31508025360EFFC074824F0B8FE02E000BF00E000BFE9
S315080253704837BD4680BD00BF60A500202CA300208B
S315080253809891002070A500209CA8050850A300202B
S3150802539080B59AB000AF3B4668220021184630F025
S315080253A0DDFE0E4826F058FA034683F00103DBB207
S315080253B0002B0ED004E03B466821184600F010F890
S315080253C03B4668221946054826F09DFA0346002BF5
S315080253D0F1D100BF6837BD4680BD00BF1C9B0020C7
S315080253E080B582B000AF78600B467B80786800F0A3
S315080253F0E3FB00BF0837BD4680BD000080B500AF9D
S31508025400174B93F86832002B28D0154B93F86E3257
S31508025410FF2B23D1124BD3F87032002B07D0104B37
S31508025420D3F87032013B0E4AC2F8703216E02422D3
S3150802543000210C4830F092FE4FF400620A490B48EC
S3150802544026F080F9064B002283F86822044B0022D4
S31508025450A3F86A22024BFF2283F86E2200BF80BDA0
S315080254602CA3002070A50020A0A5002060A500207E
S3150802547080B582B000AF78600B467B80786800F012
S31508025480C3FA00BF0837BD4680BD000080B582B0AA
S3150802549000AF78600B467B807B881A46796803489A
S315080254A026F0F6F900BF0837BD4680BD0C930020EA
S315080254B080B59AB000AF3B4668220021184630F004
S315080254C04DFE0E4826F0C8F9034683F00103DBB207
S315080254D0002B0ED004E03B4668211846FFF7C8FFAA
S315080254E03B4668221946054826F00DFA0346002B64
S315080254F0F1D100BF6837BD4680BD00BF0C930020BE
S3150802550080B582B000AF78600B4A7B681360FFF7FC
S3150802551029FA24220021094830F020FE24220021FB
S31508025520074830F01BFE24220021064830F016FEFA
S3150802553000BF0837BD4680BD089300202CA3002073
S3150802554070A50020B0AD002080B485B000AF7860A9
S315080255507B681B681B6CBB600023FB60BB68DBB205
S31508025560002B02D0BB68DBB2FB60FB681846143717
S31508025570BD465DF8047B704780B485B000AF78609D
S315080255807B681B681B6CBB600023FB60BB6803F46B
S31508025590FE43002B06D0BB6803F4FE43FB60FB68A0
S315080255A01B0AFB60FB6818461437BD465DF8047B88
S315080255B07047000080B485B000AF78607B681B68CE
S315080255C05B6CBB600023FB60BB6803F00703002B20
S315080255D02FD0BB6803F00703013B052B20D801A295
S315080255E052F823F0FD550208035602080956020826
S315080255F00F560208155602081B5602080123FB60BD
S315080256000FE00223FB600CE00323FB6009E004239E
S31508025610FB6006E00523FB6003E00623FB6000E06F
S3150802562000BF7B681B685A6C7B681B6822F00702FE
S315080256305A64FB68DBB218461437BD465DF8047B2C
S31508025640704700BF80B582B000AF786010F0BCFB2F
S3150802565003460121184610F079FF034683F0010339
S31508025660DBB2002B2AD17B68013B052B27D801A286
S3150802567052F823F08D560208955602089D560208DE
S31508025680A5560208AD560208B55602080D4816F088
S3150802569015FA14E00C4816F011FA10E00B4816F049
S315080256A00DFA0CE00A4816F009FA08E0094816F05D
S315080256B005FA04E0084816F001FA00E000BF0837C8
S315080256C0BD4680BDBCA80508CCA80508DCA8050807
S315080256D0F4A805080CA9050824A9050880B483B00E
S315080256E000AF0346FB71054AFB791370012318467E
S315080256F00C37BD465DF8047B704700BFF8B500203D
S3150802570080B400AF034B1B781846BD465DF8047B90
S31508025710704700BFF8B5002080B500AFFFF7F0FF6D
S315080257200346002B02D04FF4807301E04FF48073D6
S31508025730184680BD80B500AFFFF7E2FF0346002B8F
S3150802574002D04FF4003300E00023184680BD80B52E
S3150802575000AFFFF7D5FF0346002B02D040F209132C
S3150802576000E00023184680BDB0B5A4B006AFF860C5
S31508025770B9601346FB800023A7F87630FB683B65C1
S31508025780FFF7BEFF0346002B03D04FF080437B652D
S3150802579001E000237B650023BB65FB8802339BB2CD
S315080257A01846FFF76BF90346FB6500233B664FF481
S315080257B080137B664FF40013BB660023FB66002347
S315080257C03B6700233B743B7C5AB2FB881B0A9BB29D
S315080257D05BB203F00F035BB213435BB2DBB23B74FB
S315080257E0FB88DBB27B740223A7F8763010E0B7F8A1
S315080257F07630023BBA681A44B7F8763012787833AC
S315080258003B4403F8682CB7F876300133A7F87630AC
S31508025810B7F87620FB8801339A42E8DD0023A7F819
S3150802582076300DE0B7F8763078333B4413F8683CA7
S315080258301846FFF773FAB7F876300133A7F87630C9
S31508025840B7F87620FB8801339A42EBDD6D4607F1FD
S3150802585060040FCC0FC523682B6007F150030FCBEA
S31508025860FFF764F900BF7837BD46B0BD80B58EB084
S3150802587000AFF860B9601346FB80002387F837301B
S31508025880FB683B61FFF73CFF0346002B03D04FF052
S3150802589080437B6101E000237B610023BB61FB88B7
S315080258A0FB6100233B624FF480137B624FF40013C3
S315080258B0BB620023FB6200233B63FA8807F11003ED
S315080258C011461846FFF74AF9034687F8373097F81C
S315080258D03730002B06D0FA8897F83730B968184659
S315080258E0FFF7DEF900BF3837BD4680BDB0B5A2B0B6
S315080258F006AF7860084611461A460346FB700B4601
S31508025900BB7013467B70002387F86F307B68BB64D5
S31508025910FFF7F6FE0346002B03D04FF08043FB64E5
S3150802592001E00023FB6400233B6503237B65002318
S31508025930BB654FF48013FB654FF400133B660023E7
S315080259407B660023BB6630233B723B7A5AB297F9D1
S31508025950033003F00F035BB213435BB2DBB23B7255
S31508025960BB787B727B78BB72002387F86F300DE0B9
S3150802597097F86F3070333B4413F8683C1846FFF7C4
S31508025980CDF997F86F30013387F86F3097F86F3093
S31508025990022BEDD96D4607F158040FCC0FC52368C3
S315080259A02B6007F148030FCBFFF7C0F800BF70372B
S315080259B0BD46B0BD80B582B000AF78600023002234
S315080259C000217868FFF792FF00BF0837BD4680BD01
S315080259D080B584B000AFF860B9601346FB80FB88D7
S315080259E03E2B06D8FB881A46B968F868FFF7BCFE4C
S315080259F005E0FB881A46B968F868FFF737FF00BF63
S31508025A001037BD4680BD000080B588B000AF78600B
S31508025A10FF23FB7600237B610023FB6100237B8245
S31508025A207B68FB60FB6893F828301B09FB76FB68EA
S31508025A301B687B617B69B3F5003F02D140F209130B
S31508025A40FB61FB7E032B00F2A78001A252F823F02A
S31508025A50615A0208A35A0208ED5A02083B5B020879
S31508025A60FB6893F8283003F00F039AB24C4B1A805E
S31508025A704B4B1B881B029AB2494B1A80FB6893F858
S31508025A8029301A46464B1B8813439AB2444B1A804E
S31508025A90FB682A33424A12881146184603F0D6FE94
S31508025AA07AE0FB6893F8283003F00F039AB23C4B6E
S31508025AB01A803B4B1B881B029AB2394B1A80FB6829
S31508025AC093F829301A46364B1B8813439AB2344B3D
S31508025AD01A80344B01221A70FB682A333E21184673
S31508025AE003F0B4FEF869FFF765FF55E02D4B1B7806
S31508025AF01A46FB6893F8283003F00F039A4248D1F6
S31508025B00FB68DB681846FEF763FF0346013B7B82A8
S31508025B10FB6829337A8A1146184603F097FE214B09
S31508025B201B780133DAB21F4B1A701E4B1B780F2BE8
S31508025B302FD91C4B00221A702BE01B4BD3F8443288
S31508025B40FA699A420FD1FB6893F8283003F00F03DB
S31508025B50DAB2154B83F86E22FB6893F82920124BAA
S31508025B6083F86F2217E0104BD3F8843AFA699A42FF
S31508025B7011D1FB6893F8283003F00F03DAB20A4B07
S31508025B8083F8AE2AFB6893F82920074B83F8AF2AD5
S31508025B9001E000BF00E000BF00BF2037BD4680BD60
S31508025BA002B6002004B600202CA3002080B500AF60
S31508025BB02EF04EFD00BF80BD80B584B000AF786080
S31508025BC07B68FB60FFF79CFD0346002B0AD0FB6847
S31508025BD01B68B3F5806F10D1FB6893F82830002B49
S31508025BE00BD10AE0FB681B68B3F5806F05D1FB6829
S31508025BF093F82830002B00D100BF00BF1037BD46EE
S31508025C0080BD000080B500AF40220349034825F055
S31508025C1099FD0123184680BD18B6002008B6002053
S31508025C2080B500AF054825F017FE0346002B01D0C4
S31508025C30012300E00023184680BD00BF08B60020F5
S31508025C4080B582B000AF78600B46FB704FF47A716C
S31508025C50094824F0E7F90346002B08D1FB781A46CF
S31508025C607968064825F083FF034824F035FA0123AC
S31508025C7018460837BD4680BDCC91002008B60020DC
S31508025C8080B584B000AF78600023FB734FF47A7155
S31508025C90094824F0C7F90346002B08D17968074852
S31508025CA025F076FF0346FB73034824F015FAFB7BBF
S31508025CB018461037BD4680BDCC91002008B6002094
S31508025CC080B400AF034B1B781846BD465DF8047BCB
S31508025CD0704700BFB9B6002080B400AF034B1B78EB
S31508025CE01846BD465DF8047B704700BFC0B6002063
S31508025CF080B400AF034B1B781846BD465DF8047B9B
S31508025D00704700BFC2B6002090B583B000AF034605
S31508025D10FB717D4B1B78012B1AD108F0CFFA04468A
S31508025D20FB79184608F05EFE03461946204608F037
S31508025D305CFBFB79184608F055FE03461A46734B78
S31508025D401A70724B1B781946714815F0B7FED7E0E0
S31508025D506D4B1B78022B1AD108F0B0FA0446FB7970
S31508025D60184608F0C9FE03461946204608F03DFBC8
S31508025D70FB79184608F0C0FE03461A46634B1A70AA
S31508025D80624B1B781946634815F098FEB8E05E4BDD
S31508025D901B78032B1AD108F091FA0446FB791846A8
S31508025DA008F008FF03461946204608F01EFBFB7951
S31508025DB0184608F0FFFE03461A46544B1A70534B10
S31508025DC01B781946544815F079FE99E04E4B1B7814
S31508025DD0042B1AD108F072FA0446FB79184608F021
S31508025DE047FF03461946204608F0FFFAFB7918468C
S31508025DF008F03EFF03461A46444B1A70434B1B787B
S31508025E001946464815F05AFE7AE03F4B1B78052B91
S31508025E101AD108F053FA0446FB79184608F086FFA9
S31508025E2003461946204608F0E0FAFB79184608F0B8
S31508025E307DFF03461A46354B1A70344B1B781946B2
S31508025E40374815F03BFE5BE02F4B1B78062B1AD121
S31508025E5008F034FA0446FB79184608F0C5FF0346EB
S31508025E601946204608F0C1FAFB79184608F0BCFF25
S31508025E7003461A46254B1A70244B1B78194629489D
S31508025E8015F01CFE3CE0204B1B78072B1AD108F0B4
S31508025E9015FA0446FB79184609F004F8034619462A
S31508025EA0204608F0A2FAFB79184608F0FBFF0346DB
S31508025EB01A46164B1A70154B1B7819461A4815F0CE
S31508025EC0FDFD1DE0104B1B78082B19D108F0F6F9D9
S31508025ED00446FB79184609F043F803461946204654
S31508025EE008F083FAFB79184609F03AF803461A4687
S31508025EF0064B1A70054B1B7819460C4815F0DEFD41
S31508025F0000BF0C37BD4690BDC0B60020C1B6002002
S31508025F1030A9050850A9050870A9050890A9050819
S31508025F20B0A90508D0A90508F0A9050810AA050808
S31508025F3080B582B000AF0346FB71374B1B78012B45
S31508025F4008D1FB79184608F04DFD03461A46334B2D
S31508025F501A705DE0304B1B78022B08D1FB79184684
S31508025F6008F0CAFD03461A462C4B1A7050E02A4B13
S31508025F701B78032B08D1FB79184608F01BFE03464B
S31508025F801A46264B1A7043E0234B1B78042B08D17A
S31508025F90FB79184608F06CFE03461A461F4B1A7020
S31508025FA036E01D4B1B78052B08D1FB79184608F0FD
S31508025FB0BDFE03461A46194B1A7029E0164B1B7882
S31508025FC0062B08D1FB79184608F00EFF03461A4637
S31508025FD0124B1A701CE0104B1B78072B08D1FB7961
S31508025FE0184608F05FFF03461A460C4B1A700FE074
S31508025FF0094B1B78082B08D1FB79184608F0B0FF25
S3150802600003461A46054B1A7002E0044BFF221A7021
S3150802601000BF0837BD4680BDC0B60020C3B6002003
S3150802602080B584B000AF03460A46FB711346BB71BE
S315080260300023FB60FB795A1E13469B0013449B0000
S3150802604003F10A02BB791344FB602CF095FB024666
S31508026050FB68DBB2194610462CF0CFFBFB79BA79FE
S315080260601946034815F02AFD00BF1037BD4680BD04
S3150802607030AA0508B0B598B002AF002387F85230A7
S31508026080002387F857300023A7F85430002387F8EF
S3150802609053300FF099FE034618460FF025FF0346C4
S315080260A0002B02D0B74B00221A70FFF7B9FD034640
S315080260B0002B40F00485B44815F000FD07F11003E3
S315080260C040220021184630F049F807F11003184615
S315080260D0FFF7D6FD034687F852303B7C012B40F08A
S315080260E0E98497F85230002B00F0E4847B7CFF2B7E
S315080260F000F0F682FF2B00F3AA84302B00F0B0845E
S31508026100302B00F3A484222B00F0D783222B00F332
S315080261109E84202B00F00E83202B00F39884012BFB
S3150802612004D0062B00F0468200F091BC0FF04CFE1C
S315080261300346184610F0A5FA924B1B78002B40F03E
S31508026140918497F85230023BD9B207F11003023311
S315080261508E4A184626F041FF8C4826F09DFB0346D8
S31508026160002B00F04E81894826F096FB0346102B39
S3150802617000F24781854826F074FB0346002B00F09F
S315080261804081824826F06DFB0346082B00F23981CE
S315080261907E4826F066FB03461A467D4B1A707B48F4
S315080261A026F07AFB03461A467A4B1A70784B1B7806
S315080261B01946784B1B781A46774815F07FFC754BBB
S315080261C01B78012B03D10720FFF79EFD76E0714B62
S315080261D01B78022B03D10220FFF796FD6EE06D4B6A
S315080261E01B78032B03D10320FFF78EFD66E0694B6C
S315080261F01B78042B03D10920FFF786FD5EE0654B69
S315080262001B78052B03D10820FFF77EFD56E0614B6C
S315080262101B78062B03D10420FFF776FD4EE05D4B73
S315080262201B78072B03D10520FFF76EFD46E0594B75
S315080262301B78082B03D10620FFF766FD3EE0554B77
S315080262401B78092B03D10A20FFF75EFD36E0514B76
S315080262501B780A2B03D10B20FFF756FD2EE04D4B78
S315080262601B780B2B03D10C20FFF74EFD26E0494B7A
S315080262701B780C2B03D10D20FFF746FD1EE0454B7C
S315080262801B780D2B03D10E20FFF73EFD16E0414B7E
S315080262901B780E2B03D10F20FFF736FD0EE03D4B80
S315080262A01B780F2B03D11020FFF72EFD06E0394B82
S315080262B01B78102B02D11120FFF726FD334826F052
S315080262C006FB0346002B00F08B80304826F0FFFAC7
S315080262D00346102B00F284802C4826F0F8FA03466F
S315080262E0013B0F2B6ED801A252F823F02D63020848
S315080262F0356302083D630208456302084D630208D6
S31508026300556302085D630208656302086D63020845
S31508026310756302087D6302089D630208A563020885
S31508026320AD630208B5630208BD6302080720FFF7DA
S31508026330FFFD4BE00220FFF7FBFD47E00320FFF7D6
S31508026340F7FD43E00920FFF7F3FD3FE00820FFF7DA
S31508026350EFFD3BE00420FFF7EBFD37E00520FFF7F2
S31508026360E7FD33E00620FFF7E3FD2FE00A20FFF7FB
S31508026370DFFD2BE00B20FFF7DBFD27E00C20FFF704
S31508026380D7FD23E0B9B600206CAA0508B4B60020EA
S31508026390C0B60020C2B6002098AA05080D20FFF74D
S315080263A0C7FD13E00E20FFF7C3FD0FE00F20FFF72E
S315080263B0BFFD0BE01020FFF7BBFD07E01120FFF73A
S315080263C0B7FD03E0CB4BFF221A7000BF07F076FF3A
S315080263D00246C84B1B781946104608F023F806E011
S315080263E007F06CFF0346FF21184608F01BF8C2485F
S315080263F015F064FBC14B00221A60C14B01221A70C8
S3150802640030E3C04826F048FA0346FE2B40F0C38024
S31508026410BC4826F026FA03461A46BB4B1A70B948F8
S3150802642026F03AFA03461A46B84B1A70B64B1B7848
S315080264301946B64B1B781A46B54815F03FFB07F0C6
S315080264403DFF0346FE21184607F0CFFF07F036FF49
S315080264500346FF21184607F0E5FFAB4B1B78012BD5
S315080264600ED107F02BFF0346184607F097FF03469F
S31508026470184608F063FA03461A46A64B1A7083E0D2
S31508026480A14B1B78022B0ED107F018FF03461846BC
S3150802649007F084FF0346184608F0F8FA03461A4638
S315080264A09C4B1A7070E0984B1B78032B0ED107F0A1
S315080264B005FF0346184607F071FF0346184608F01B
S315080264C043FB03461A46934B1A705DE08E4B1B78C4
S315080264D0042B0ED107F0F2FE0346184607F05EFFBC
S315080264E00346184608F08EFB03461A46894B1A706D
S315080264F04AE0854B1B78052B0ED107F0DFFE0346D3
S31508026500184607F04BFF0346184608F0D9FB034620
S315080265101A46804B1A7037E07B4B1B78062B0ED136
S3150802652007F0CCFE0346184607F038FF034618461E
S3150802653008F024FC03461A46764B1A7024E0724B7E
S315080265401B78072B0ED107F0B9FE0346184607F04B
S3150802655025FF0346184608F06FFC03461A466D4B9C
S315080265601A7011E0684B1B78082B0DD107F0A6FEAE
S315080265700346184607F012FF0346184608F0BAFC07
S3150802658003461A46634B1A705C4B00221A605C4B30
S3150802659001221A7066E25B4826F07EF903461C461B
S315080265A0584826F05EF903461A4621465A4815F017
S315080265B085FA57E20FF008FC0346184610F061F810
S315080265C007F1100302335549184626F0ADFD534824
S315080265D026F0EAFB0346002B0AD15149022010F0A5
S315080265E09BF90FF0F1FB034618460FF039FC3AE225
S315080265F04A4826F0D9FB0346022B68D149490220AC
S3150802660010F08AF92CF0B8F8034618462CF0DAF896
S3150802661003460021184626F09DF82CF0ADF80346ED
S3150802662018462CF0CFF803460021184626F0ADF896
S315080266302CF0A2F803460A2118462CF064F92CF02D
S315080266409BF803460B2118462CF05DF92CF094F8BA
S3150802665003460C2118462CF056F92CF08DF8034601
S315080266600D2118462CF04FF92CF086F803460E2118
S3150802667018462CF048F92CF07FF803460F211846E5
S315080266802CF041F92CF078F80346102118462CF024
S315080266903AF92CF071F80346112118462CF033F911
S315080266A029F034FE0346184629F00DFF0FF08CFB3D
S315080266B0034618460FF03AFC0FF086FB0346012103
S315080266C018460FF002FC184B00221A70CBE1134849
S315080266D026F06AFB03461946144815F0EFF9C2E19B
S315080266E0134815F0EBF90FF06FFB034618460FF047
S315080266F0B7FBB8E1C3B60020F0AA0508BCB600206D
S31508026700B9B60020B4B60020C0B60020C2B6002032
S3150802671098AA0508C1B600202CAB0508B8B6002011
S3150802672094AB0508C4AB050809050220E4AB0508C5
S315080267300CAC050807F10C0207F1100302331146E7
S31508026740184628F087FEBB891A46BB7BC649022033
S3150802675010F0E2F8BA7BC54B1B789A4209D1BB897D
S31508026760C34A1278934204D1C249022010F0D4F8DF
S3150802677079E1BA89C04B1A80BA7BBF4B9A70BA7B49
S31508026780BA4B1A70BB89DAB2B94B1A70002387F86A
S31508026790573028E02BF0F0FF034618462CF012F883
S315080267A0024697F857301946104626F033F803463C
S315080267B0A7F85430B04826F0A5F803461A46B7F8A3
S315080267C0543093420AD1B7F854301A46AB490220DC
S315080267D010F0A2F8012387F8533008E097F85730EB
S315080267E0013387F8573097F85730072BD2D997F8DD
S315080267F05330002B04D004219F4806F0D5FE32E11F
S31508026800B7F854301A469E49022010F085F829F046
S315080268107DFD01230622382129F0F4FD0FF0D4FA72
S315080268200346382118460FF051FF0FF0CDFA0346FA
S31508026830062118460FF068FF8F4B1B881A468E4BA7
S315080268409B781946002300930B468E49022010F0C6
S3150802685063F88D4B0022DA70874B1A888A4B1A80A6
S31508026860854B9A78884B9A700FF0AEFA034618460B
S315080268700FF01FFF03461A46834B1A710FF0A4FA4C
S31508026880034618460FF033FF03461A467E4B5A71E3
S315080268907E497D4828F027FE26F0DAFE04467B4824
S315080268A028F01AFB0546794828F022FB03461A46C1
S315080268B0294620462DF0B8FFD5E03A1D07F1100308
S315080268C002331146184628F04DFE3B791A46FB88D4
S315080268D019463B7A00930B466D49022010F01CF8C4
S315080268E03A796C4B1B789A4204D16B49022010F014
S315080268F013F8B8E03A79674B1A703B1D184628F028
S3150802690085FA0346002B32D0002387F8573029E050
S315080269102BF032FF034618462BF054FF024697F82F
S3150802692057301946104625F075FF0346A7F8543026
S315080269303B1D184628F06AFA03461A46B7F8543039
S3150802694093420AD1B7F854301A46544902200FF036
S31508026950E3FF012387F853301DE097F857300133D8
S3150802696087F8573097F85730072BD1D913E03B1DD4
S31508026970184628F066FA0346002B0CD03B1D18462B
S3150802698028F05FFA03461A46454902200FF0C4FF6B
S31508026990012387F8533097F85330002B05D03B1D57
S315080269A00621184606F020FE5DE0B7F854301A466E
S315080269B03C4902200FF0B0FF3B1D184628F00BFA9F
S315080269C003461C463B1D184628F020FA03461D4678
S315080269D03B1D184628F035FA03461A460223019348
S315080269E000922B462246304902200FF095FF2F4B84
S315080269F002225A713B1D184628F008FA03461A461F
S31508026A002A4B5A803B1D184628F0E5F903461A46D2
S31508026A10264B1A703B1D184628F013FA03461A46E7
S31508026A20224B1A711949214828F0F0FD26F010FE6A
S31508026A300446164828F050FA0546144828F058FA2B
S31508026A4003461A46294620462DF0EEFE0BE07B7CCD
S31508026A50194697F852301A46154815F02FF802E0EB
S31508026A6000BF2CE000BF2AE028AC0508DC12002093
S31508026A7058B6002040AC05085CB600205CAC050898
S31508026A8080AC0508A8AC050860B6002068B60020E8
S31508026A90CCAC0508DD120020E0AC0508F8AC050808
S31508026AA014AD05082CAD05084CAD0508ACB600209A
S31508026AB070AD05083B7C1946B74814F0FFFFB74B83
S31508026AC01B78002B02D0012B04D0AEE3B44B002274
S31508026AD01A60AAE307F0F2FB0346184607F0B5FE6A
S31508026AE00346012B0BD107F0E9FB0346184607F0CC
S31508026AF055FC03461A46AB4B1B789A420ED007F052
S31508026B00DDFB0346184607F0A0FE0346012B40F0BC
S31508026B100983A54B1B78FE2B40F00483A24B1B78F6
S31508026B20002B16D0A04B1B78102B12D89F4B1B7824
S31508026B30002B00F0C2829D4B1B78082B00F2BD8207
S31508026B409A4B1B78984A127811461846FFF768FA44
S31508026B50B3E2954B1B78FE2B40F0B082914B1B7823
S31508026B60072B4CD1914B1B78012B0ED12BF004FE2F
S31508026B70034618462BF026FE03460B21184625F037
S31508026B80E9FD8B4814F09AFF98E2884B1B78022B92
S31508026B900ED12BF0F1FD034618462BF013FE0346E1
S31508026BA01F21184625F0D6FD824814F087FF85E294
S31508026BB07E4B1B78032B0ED12BF0DEFD03461846BF
S31508026BC02BF000FE03463321184625F0C3FD7A480A
S31508026BD014F074FF72E2754B1B78042B40F06E8238
S31508026BE02BF0CAFD034618462BF0ECFD0346472157
S31508026BF0184625F0AFFD714814F060FF5EE2694B56
S31508026C001B78022B4CD1694B1B78012B0ED12BF02A
S31508026C10B3FD034618462BF0D5FD03460C2118464C
S31508026C2025F098FD664814F049FF47E25F4B1B784A
S31508026C30022B0ED12BF0A0FD034618462BF0C2FDFF
S31508026C4003462021184625F085FD5E4814F036FFD6
S31508026C5034E2564B1B78032B0ED12BF08DFD0346DF
S31508026C6018462BF0AFFD03463421184625F072FD6F
S31508026C70554814F023FF21E24C4B1B78042B40F0B5
S31508026C801D822BF079FD034618462BF09BFD034621
S31508026C904821184625F05EFD4C4814F00FFF0DE218
S31508026CA0404B1B78032B4CD1404B1B78012B0ED142
S31508026CB02BF062FD034618462BF084FD03460D2190
S31508026CC0184625F047FD424814F0F8FEF6E1374B20
S31508026CD01B78022B0ED12BF04FFD034618462BF0DC
S31508026CE071FD03462121184625F034FD394814F072
S31508026CF0E5FEE3E12D4B1B78032B0ED12BF03CFD71
S31508026D00034618462BF05EFD03463521184625F044
S31508026D1021FD314814F0D2FED0E1244B1B78042B16
S31508026D2040F0CC812BF028FD034618462BF04AFD8D
S31508026D3003464921184625F00DFD284814F0BEFEE3
S31508026D40BCE1184B1B78092B75D1184B1B78012B04
S31508026D500ED12BF011FD034618462BF033FD0346E0
S31508026D600E21184625F0F6FC1D4814F0A7FEA5E1EB
S31508026D700E4B1B78022B37D12BF0FEFC0346184626
S31508026D802BF020FD03462221184625F0E3FC154880
S31508026D9014F094FE92E100BFA0AD0508B9B6002032
S31508026DA0BCB60020C1B60020C2B60020C0B600207C
S31508026DB0D4AD050810AE05084CAE050888AE050820
S31508026DC0C4AE050800AF05083CAF050878AF05084C
S31508026DD0B4AF0508F0AF05082CB0050868B0050879
S31508026DE0A4B00508E0B00508B94B1B78032B0ED1F1
S31508026DF02BF0C2FC034618462BF0E4FC0346362168
S31508026E00184625F0A7FCB34814F058FE56E1B04BD5
S31508026E101B78042B40F052812BF0AEFC0346184631
S31508026E202BF0D0FC03464A21184625F093FCAA48C3
S31508026E3014F044FE42E1A94B1B78082B4CD1A44B13
S31508026E401B78012B0ED12BF097FC034618462BF024
S31508026E50B9FC03460F21184625F07CFCA04814F01D
S31508026E602DFE2BE19A4B1B78022B0ED12BF084FCBC
S31508026E70034618462BF0A6FC03462321184625F09E
S31508026E8069FC984814F01AFE18E1914B1B78032BFB
S31508026E900ED12BF071FC034618462BF093FC0346E1
S31508026EA03721184625F056FC8F4814F007FE05E1EF
S31508026EB0874B1B78042B40F001812BF05DFC0346BF
S31508026EC018462BF07FFC03464B21184625F042FC58
S31508026ED0864814F0F3FDF1E0804B1B78042B4CD165
S31508026EE07B4B1B78012B0ED12BF046FC034618462A
S31508026EF02BF068FC03461021184625F02BFC7C482B
S31508026F0014F0DCFDDAE0724B1B78022B0ED12BF063
S31508026F1033FC034618462BF055FC03462421184633
S31508026F2025F018FC734814F0C9FDC7E0684B1B78B6
S31508026F30032B0ED12BF020FC034618462BF042FCFD
S31508026F4003463821184625F005FC6B4814F0B6FDB1
S31508026F50B4E05F4B1B78042B40F0B0802BF00CFC9E
S31508026F60034618462BF02EFC03464C21184625F0FC
S31508026F70F1FB624814F0A2FDA0E0584B1B78052BE2
S31508026F804BD1534B1B78012B0ED12BF0F5FB034645
S31508026F9018462BF017FC03461121184625F0DAFB92
S31508026FA0574814F08BFD89E0494B1B78022B0ED10A
S31508026FB02BF0E2FB034618462BF004FC0346252178
S31508026FC0184625F0C7FB4F4814F078FD76E0404B8B
S31508026FD01B78032B0ED12BF0CFFB034618462BF05A
S31508026FE0F1FB03463921184625F0B4FB464814F04E
S31508026FF065FD63E0364B1B78042B5FD12BF0BCFB97
S31508027000034618462BF0DEFB03464D21184625F0AB
S31508027010A1FB3E4814F052FD50E0304B1B78062B7C
S315080270204CD12B4B1B78012B0ED12BF0A5FB03461B
S3150802703018462BF0C7FB03461221184625F08AFB91
S31508027040334814F03BFD39E0214B1B78022B0ED155
S315080270502BF092FB034618462BF0B4FB0346262177
S31508027060184625F077FB2B4814F028FD26E0184B26
S315080270701B78032B0ED12BF07FFB034618462BF009
S31508027080A1FB03463A21184625F064FB224814F070
S3150802709015FD13E00E4B1B78042B0FD12BF06CFB5E
S315080270A0034618462BF08EFB03464E21184625F05A
S315080270B051FB1A4814F002FD00E000BF0EF084FEF0
S315080270C0034618460FF034FA154B00221A7069E087
S315080270D0C0B6002068B005081CB10508C1B6002074
S315080270E058B1050894B10508D0B105080CB20508CF
S315080270F048B2050884B20508C0B20508FCB20508FC
S3150802710038B3050874B30508B0B30508ECB3050827
S3150802711028B4050864B40508A0B40508DCB4050853
S31508027120B9B6002007F0CAF80346184607F08DFBE1
S315080271300346012B0CD107F0C1F80346184607F09F
S3150802714048F90346FF2B03D1002008F0BFFE29E0C9
S3150802715007F0B4F80346184607F077FB0346012BF7
S3150802716020D107F0ABF80346184607F017F903468D
S315080271701C4607F0A3F80346184607F02AF9034601
S315080271809C420FD107F09AF80346FF21184607F0EA
S3150802719049F907F093F80246264B1B78194610461A
S315080271A007F023F9244B1B680133234A1360224B49
S315080271B01B684AF6C772934208D807F07FF8034657
S315080271C0184607F042FB0346032B2DD11B4814F041
S315080271D075FC29F09BF81A4B1B781A469200134441
S315080271E09B00DAB2174B1B781344DBB2143BDAB2B4
S315080271F00123372129F006F907F060F803461846F5
S3150802720007F023FB0346032B0BD008F031FC034699
S31508027210002B06D12BF0B0FA03460A2118462BF0AA
S3150802722050FB094B00221A7000BF00BF5837BD46F3
S31508027230B0BD00BFC1B60020BCB6002018B505080F
S31508027240C0B60020C2B60020B9B6002080B500AF8D
S315080272504FF400720349044824F074FA01231846CD
S3150802726080BD00BFC4B60020C4B8002080B582B075
S3150802727000AF0023FB71074824F0EEFA0346FB71C0
S31508027280FB79002B01D0012300E0002318460837BA
S31508027290BD4680BDC4B8002080B584B000AF786012
S315080272A00B46FB700023FB604FF47A710F4822F0FD
S315080272B0B9FE0346002B0AD1FB781A4679680C48B0
S315080272C024F055FCF860094822F006FF02E0094856
S315080272D014F0F4FBFB68002B02D1074814F0EEFB0E
S315080272E0012318461037BD4680BD00BFD092002044
S315080272F0C4B8002038B5050874B5050880B584B049
S3150802730000AF78600023FB734FF47A710B4822F0C2
S3150802731089FE0346002B09D17968094824F038FC0E
S315080273200346FB73054822F0D7FE02E0054814F02F
S31508027330C5FBFB7B18461037BD4680BDD0920020A0
S31508027340C4B80020A0B5050880B584B000AF78603F
S315080273500B46FB700023FB600023FB6009E0FB7809
S31508027360184614F0C5FC012021F014FFFB6801330E
S31508027370FB60FA687B689A42F1D300BF00BF1037F8
S31508027380BD4680BD80B485B000AF87ED010A0023F3
S31508027390FB81D7ED017AF5EEC07AF1EE10FA0BDB36
S315080273A0D7ED017AB2EE047A67EE877AFCEEE77ACF
S315080273B017EE903A9BB216E0D7ED017AF5EEC07A4F
S315080273C0F1EE10FA0ED5D7ED017ABAEE047A67EE27
S315080273D0877AFCEEE77A17EE903AFB81FB895B42E5
S315080273E09BB200E0002318461437BD465DF8047BBD
S315080273F070470000B0B584B000AF0346FB710023A6
S31508027400FB600023FB7200237B720023BB72FFF72B
S315080274102DFF0346002B40F01286E14B00221A701C
S3150802742080220021DF482EF099FEDE48FFF766FF2C
S3150802743003461A46DA4B1A70DA4B1B78213B512B54
S3150802744000F2F28501A252F823F000BF95750208F0
S31508027450BD750208DF75020829800208298002081C
S31508027460298002082980020829800208EB75020889
S315080274702980020829800208298002082980020830
S315080274802980020829800208F77502086778020827
S315080274909F7A0208298002082980020829800208A0
S315080274A02980020829800208298002082980020800
S315080274B029800208298002082980020829800208F0
S315080274C029800208298002082980020829800208E0
S315080274D029800208298002082980020829800208D0
S315080274E029800208298002082980020829800208C0
S315080274F029800208298002082980020829800208B0
S31508027500298002082980020829800208298002089F
S31508027510298002082980020829800208298002088F
S31508027520298002082980020829800208298002087F
S31508027530298002082980020829800208298002086F
S315080275402980020829800208A97A020829800208E5
S31508027550298002082980020829800208298002084F
S31508027560298002082980020829800208298002083F
S31508027570298002082980020829800208298002082F
S315080275802980020829800208177D0208AB7D0208B5
S31508027590BD7F0208844902200FF0BEF98349844858
S315080275A023F064FB814822F0D0FF0346002B40F00B
S315080275B04385012008F08AFC00F03EBD7D49022081
S315080275C00FF0AAF97C497A4823F0ABFB0EF0FCFBD4
S315080275D00346012118460EF05DFC00F030BD7749DE
S315080275E002200FF099F900F02ABD754902200FF022
S315080275F093F900F024BD734902200FF08DF9724900
S315080276006B4823F004FC704823F00BF8034619462E
S315080276106E4824F0A1FD6E496C4825F003F825F062
S31508027620C1FF04466A4824F0C1FD0546684824F0AD
S31508027630C9FD03461A46294620462DF0F5F8FB7978
S3150802764019464FF47A70FFF77FFE22F0D3FE0346FF
S31508027650184622F008FF034619465E4823F059F8F1
S31508027660594822F0DEFF0346013B072B00F2E08071
S3150802767001A252F823F000BF99760208C5760208DD
S31508027680F17602081D77020849770208757702081B
S31508027690D97702080578020801214E4823F054F8E2
S315080276A00EF092FB034618460EF0FEFCF0EE407A08
S315080276B0B0EE670AFFF766FE03461946454823F009
S315080276C05EF8BFE00221434823F03EF80EF07CFB49
S315080276D0034618460EF006FDF0EE407AB0EE670A4B
S315080276E0FFF750FE034619463A4823F048F8A9E040
S315080276F00321384823F028F80EF066FB034618469D
S315080277000EF00EFDF0EE407AB0EE670AFFF73AFE8B
S31508027710034619462F4823F032F893E004212D48F0
S3150802772023F012F80EF050FB034618460EF016FD2B
S31508027730F0EE407AB0EE670AFFF724FE03461946D2
S31508027740244823F01CF87DE00521224822F0FCFF9C
S315080277500EF03AFB034618460EF01EFDF0EE407A8E
S31508027760B0EE670AFFF70EFE03461946194823F0DC
S3150802777006F867E00621174822F0E6FF0EF024FB1A
S31508027780034618460EF026FDF0EE407AB0EE670A7A
S31508027790FFF7F8FD034619460E4822F0F0FF51E0BE
S315080277A054B90020D4B800201CB605085CBA0020DB
S315080277B0D5B800203CB6050860BA002060B60508B0
S315080277C080B60508A4B6050864BA0020CCBA00201B
S315080277D088BA002068BA00200721DB4822F0B4FFE5
S315080277E00EF0F2FA034618460EF012FDF0EE407A53
S315080277F0B0EE670AFFF7C6FD03461946D24822F0DD
S31508027800BEFF1FE00821D04822F09EFF0EF0DCFAE8
S31508027810034618460EF01AFDF0EE407AB0EE670AF5
S31508027820FFF7B0FD03461946C74822F0A8FF09E04C
S31508027830C64822F0F6FE03461A46C54902200FF04C
S315080278406BF800BFC349C04823F036FBC14829F08C
S31508027850BDFF0446BF4829F0C5FF03461946204620
S3150802786001F0E0FFEBE3BC4902200FF055F8BB49F3
S31508027870BB4823F075FBB94822F0ABFF034619460D
S31508027880B84824F084FCB849B64824F0EAFE25F044
S3150802789089FE0446B44824F089FC0546B24824F019
S315080278A091FC03461A46294620462CF0BDFFFB7971
S315080278B019464FF47A70FFF747FD22F09BFD0346FF
S315080278C0184622F0D0FD03461946A84822F0F9FFC9
S315080278D0A24822F07EFF0346013B072B00F2C48032
S315080278E001A252F823F000BF097902083579020885
S315080278F0617902088D790208B9790208E5790208E0
S31508027900117A02083D7A02080121984822F0F4FF0A
S315080279100EF05AFA034618460EF0C6FBF0EE407A07
S31508027920B0EE670AFFF72EFD034619468F4822F086
S31508027930FEFFA3E002218D4822F0DEFF0EF044FA94
S31508027940034618460EF0CEFBF0EE407AB0EE670A12
S31508027950FFF718FD03461946844822F0E8FF8DE032
S315080279600321824822F0C8FF0EF02EFA0346184673
S315080279700EF0D6FBF0EE407AB0EE670AFFF702FD8C
S3150802798003461946794822F0D2FF77E00421774860
S3150802799022F0B2FF0EF018FA034618460EF0DEFB86
S315080279A0F0EE407AB0EE670AFFF7ECFC034619469A
S315080279B06E4822F0BCFF61E005216C4822F09CFF6C
S315080279C00EF002FA034618460EF0E6FBF0EE407A8F
S315080279D0B0EE670AFFF7D6FC03461946634822F05B
S315080279E0A6FF4BE00621614822F086FF0EF0ECF96D
S315080279F0034618460EF0EEFBF0EE407AB0EE670A42
S31508027A00FFF7C0FC03461946584822F090FF35E0B6
S31508027A100721564822F070FF0EF0D6F9034618469B
S31508027A200EF0F6FBF0EE407AB0EE670AFFF7AAFC14
S31508027A30034619464D4822F07AFF1FE008214B48B3
S31508027A4022F05AFF0EF0C0F9034618460EF0FEFB66
S31508027A50F0EE407AB0EE670AFFF794FC0346194641
S31508027A60424822F064FF09E0384822F0DAFD03466C
S31508027A701A463F4902200EF04FFF00BF35493B48E0
S31508027A8023F0C3FA334829F0A1FE0446314829F007
S31508027A90A9FE03461946204601F0C4FECFE235493F
S31508027AA002200EF039FFCAE2334902200EF034FFF3
S31508027AB032492B48FCF75DFD3048FCF7B1FB03461B
S31508027AC0013B182B00F28F8001A252F823F000BF67
S31508027AD0357B02083B7B0208417B0208817B020850
S31508027AE0877B02088D7B0208937B0208997B020832
S31508027AF09F7B0208A57B0208AB7B0208B17B0208C2
S31508027B00B77B0208BD7B0208C37B0208E77B020833
S31508027B10E77B0208E77B0208E77B0208E77B0208A5
S31508027B20C97B0208CF7B0208D57B0208DB7B0208E9
S31508027B30E17B02080723FB725FE01123FB725CE01C
S31508027B400623FB7259E000BF68BA002064BA002017
S31508027B50C0B6050858B90020ECB605086CBA00206C
S31508027B60D5B80020D0BA002088BA002070BA002002
S31508027B700CB705083CB705085CB7050874BA0020B7
S31508027B801023FB7239E00523FB7236E00F23FB72E2
S31508027B9033E00423FB7230E00E23FB722DE0082348
S31508027BA0FB722AE00D23FB7227E00923FB7224E00D
S31508027BB00C23FB7221E00323FB721EE00B23FB72EC
S31508027BC01BE00223FB7218E00723FB7215E005236C
S31508027BD0FB7212E00423FB720FE00823FB720CE02F
S31508027BE00323FB7209E0BA48FCF71AFB03461A4656
S31508027BF0B84902200EF090FE00BFB548FCF7F5FA28
S31508027C000346013B072B7BD801A252F823F000BF9B
S31508027C10317C02084B7C0208657C02087F7C0208DC
S31508027C20997C0208B37C0208CD7C0208E77C02082C
S31508027C3006F044FB0446FB7A184606F0D3FE0346D2
S31508027C401946204606F0D1FB64E006F037FB0446E7
S31508027C50FB7A184607F084F903461946204606F0C9
S31508027C60C4FB57E006F02AFB0446FB7A184607F0DF
S31508027C7019F903461946204606F0B7FB4AE006F00C
S31508027C801DFB0446FB7A184607F0AEF8034619466A
S31508027C90204606F0AAFB3DE006F010FB0446FB7AF6
S31508027CA0184607F043F803461946204606F09DFB98
S31508027CB030E006F003FB0446FB7A184606F0D8FFC6
S31508027CC003461946204606F090FB23E006F0F6FA2C
S31508027CD00446FB7A184606F06DFF03461946204607
S31508027CE006F083FB16E006F0E9FA0446FB7A184624
S31508027CF006F002FF03461946204606F076FB09E01F
S31508027D007348FCF772FA03461A46734902200EF0C4
S31508027D1003FE00BF93E1714902200EF0FDFD704992
S31508027D207048FCF79CFC6E48FCF7CBFA03467B725C
S31508027D307B7A642B03D9642000F056FD03E07B7A34
S31508027D40184600F051FD6648FCF7A0FA0346002BD8
S31508027D5002D07B7A002B07D100F010FE00F054FE09
S31508027D60614B00221A706AE15D48FCF78FFA0346F6
S31508027D70012B09D15C4B01221A7000F0CDFD7B7AEA
S31508027D80184600F031FD59E15548FCF77FFA0346DB
S31508027D90022B40F05381544B01221A7000F002FE66
S31508027DA07B7A184600F020FD48E1504902200EF081
S31508027DB0B3FD4F494B48FCF7D0FC22F01BFB0346A8
S31508027DC0184622F050FB034619464A48FCF70CFBB4
S31508027DD000214848FCF723FB4548FCF7DEFA034630
S31508027DE0BB72BB7A632B01D96323BB724048FCF78B
S31508027DF09EFA0346012B35D13D48FCF7B3FA0346F2
S31508027E00002B02D0BB7A002B04D100F079FE00F0D9
S31508027E108DFEC2E03648FCF7A5FA0346012B06D1C9
S31508027E20354B1B68BA7ADA6300F04EFEB5E0304885
S31508027E30FCF798FA0346022B06D12F4B1B68BA7A2F
S31508027E401A6400F04FFEA8E02948FCF78BFA0346AD
S31508027E501A462A4902200EF05FFD03212548FCF73F
S31508027E60DEFA9AE02248FCF762FA0346022B40F051
S31508027E7087801F48FCF776FA03460B2B44D1204B22
S31508027E801B68BA7ADA6300F06DFE0023FB600821EC
S31508027E901C4815F001FE0346012B12D1FB6801337B
S31508027EA0FB60FB681E2B04D901211248FCF7B7FABE
S31508027EB008E0FB79184613F01BFF642021F06AF9E3
S31508027EC0E5E700BF00F05CFE00F070FE65E000BF6B
S31508027ED074BA00207CB70508B0B70508E0B70508EC
S31508027EE078BA0020D5B80020228F002000B80508ED
S31508027EF07CBA002080BA00202405012024B805088F
S31508027F00BC050120001402424F48FCF72BFA03462F
S31508027F100C2B27D14D4B1B68BA7A1A6400F014FE53
S31508027F200023FB6004214A4815F0B6FD0346012BDF
S31508027F3012D1FB680133FB60FB681E2B04D90221B0
S31508027F404448FCF76CFA08E0FB79184613F0D0FEB1
S31508027F50642021F01FF9E5E700BF00F011FE00F0EA
S31508027F6025FE1AE03848FCF7FDF903461A463A494F
S31508027F7002200EF0D1FC03213648FCF750FA0CE039
S31508027F803148FCF7D4F903461A46344902200EF062
S31508027F90C3FC03212F48FCF742FA31492D48FCF766
S31508027FA019FC2F4829F012FC04462D4829F01AFC20
S31508027FB003461946204601F035FC40E029490220CD
S31508027FC00EF0AAFC28492948FCF750FC2648FCF77B
S31508027FD050FA0346002B0BD105F058FE0346022140
S31508027FE0184605F09DFE224902200EF095FC26E071
S31508027FF01D48FCF73EFA0346012B0BD105F046FE57
S3150802800003460321184605F08BFE1A4902200EF094
S3150802801083FC14E01448FCF72CFA03461A46164960
S3150802802002200EF079FC0AE0144B1B781A46144912
S3150802803002200EF071FC02E000BF00E000BF00BFA4
S315080280401037BD46B0BD00BF7CBA0020BC05012072
S315080280500014024280BA002024B8050858B8050858
S3150802806058B900208CB8050884BA0020D5B8002073
S31508028070ACB80508C8B80508E4B80508D4B800209D
S3150802808014B9050880B500AF084B1B78DBB2002B84
S3150802809008D1064B01221A7042F66872002104487A
S315080280A02EF05CF8024B184680BD00BF42EA00205B
S315080280B0D4BA002080B500AF074B1B78DBB2002B81
S315080280C007D1054B01221A700622002103482EF019
S315080280D045F8024B184680BD43EA00203CEA0020D8
S315080280E080B483B000AF78600B46FB70FB7841F230
S315080280F0B07202FB03F37A68134418460C37BD467E
S315080281005DF8047B704780B584B000AF78600B4693
S315080281107B800023FB730023BB7300237B7300233E
S31508028120FB7312E0FB7B19467868FFF7D9FFB86044
S31508028130BB681B887A889A4204D10123BB73FB7BEE
S315080281407B7305E0FB7B0133FB73FB7B012BE9D9D0
S31508028150BB7B002B07D07B7B41F2B07202FB03F399
S315080281607A68134400E0002318461037BD4680BDDE
S3150802817080B584B000AF78600B467B800023FB7322
S315080281800023BB7300237B730023FB7312E0FB7B84
S3150802819019467868FFF7A4FFB860BB681B887A8817
S315080281A09A4204D10123BB73FB7B7B7305E0FB7BFD
S315080281B00133FB73FB7B012BE9D9BB7B002B0BD06D
S315080281C07B7B19467868FFF78BFFB86041F2B0727D
S315080281D00021B8682DF0C2FF00BF1037BD4680BD2A
S315080281E080B483B000AF78607B6803F50053B3F8B8
S315080281F0603F18460C37BD465DF8047B704780B46D
S3150802820083B000AF78600B46FB70FB787A6803F59B
S31508028210BD53103332F8133018460C37BD465DF895
S31508028220047B704780B588B002AF78600B467B80C6
S3150802823013467B700023FB750023BB7500237B75F1
S315080282400023BB7400233B750023FB740023FB75D4
S315080282502EE0FB7D19467868FFF742FFF860FB6857
S315080282601B887A889A4201D101237B75FB7D1946C0
S315080282707868FFF7C4FF03461A467B88934202D101
S315080282800123BB7517E0FB7D19467868FFF7B7FF30
S315080282900346002B09D1BB7C002B06D1FB7C002BA5
S315080282A003D1FB7D3B750123FB74FB7D0133FB7513
S315080282B0FB7D012BCDD9BB7D012B02D07B7D002B0B
S315080282C009D17A88B97D7B7D00930B460E49022037
S315080282D00EF022FB14E03B7D7A6803F5BD5310339A
S315080282E0798822F813107B881946084813F0E6FBAA
S315080282F03B7D7A68134403F53D5326337A781A7020
S315080283001837BD4680BD00BF34B9050894B90508BB
S3150802831080B483B000AF78607B6803F50053B3F886
S31508028320643F18460C37BD465DF8047B704780B437
S3150802833083B000AF78607B6803F500530022A3F888
S31508028340642F00BF0C37BD465DF8047B704780B5C5
S3150802835084B000AF78600023FB817868FFF740FF9E
S315080283600346FB817B6803F500531A46FB89A2F88C
S31508028370643F00BF1037BD4680BD000090B589B086
S3150802838002AF78600B467B800023FB750023BB7522
S3150802839000233B610023BB817B6803F53D532033F1
S315080283A01B683B617B6803F53D5326331B889BB2EA
S315080283B0BB813B7B19467B7B1846BB7B1C46FB7BFA
S315080283C03A7C01920093234602463C4813F076FB18
S315080283D00023FB7518E0FB7D5B0018333B4433F83A
S315080283E0083C7A889A420CD1FB7D5B0018333B44E1
S315080283F0002223F8082CFB7D18333B44002203F89D
S315080284000C2CFB7D0133FB75FB7D012BE3D97B68C5
S3150802841003F53D5320330422002118462DF09EFE13
S315080284207B6803F53D5326330222002118462DF0B8
S3150802843095FE0023BB750023FB7528E0FB7D5B00D8
S3150802844018333B4433F8083C002B1DD0FB7DB97D1D
S315080284505B0018333B4433F8080C7A6801F5BD53C0
S315080284601033014622F81310FA7DBB7D591CB975E3
S31508028470194602F118033B4413F80C2C7B680B448B
S3150802848003F53D5326331A70FB7D0133FB75FB7DDD
S31508028490012BD3D97B8819467868FFF769FE786875
S315080284A0FFF736FF03461A467B88934202D178685D
S315080284B0FFF73DFF00BF1C37BD4690BDE0B9050872
S315080284C080B483B000AF78607B6803F5005393F8F5
S315080284D0663F18460C37BD465DF8047B70470000B8
S315080284E080B584B000AF786039600023FB7300233F
S315080284F0BB7300237B730023BB600023FB7311E06D
S31508028500FB7B19467868FFF7EBFDB860BB681B88EA
S31508028510002B04D10123BB73FB7B7B7305E0FB7B3A
S315080285200133FB73FB7B012BEAD9BB7B002B0FD0F4
S315080285307B7B19467868FFF7D3FDB86041F2B072C3
S315080285403968B8682DF0C1FE044902200EF0E4F934
S31508028550012318461037BD4680BD00BFF4BB050887
S3150802856080B483B000AF78607B685B7818460C37B6
S31508028570BD465DF8047B704780B483B000AF78606F
S315080285800B46FB707B68FA785A70012318460C373B
S31508028590BD465DF8047B704780B483B000AF78604F
S315080285A07B685B8818460C37BD465DF8047B7047C6
S315080285B080B483B000AF78600B467B807B687A888C
S315080285C05A80012318460C37BD465DF8047B70476E
S315080285D080B483B000AF78607B689B88DBB21846AC
S315080285E00C37BD465DF8047B704780B483B000AF94
S315080285F078600B46FB70FB789AB27B689A800123F7
S3150802860018460C37BD465DF8047B704780B500AF47
S31508028610184B1B78DBB2002B28D1164B01221A7095
S315080286202722022114482DF099FD134B012283F8C3
S31508028630202001220021104800F0B2F8012201216F
S315080286400D4800F0ADF8012202210B4800F0A8F807
S3150802865001220321084800F0A3F801220421064852
S3150802866000F09EF80121044800F0AEF8024B1846C5
S3150802867080BD00BF79EA002044EA002080B483B0B6
S3150802868000AF78607B68DB79012B01D1012306E014
S315080286907B68DB79022B01D1022300E0002318460E
S315080286A00C37BD465DF8047B704780B483B000AFD3
S315080286B078600B46FB707B68FA78DA7101231846F4
S315080286C00C37BD465DF8047B704780B483B000AFB3
S315080286D078600B46FB70FB787A6813441B7A012B89
S315080286E001D1012308E0FB787A6813441B7A022B2E
S315080286F001D1022300E0002318460C37BD465DF877
S31508028700047B704780B483B000AF78600B46FB7079
S315080287101346BB70FB787A681344BA781A72012337
S3150802872018460C37BD465DF8047B704780B483B0A3
S3150802873000AF78600B46FB70FB787A6813441B7BA4
S31508028740012B01D1012308E0FB787A6813441B7BCD
S31508028750022B01D1022300E0002318460C37BD463E
S315080287605DF8047B704780B483B000AF78600B462F
S31508028770FB70FB787A6813445B7D012B01D10123D8
S3150802878008E0FB787A6813445B7D022B01D1022349
S3150802879000E0002318460C37BD465DF8047B704797
S315080287A080B483B000AF78600B46FB701346BB708B
S315080287B0FB787A681344BA785A75012318460C3737
S315080287C0BD465DF8047B704780B483B000AF78601D
S315080287D00B46FB707B68FA781A77012318460C3722
S315080287E0BD465DF8047B704780B582B000AF03468C
S315080287F0FB71FB791846F7F7B3FF02460B46384971
S31508028800C1E90023FB79002B3FD0FB79194635488D
S3150802881013F054F9FFF7FAFE03460321184600F04F
S3150802882020FAFFF7F3FE0346184600F02AFA034633
S31508028830012B10D12C4B1B68FA799A632B4B1B78A8
S31508028840002B49D0042128481BF08CFB0821264816
S315080288501BF0E8FC40E0FFF7D9FE0346184600F095
S3150802886010FA0346022B37D11F4B1B68FA79DA63D3
S315080288701E4B1B78002B2FD004211B481BF0D2FC61
S31508028880082119481BF06EFB26E0FB79002B23D141
S31508028890FFF7BCFE0346184600F0D6F90346012B3D
S315080288A006D0FFF7B3FE03460421184600F0D9F9AD
S315080288B00F4B1B78002B0FD10B4B1B6863229A6355
S315080288C0094B1B686322DA63042107481BF04AFB3B
S315080288D0082105481BF046FB00BF0837BD4680BD88
S315080288E070EA002014BC05087005012078EA002009
S315080288F0C404022080B400AF064BD3E9002343EC3C
S31508028900172BB0EE470AF0EE670ABD465DF8047B00
S31508028910704700BF70EA002080B500AFFFF776FE09
S3150802892003460321184600F09CF900F0B7F8FFF752
S31508028930E1FF51EC100B4FF000024FF00003F8F77D
S31508028940F1F90346002B08D004210A481BF06AFCF9
S31508028950082108481BF066FC07E0042105481BF0BD
S3150802896001FB082103481BF05DFC034B01221A7028
S3150802897000BF80BD7005012078EA002080B500AFEF
S31508028980FFF744FE03460421184600F06AF9044B31
S3150802899000221A700020FFF727FF00BF80BD00BF24
S315080289A078EA002080B500AFFFF730FE03460321C0
S315080289B0184600F056F900F07CF8FFF79BFF51ECD9
S315080289C0100B4FF000024FF00003F8F7ABF903461D
S315080289D0002B08D004210A481BF024FC0821084869
S315080289E01BF020FC07E0042105481BF01BFC0821AC
S315080289F003481BF0B7FA034B01221A7000BF80BD69
S31508028A007005012078EA002080B500AFFFF7FEFD69
S31508028A1003460421184600F024F9054B00221A7071
S31508028A200020FFF7E1FE00F039F800BF80BD00BF65
S31508028A3078EA002080B500AFFFF7E8FD0346022179
S31508028A40184600F00EF9042105481BF0EBFB082135
S31508028A5003481BF0E7FB034B00221A7000BF80BDD8
S31508028A607005012078EA002080B500AFFFF7CEFD39
S31508028A7003460121184600F0F4F8042105481BF0C4
S31508028A80D1FB082103481BF0CDFB034B00221A70C9
S31508028A9000BF80BD7005012078EA002080B500AFCE
S31508028AA0FFF7B4FD03460121184600F0F7F800BFA8
S31508028AB080BD80B500AFFFF7A9FD0346022118461F
S31508028AC000F0ECF800BF80BD80B500AF082104486D
S31508028AD01BF048FA0C2102481BF0A4FB00BF80BD1C
S31508028AE02405012080B500AF082104481BF09AFB33
S31508028AF00C2102481BF036FA00BF80BD240501206E
S31508028B0080B500AF084B1B686322DA63064B1B6805
S31508028B1063221A64082104481BF024FA0C2102482D
S31508028B201BF020FA00BF80BD2405012080B500AFE6
S31508028B30082104481BF076FB0C2102481BF072FB45
S31508028B4000BF80BD2405012080B500AF0C21044872
S31508028B501BF008FA082102481BF064FB00BF80BD1F
S31508028B60BC05012080B500AF0C2104481BF05AFB56
S31508028B70082102481BF0F6F900BF80BDBC0501209A
S31508028B8080B500AF084B1B6863221A64064B1B6844
S31508028B906322DA630C2104481BF0E4F9082102482F
S31508028BA01BF0E0F900BF80BDBC05012080B500AF0F
S31508028BB00C2104481BF036FB082102481BF032FB45
S31508028BC000BF80BDBC05012080B500AF0421044862
S31508028BD01BF0C8F9002102481BF024FB00BF80BD28
S31508028BE0BC05012080B500AF042104481BF01AFB1E
S31508028BF0002102481BF0B6F900BF80BDBC05012062
S31508028C0080B500AF084B1B6863229A63064B1B6844
S31508028C1063225A63042104481BF0A4F9002102487E
S31508028C201BF0A0F900BF80BDBC05012080B500AFCE
S31508028C30042104481BF0F6FA002102481BF0F2FA56
S31508028C4000BF80BDBC05012080B483B000AF786048
S31508028C507B6893F8233018460C37BD465DF8047BCB
S31508028C60704780B483B000AF78600B46FB707B68B0
S31508028C70FA7883F8232000BF0C37BD465DF8047BDB
S31508028C80704780B483B000AF78607B6893F826306B
S31508028C9018460C37BD465DF8047B704780B483B02E
S31508028CA000AF78600B46FB707B68FA7883F826205B
S31508028CB0012318460C37BD465DF8047B704780B41D
S31508028CC083B000AF78600B46FB70FB787A68134472
S31508028CD09B7F012B01D1012308E0FB787A681344B4
S31508028CE09B7F022B01D1022300E0002318460C3792
S31508028CF0BD465DF8047B704780B483B000AF7860E8
S31508028D000B46FB701346BB70FB787A681344BA7835
S31508028D109A77012318460C37BD465DF8047B7047DF
S31508028D2080B582B000AF4FF48071434814F0B4FEA8
S31508028D300346012B0CBF01230023DBB2BB710023C0
S31508028D40FB71BB79012B02D13C4812F0B7FE3C4BB2
S31508028D501B78BA799A421BD13A4B1B78012B02D956
S31508028D60BB79FB7128E0374B1B780133DAB2354BF6
S31508028D701A70FFF74BFC03461846FFF77FFC0346BB
S31508028D80012B02D10123FB7116E00023FB7113E0CC
S31508028D902B4ABB7913702B4B00221A70FFF736FC4D
S31508028DA003461846FFF76AFC0346012B02D1012344
S31508028DB0FB7101E00023FB71FB79002B1CD0FFF746
S31508028DC025FC034601211846FFF76FFC1E4B1B784C
S31508028DD0FA799A422CD00CF0F7FF0346042118467A
S31508028DE00DF0B4FB0346002B02D0184812F066FEBB
S31508028DF0154AFB7913701BE0FFF708FC03460221AC
S31508028E001846FFF752FC104B1B78FA799A420FD094
S31508028E100CF0DAFF0346042118460DF097FB0346C9
S31508028E20002B02D00A4812F049FE074AFB79137052
S31508028E3000BF0837BD4680BD000C0242C4BF050804
S31508028E407AEA00207BEA00207CEA0020D4BF0508E3
S31508028E5010C0050880B582B000AF4FF48051424871
S31508028E6014F01AFE0346012B0CBF01230023DBB2C2
S31508028E70BB710023FB713D4B1B78BA799A421CD110
S31508028E803B4B1B78032B02D9BB79FB712AE0384B83
S31508028E901B780133DAB2364B1A70FFF7B7FB034673
S31508028EA000211846FFF711FC0346012B02D10123C4
S31508028EB0FB7117E00023FB7114E02C4ABB7913708F
S31508028EC02B4B00221A70FFF7A1FB03460021184616
S31508028ED0FFF7FBFB0346012B02D10123FB7101E0DD
S31508028EE00023FB71FB79002B1DD0FFF78FFB03468E
S31508028EF0012200211846FFF705FC1E4B1B78FA795A
S31508028F009A422DD00CF060FF0346042118460DF054
S31508028F101DFB0346002B02D0174812F0CFFD154A57
S31508028F20FB7913701CE0FFF771FB0346022200214E
S31508028F301846FFF7E7FB0F4B1B78FA799A420FD0D0
S31508028F400CF042FF0346042118460DF0FFFA0346C9
S31508028F50002B02D0094812F0B1FD064AFB791370BC
S31508028F6000BF0837BD4680BD000C02427DEA0020DC
S31508028F707EEA00207FEA00204CC0050888C0050862
S31508028F8080B582B000AF4FF40061424814F084FD08
S31508028F900346012B0CBF01230023DBB2BB7100235E
S31508028FA0FB713D4B1B78BA799A421CD13B4B1B7815
S31508028FB0032B02D9BB79FB712AE0384B1B780133A4
S31508028FC0DAB2364B1A70FFF721FB0346012118461F
S31508028FD0FFF77BFB0346012B02D10123FB7117E046
S31508028FE00023FB7114E02C4ABB7913702B4B002229
S31508028FF01A70FFF70BFB034601211846FFF765FBBC
S315080290000346012B02D10123FB7101E00023FB7108
S31508029010FB79002B1DD0FFF7F9FA0346012201213D
S315080290201846FFF76FFB1E4B1B78FA799A422DD02A
S315080290300CF0CAFE0346042118460DF087FA0346C9
S31508029040002B02D0174812F039FD154AFB79137026
S315080290501CE0FFF7DBFA0346022201211846FFF756
S3150802906051FB0F4B1B78FA799A420FD00CF0ACFEE3
S315080290700346042118460DF069FA0346002B02D06E
S31508029080094812F01BFD064AFB79137000BF083720
S31508029090BD4680BD000C024280EA002081EA00201B
S315080290A082EA0020C8C0050804C1050880B582B056
S315080290B000AF4FF48061424814F0EEFC0346012BE0
S315080290C00CBF01230023DBB2BB710023FB713D4BAE
S315080290D01B78BA799A421CD13B4B1B78032B02D9CF
S315080290E0BB79FB712AE0384B1B780133DAB2364B6F
S315080290F01A70FFF78BFA034602211846FFF7E5FABC
S315080291000346012B02D10123FB7117E00023FB71F1
S3150802911014E02C4ABB7913702B4B00221A70FFF706
S3150802912075FA034602211846FFF7CFFA0346012BC2
S3150802913002D10123FB7101E00023FB71FB79002BAD
S315080291401DD0FFF763FA0346012202211846FFF7EC
S31508029150D9FA1E4B1B78FA799A422DD00CF034FEB6
S315080291600346042118460DF0F1F90346002B02D0F6
S31508029170174812F0A3FC154AFB7913701CE0FFF797
S3150802918045FA0346022202211846FFF7BBFA0F4B9D
S315080291901B78FA799A420FD00CF016FE0346042180
S315080291A018460DF0D3F90346002B02D0094812F0EF
S315080291B085FC064AFB79137000BF0837BD4680BD99
S315080291C0000C024283EA002084EA002085EA002095
S315080291D044C1050880C1050880B582B000AF4FF4C6
S315080291E00071424814F058FC0346012B0CBF0123B8
S315080291F00023DBB2BB710023FB713D4B1B78BA79A6
S315080292009A421CD13B4B1B78032B02D9BB79FB71C3
S315080292102AE0384B1B780133DAB2364B1A70FFF75D
S31508029220F5F9034603211846FFF74FFA0346012BC1
S3150802923002D10123FB7117E00023FB7114E02C4ACB
S31508029240BB7913702B4B00221A70FFF7DFF903461E
S3150802925003211846FFF739FA0346012B02D10123E7
S31508029260FB7101E00023FB71FB79002B1DD0FFF790
S31508029270CDF90346012203211846FFF743FA1E4B8E
S315080292801B78FA799A422DD00CF09EFD03460421EA
S3150802929018460DF05BF90346002B02D0174812F068
S315080292A00DFC154AFB7913701CE0FFF7AFF903466C
S315080292B0022203211846FFF725FA0F4B1B78FA7983
S315080292C09A420FD00CF080FD0346042118460DF091
S315080292D03DF90346002B02D0094812F0EFFB064A75
S315080292E0FB79137000BF0837BD4680BD000C0242E9
S315080292F086EA002087EA002088EA0020C0C105081D
S31508029300FCC1050880B582B000AF0121424814F0BD
S31508029310C3FB0346012B0CBF01230023DBB2BB713F
S315080293200023FB713D4B1B78BA799A421CD13C4B00
S315080293301B788B2B02D9BB79FB712AE0384B1B7839
S315080293400133DAB2364B1A70FFF760F90346002189
S315080293501846FFF7B4FC0346022B02D10123FB7120
S3150802936017E00023FB7114E02C4ABB7913702C4BCF
S3150802937000221A70FFF74AF9034600211846FFF73A
S315080293809EFC0346022B02D10123FB7101E0002356
S31508029390FB71FB79002B1DD0FFF738F90346022231
S315080293A000211846FFF7A8FC1E4B1B78FA799A4249
S315080293B02DD00CF009FD0346042118460DF0C6F817
S315080293C00346002B02D0184812F078FB154AFB799F
S315080293D013701CE0FFF71AF903460122002118460A
S315080293E0FFF78AFC0F4B1B78FA799A420FD00CF0DA
S315080293F0EBFC0346042118460DF0A8F80346002B99
S3150802940002D00A4812F05AFB064AFB79137000BFCB
S315080294100837BD4680BD00BF0014024289EA002013
S315080294208AEA00208BEA002088CA0508C8CA050805
S3150802943080B582B000AF0221424814F02DFB0346E4
S31508029440012B0CBF01230023DBB2BB710023FB7186
S315080294503D4B1B78BA799A421CD13C4B1B788B2B15
S3150802946002D9BB79FB712AE0384B1B780133DAB291
S31508029470364B1A70FFF7CAF8034601211846FFF75A
S315080294801EFC0346022B02D10123FB7117E00023BF
S31508029490FB7114E02C4ABB7913702C4B00221A700C
S315080294A0FFF7B4F8034601211846FFF708FC0346FE
S315080294B0022B02D10123FB7101E00023FB71FB7928
S315080294C0002B1DD0FFF7A2F80346022201211846F7
S315080294D0FFF712FC1E4B1B78FA799A422DD00CF034
S315080294E073FC0346042118460DF030F80346002B98
S315080294F002D0184812F0E2FA154AFB7913701CE0FA
S31508029500FFF784F80346012201211846FFF7F4FB08
S315080295100F4B1B78FA799A420FD00CF055FC03468A
S31508029520042118460DF012F80346002B02D00A4809
S3150802953012F0C4FA064AFB79137000BF0837BD4613
S3150802954080BD00BF001402428CEA00208DEA00208A
S315080295508EEA002008CB050844CB050880B582B000
S3150802956000AF78600B467B80144822F017F9024652
S315080295707B889A4217D34FF47A71114820F052FD2C
S315080295800346002B14D17B881A4679680B4822F0C9
S31508029590EEFA0346002B02D10A4812F08FFA08485F
S315080295A020F09AFD04E0084812F088FA002300E049
S315080295B0012318460837BD4680BD00BF90EA002041
S315080295C03091002084CB050898CB050880B5ADF507
S315080295D0016D00AF024607F50163A3F609031A7087
S315080295E0002387F80F3850E007F10C034FF40062A6
S315080295F0002118462CF0B2FD4FF47A712C4820F05F
S3150802960011FD0346002B0BD107F10C031946294815
S3150802961022F024FB034687F80F38254820F05CFD24
S315080296204FF47A71224820F0FDFC0346002B0BD139
S3150802963007F10C0319461F4822F0AAFA034687F8CF
S315080296400F381B4820F048FD4FF47A711A4820F06B
S31508029650E9FC0346002B0DD1FCF779F897F80F3889
S315080296609AB207F10C031946FCF7B2F9124820F030
S3150802967033FD02E0114812F021FA07F50163A3F659
S3150802968009031B78184612F033FB0A4822F0E4F85D
S31508029690034683F00103DBB2002B03D0084B1B7889
S315080296A0002BA1D000BF07F50167BD4680BD00BFEC
S315080296B03091002090EA002064910020A8CB05088A
S315080296C0A0F2002080B483B000AF78600B467B809E
S315080296D000BF00BF0C37BD465DF8047B704700002B
S315080296E080B582B000AF0023FB712E4B1B78002B8E
S315080296F051D02D4B1B780133DAB22B4B1A702A4BF9
S315080297001B78092B4AD9284B00221A70254B5B78FD
S31508029710012B1FD8234B5B780133DAB2214B5A70DF
S315080297204FF47A71214820F07DFC0346002B0DD1B7
S31508029730FCF70DF803461B4A92F883201C49184683
S31508029740FCF746F9194820F0C7FC27E0194812F039
S31508029750B5F923E00023FB7102E0FB790133FB71C3
S31508029760104B93F88330FA799A42F6D34FF47A710A
S31508029770114820F057FC0346002B06D10C490F4826
S3150802978022F006FA0C4820F0A7FC8422002105489C
S315080297902CF0E4FC02E0044B00221A7000BF0837E2
S315080297A0BD4680BDA0F2002024F30020649100206B
S315080297B0A3F20020A8CB05083091002090EA0020E9
S315080297C080B500AF4FF400620249034821F0BAFFA0
S315080297D000BF80BDA0EA002090EA002080B500AF55
S315080297E0FFF7EEFF00BF80BD80B582B000AF78609C
S315080297F039603B68DBB21946786800F04BF800BF5F
S315080298000837BD4680BD80B582B000AF7860396042
S315080298103B689BB219467868FFF7A0FE00BF083777
S31508029820BD4680BD80B582B000AF78603960064B10
S315080298301B683A6892B27968184621F07EFD00BF25
S315080298400837BD4680BD00BFE012002080B582B051
S3150802985000AF78603960054B1B683A687968184624
S3150802986021F004FE00BF0837BD4680BDE012002085
S3150802987080B500AF044B1868044B054A002121F055
S3150802988021FD00BF80BD00BFE01200200798020834
S31508029890E9970208F0B587B002AF78600B46FB700D
S315080298A00CF092FAF860FB789BB219467868FFF7D3
S315080298B009FF7B681B78013B7F2B00F2B08601A269
S315080298C052F823F0C59A02081FA602081FA6020824
S315080298D01FA602082B9B02081FA602081FA602083B
S315080298E01FA602081FA602081FA602081FA602082C
S315080298F01FA602081FA602081FA60208019B020845
S315080299001FA602081FA602081FA602081FA602080B
S315080299101FA602081FA602081FA602081FA60208FB
S315080299201FA602081FA602081FA602081FA60208EB
S315080299301FA602081FA602081FA602081FA60208DB
S315080299401FA60208599B0208339C0208019D0208B9
S315080299501FA602081FA602081FA602081FA60208BB
S315080299600B9D0208559D02081FA602081FA602089B
S315080299701FA602081FA602081FA602081FA602089B
S315080299805F9D0208D19E0208E79F02081FA60208E9
S315080299901FA602081FA602081FA602081FA602087B
S315080299A01FA602081FA602081FA602081FA602086B
S315080299B01FA602081FA602081FA602081FA602085B
S315080299C01FA602081FA602081FA602081FA602084B
S315080299D01FA602081FA602081FA602081FA602083B
S315080299E01FA602081FA602081FA602081FA602082B
S315080299F01FA602081FA602081FA602081FA602081B
S31508029A001FA602081FA602081FA602081FA602080A
S31508029A101FA602081FA602081FA602081FA60208FA
S31508029A201FA602081FA602081FA602081FA60208EA
S31508029A301FA602081FA602081FA602081FA60208DA
S31508029A402FA202081FA602081FA602081FA60208BE
S31508029A501FA602081FA602081FA602081FA60208BA
S31508029A601FA602081FA602081FA602081FA60208AA
S31508029A701FA602081FA602081FA602081FA602089A
S31508029A8011A302082BA40208FBA402081FA60208B7
S31508029A901FA602081FA602081FA602081FA602087A
S31508029AA01FA602081FA602081FA602081FA602086A
S31508029AB01FA602081FA602081FA602081FA602085A
S31508029AC0D3A50208BC4B9B781946BC4827F0A2FED0
S31508029AD0B94BDB781946B94827F0B8FEB849B748F2
S31508029AE027F026FEB64827F071FE0446B44827F04A
S31508029AF079FE034619462046FFF794FE00F090BD0C
S31508029B00B04B01221A70AE49AE4827F034FEAC4873
S31508029B1027F05CFE0446AA4827F064FE0346194667
S31508029B202046FFF77FFE00F07BBDA74811F0C6FF6F
S31508029B30F8680CF095F9A24827F036FEA04827F0F7
S31508029B4045FE04469E4827F04DFE03461946204622
S31508029B50FFF768FE00F064BD9C4811F0AFFF7B6812
S31508029B6001339B49184621F081F820F043FC03464D
S31508029B70184620F096FC03461C46954820F0CAFC77
S31508029B8003469C4211D1924820F0C4FC03461C4667
S31508029B9020F030FC0346184620F083FC03461A469A
S31508029BA021468C4811F08AFF31E0894820F0B2FC40
S31508029BB0874820F0AFFC03460F2B1ED8844820F0B6
S31508029BC0A9FC03461C46824820F0BFFC03461A46F7
S31508029BD02146814811F072FF20F00CFC04467C48AD
S31508029BE020F098FC03461946204620F066FCFB78CE
S31508029BF019467868FDF750FB09E0754820F08AFC9B
S31508029C00034619460F230022744811F057FF6C4980
S31508029C106F4821F052F86A4827F0D8FD044668488A
S31508029C2027F0E0FD034619462046FFF7FBFD00F044
S31508029C30F7BC6B4811F042FF7B6801336949184645
S31508029C4021F06FF820F0D6FB0346184620F029FCCF
S31508029C5003461C46634820F093FC03469C4211D1F6
S31508029C60604820F08DFC03461C4620F0C3FB0346E1
S31508029C70184620F016FC03461A4621465A4811F0A1
S31508029C801DFF2BE0574820F07BFC564820F078FC55
S31508029C9003460F2B18D8534820F072FC0346194680
S31508029CA0524811F00BFF20F0A5FB04464D4820F060
S31508029CB067FC03461946204620F0FFFBFB78194647
S31508029CC07868FDF7E9FA09E0464820F059FC0346A8
S31508029CD019460F230022464811F0F0FE384941483A
S31508029CE021F03BF8364827F071FD0446344827F040
S31508029CF079FD034619462046FFF794FD00F090BC0D
S31508029D003C4811F0DBFE00F08BBC3B4811F0D6FE56
S31508029D100122002139482CF021FA20F06BFB034678
S31508029D20184620F0BEFB03461946344820F04FFC7D
S31508029D302349324821F027F8214827F047FD0446EF
S31508029D401F4827F04FFD034619462046FFF76AFDCE
S31508029D5000F066BC2A4811F0B1FE00F061BC294841
S31508029D6011F0ACFE7B6801332749184621F04FF8FB
S31508029D7020F040FB0346184620F093FB03461C4698
S31508029D80214820F033FC03469C4243D102211F4856
S31508029D9020F0A4FC1C4820F029FC03461C4620F0AF
S31508029DA029FB0346184620F07CFB03461A46214641
S31508029DB0174811F083FE67E0E0BF1F085C04012024
S31508029DC05403012058040120C8CB0508E4CB050832
S31508029DD06004012000CC05082CCC05085CCC0508DB
S31508029DE08CCC050864040120ACCC0508DCCC05083B
S31508029DF004CD050838CD050854CD050868040120A8
S31508029E0070CD050890CD05086C0401207804012060
S31508029E10A8CD05088A4820F0E9FB894820F0E6FB28
S31508029E2003460F2B22D80021864820F057FC844887
S31508029E3020F0DCFB03461C46814820F0F2FB034671
S31508029E401A462146804811F039FE20F0D3FA044614
S31508029E507B4820F0CBFB03461946204620F02DFB13
S31508029E60FB7819467868FDF717FA0DE0012175485F
S31508029E7020F034FC724820F0B9FB034619460F233A
S31508029E800022724811F01AFE20F0B4FA0346184668
S31508029E9020F0E9FA034619466A4820F0E9FB6848C1
S31508029EA020F0BFFB03461946664820F0FCFB6849CA
S31508029EB0644820F0D3FF664827F088FC04466448C5
S31508029EC027F090FC034619462046FFF7ABFCA7E3AA
S31508029ED0604811F0F3FD7B6801335F49184621F0AB
S31508029EE03FF820F087FA0346184620F0DAFA0346C6
S31508029EF01C46594820F052FC03469C4215D10221C1
S31508029F00564820F0C3FC544820F048FC03461C4639
S31508029F1020F070FA0346184620F0C3FA03461A469A
S31508029F2021464F4811F0CAFD39E04B4820F036FC6D
S31508029F30494820F033FC03460F2B22D80021474814
S31508029F4020F0A4FC444820F029FC03461C4642485B
S31508029F5020F03FFC03461A462146424811F0AEFD60
S31508029F6020F048FA04463C4820F018FC03461946F5
S31508029F70204620F0A2FAFB7819467868FDF78CF994
S31508029F800DE00121354820F081FC334820F006FC1B
S31508029F90034619460F230022334811F08FFD20F09D
S31508029FA029FA0346184620F05EFA034619462B4854
S31508029FB020F036FC284820F00CFC034619462748B0
S31508029FC020F049FC2249254820F0F1FF204827F0D5
S31508029FD0FDFB04461E4827F005FC034619462046A3
S31508029FE0FFF720FC1CE3214811F068FD7B6801336A
S31508029FF01F49184621F055F820F0FCF90346184681
S3150802A00020F04FFA03461C46194820F09FFC0346E7
S3150802A0109C4233D10221174820F0BEFD144820F095
S3150802A02095FC03461C4620F0E5F90346184620F03F
S3150802A03038FA03461A4621460F4811F03FFDDAE080
S3150802A0406C04012078040120D0CD0508F8CD050856
S3150802A0505403012024CE0508700401207C04012043
S3150802A06040CE05086CCE050898CE0508C8CE050868
S3150802A0707404012080040120E4CE0508CF4820F0AC
S3150802A08065FCCE4820F062FC03460F2B00F2A58041
S3150802A0900021CB4820F080FDC84820F057FC034633
S3150802A0A01946C84811F00AFD20F0A4F90446C34827
S3150802A0B020F04CFC03461946204620F0FEF9FB78B0
S3150802A0C019467868FDF7E8F80BF07EFE034618464F
S3150802A0D00BF0EAFFF0EE407AB0EE670AFDF752F9A6
S3150802A0E003461946B64820F073FC0BF06DFE03468C
S3150802A0F018460BF0F7FFF0EE407AB0EE670AFDF766
S3150802A10041F903461946AE4820F07DFC0BF05CFE89
S3150802A110034618460CF004F8F0EE407AB0EE670AE9
S3150802A120FDF730F903461946A54820F087FC0BF0DF
S3150802A1304BFE034618460CF011F8F0EE407AB0EEE4
S3150802A140670AFDF71FF9034619469D4820F091FC58
S3150802A1500BF03AFE034618460CF01EF8F0EE407A6B
S3150802A160B0EE670AFDF70EF903461946944820F041
S3150802A1709BFC0BF029FE034618460CF02BF8F0EE72
S3150802A180407AB0EE670AFDF7FDF8034619468C4891
S3150802A19020F0A5FC0BF018FE034618460CF038F81A
S3150802A1A0F0EE407AB0EE670AFDF7ECF80346194678
S3150802A1B0834820F0AFFC0BF007FE034618460CF066
S3150802A1C045F8F0EE407AB0EE670AFDF7DBF803468B
S3150802A1D019467B4820F0B9FC0DE00121784820F0A9
S3150802A1E0DBFC764820F0B2FB034619460F23002211
S3150802A1F0754811F063FC20F0FDF80346184620F076
S3150802A20032F9034619466E4820F0C7FB6F496C4877
S3150802A21020F063FF6D4827F0D9FA04466B4827F009
S3150802A220E1FA034619462046FFF7FCFAF8E16848C0
S3150802A23011F044FC7B68013366491846FAF799F926
S3150802A24020F0D8F80346184620F02BF903461C4698
S3150802A2506048F9F7AFFF03469C4211D15D48F9F70A
S3150802A260A9FF03461C4620F0C5F80346184620F007
S3150802A27018F903461A462146574811F01FFC36E0DC
S3150802A2805448F9F797FF5348F9F794FF03460F2BFB
S3150802A29023D85048F9F78EFF03461C464D48F9F76E
S3150802A2A0A4FF03461D464B48F9F7BAFF03462A465A
S3150802A2B021464A4811F002FC20F09CF8044645481B
S3150802A2C0F9F778FF03461946204620F0F6F8FB7898
S3150802A2D019467868FCF7E0FF09E03E48F9F76AFF95
S3150802A2E0034619460F2300223D4811F0E7FB37497A
S3150802A2F03848FAF770F9354827F068FA04463348B9
S3150802A30027F070FA034619462046FFF78BFA87E1CB
S3150802A310344811F0D3FB7B68013333491846FAF700
S3150802A3209EF920F067F80346184620F0BAF8034665
S3150802A3301C462D48F9F78FFF03469C4211D12A483D
S3150802A340F9F789FF03461C4620F054F803461846D7
S3150802A35020F0A7F803461A462146244811F0AEFB18
S3150802A36052E02148F9F777FF1F48F9F774FF0346C9
S3150802A3700F2B3FD81C48F9F76EFF03461C461A48AE
S3150802A380F9F784FF03461D461748F9F79AFF03466D
S3150802A3902A462146164811F091FB20F02BF804466E
S3150802A3A01148F9F758FF03461946204620F085F862
S3150802A3B0FB7819467868FCF76FFF25E074040120DC
S3150802A3C08004012010CF050838CF05085403012060
S3150802A3D068CF05089804012088CF0508B4CF050878
S3150802A3E0E8CF05081CD005089C0401203CD00508C6
S3150802A3F068D005088C48F9F72EFF034619460F233D
S3150802A40000228A4811F05AFB89498748FAF759F90E
S3150802A410874827F0DBF90446854827F0E3F903461F
S3150802A42019462046FFF7FEF9FAE0824811F046FB84
S3150802A4307B68013380491846FAF78FF91FF0DAFF6D
S3150802A4400346184620F02DF803461C467A48F9F7C3
S3150802A45053FF03469C4211D17748F9F74DFF03464D
S3150802A4601C461FF0C7FF0346184620F01AF8034693
S3150802A4701A462146714811F021FBD1E06E48F9F7D8
S3150802A4803BFF6D48F9F738FF03460F2B2AD86A486F
S3150802A490F9F732FF03461C466748F9F748FF0346B1
S3150802A4A01D466548F9F75EFF03461E466248F9F7F8
S3150802A4B074FF0346009333462A462146604811F044
S3150802A4C0FDFA1FF097FF04465B48F9F715FF0346A6
S3150802A4D0194620461FF0F1FFFB7819467868FCF703
S3150802A4E0DBFE9DE05448F9F707FF034619460F239A
S3150802A4F00022544811F0E2FA92E0534811F0DEFACB
S3150802A5007B68013351491846FAF7B0F91FF072FF12
S3150802A510034618461FF0C5FF03461C464B48F9F783
S3150802A5208DFF03469C4211D14848F9F787FF034637
S3150802A5301C461FF05FFF034618461FF0B2FF03468C
S3150802A5401A462146424811F0B9FA31E03F48F9F76E
S3150802A55075FF3E48F9F772FF03460F2B1ED83B4894
S3150802A560F9F76CFF03461C463848F9F782FF03469B
S3150802A5701A462146374811F0A1FA1FF03BFF044656
S3150802A5803248F9F75BFF0346194620461FF095FF46
S3150802A590FB7819467868FCF77FFE09E02B48F9F73D
S3150802A5A04DFF034619460F2300222B4811F086FA5F
S3150802A5B01F492648FAF781F91D4827F007F9044684
S3150802A5C01B4827F00FF9034619462046FFF72AF9D2
S3150802A5D026E07B68013321491846FAF784F90BF01D
S3150802A5E0F3FB034618460BF024FC04461B48F9F70E
S3150802A5F05BFF034619462046F6F7CCFF0C49174877
S3150802A600FAF78DF90A4827F0E1F80446084827F0D0
S3150802A610E9F8034619462046FFF704F900E000BFA9
S3150802A62000BF1437BD46F0BD9C0401209CD0050826
S3150802A63054030120D0D00508A0040120F0D0050853
S3150802A64020D1050860D1050894D10508A404012083
S3150802A650B4D10508E0D1050810D20508A8040120DE
S3150802A66080B500AF03481BF057FB02481BF014FAEB
S3150802A67000BF80BD5406012080B500AF00F0FCFB88
S3150802A68011F00CFA00BF80BDB0B594B000AF5C4BB8
S3150802A690D3F8F430002B09DA5A4811F00FFA07F109
S3150802A6A048030621184622F0DEF95DE0544BD3F83A
S3150802A6B0F43003F08043002B09D0534811F0FEF919
S3150802A6C007F148030521184622F0CDF94CE04C4B18
S3150802A6D0D3F8F43003F00053002B09D04B4811F09D
S3150802A6E0EDF907F148030421184622F0BCF93BE0CC
S3150802A6F0434BD3F8F43003F08053002B09D0444877
S3150802A70011F0DCF907F148030321184622F0ABF9E8
S3150802A7102AE03B4BD3F8F43003F00063002B09D050
S3150802A7203C4811F0CBF907F148030221184622F0FA
S3150802A7309AF919E0324BD3F8F43003F08063002B10
S3150802A74009D0354811F0BAF907F14803012118462C
S3150802A75022F089F908E0314811F0B0F907F1480307
S3150802A7600021184622F07FF9254BD3F8F430244A03
S3150802A77043F40003C2F8F430294826F00EFF0346D4
S3150802A7801B0ADAB207F148031146184622F086F97F
S3150802A790234826F002FF0346DAB207F148031146B8
S3150802A7A0184622F096F91F4B9A7807F14803114684
S3150802A7B0184622F0A9F91B4BDA7807F14803114625
S3150802A7C0184622F0BCF93A1D07F148031146184605
S3150802A7D022F011FD22F03CFF04463B1D184622F0EA
S3150802A7E0FEFA05463B1D184622F005FB03461A46A5
S3150802A7F0294620462AF018F800BF5037BD46B0BD94
S3150802A800000C024444D2050860D205087CD2050829
S3150802A81098D20508B8D20508D0D20508E8D20508A4
S3150802A82000E00108E0BF1F0880B500AF214B224AAD
S3150802A8309A6062B600BF11F01BFB00F045F800F003
S3150802A84067FB00F015F900F0F1F800F0A7F800F040
S3150802A85013FB00F053FA00F0CFF900F0E7FA00F024
S3150802A8600FF9164819F06EFA0BF0AEFA0BF0ACFABD
S3150802A870034618460BF0DDFA03461846F6F77CFD42
S3150802A880FEF7ACFF0E48FAF73BFEFEF7F1FF11F0B2
S3150802A89005F900F009FE29F041FE04F0A5FB0122A4
S3150802A8A04FF40041074813F00FF9F9F77DFC00BF92
S3150802A8B0FDE700BF00ED00E00000020808060120DF
S3150802A8C0AC0401200004024280B59CB000AF07F137
S3150802A8D020035022002118462BF040FC07F10803FA
S3150802A8E000221A605A609A60DA601A615A612A4B23
S3150802A8F01B69294A43F030031361274B1B6903F08E
S3150802A90030037B607B6800BF234B5B6903F0080357
S3150802A910082BF9D109233B624FF480337B624FF04F
S3150802A9208063BB630223BB640323FB6403233B6587
S3150802A9307D237B650223BB650223FB6502233B66F7
S3150802A94008237B660023BB660023FB6607F1200308
S3150802A950184613F09BF90346002B01D000F03CFC85
S3150802A9601F23BB600323FB6000233B6100237B613B
S3150802A9700023BB610023FB6107F108030521184682
S3150802A98013F0BCFD0346002B01D000F025FC00BFE6
S3150802A9907037BD4680BD00BF0008024480B500AFCF
S3150802A9A0204B214A1A601F4B00225A601D4B4FF456
S3150802A9B040729A601B4B0022DA601A4B00221A7404
S3150802A9C0184B00225A74174B00229A74154B05220B
S3150802A9D05A61144B0A229A61124B2722DA61114BE9
S3150802A9E00A221A620F4B05225A620E4B02229A62F9
S3150802A9F00C4B0722DA620B4B02221A63094B01221D
S3150802AA005A63084B01229A63064B0022DA63054809
S3150802AA1011F02CFC0346002B01D000F0DDFB00BF31
S3150802AA2080BD00BFAC04012000A4004080B500AF81
S3150802AA300D4B0E4A1A600C4B05225A600A4B40F21D
S3150802AA40EE22DA60084B40F2EE229A60064B0022AA
S3150802AA501A61054813F081F80346002B01D000F06D
S3150802AA60BBFB00BF80BD00BF1005012000300040BF
S3150802AA7080B400AF00BFBD465DF8047B7047000096
S3150802AA8080B59CB000AF07F1600300221A605A60D5
S3150802AA909A60DA6007F1540300221A605A609A60D3
S3150802AAA007F1380300221A605A609A60DA601A615E
S3150802AAB05A619A613B1D3422002118462BF04EFB3F
S3150802AAC04B4B4C4A1A604A4B46F2A7125A60484BFD
S3150802AAD000229A60464B6322DA60454B00221A61CD
S3150802AAE0434B00225A61424B00229A61404819F0B0
S3150802AAF0D1F80346002B01D000F06EFB4FF48053C9
S3150802AB003B6607F160031946394819F0A1FE034668
S3150802AB10002B01D000F060FB354819F0C1F9034655
S3150802AB20002B01D000F058FB00237B650023BB6590
S3150802AB300023FB6507F1540319462D481AF084FDD4
S3150802AB400346002B01D000F047FB6023BB630023BA
S3150802AB50FB6300233B6400237B640023BB6400235E
S3150802AB60FB6400233B6507F138030822194620488F
S3150802AB7019F05AFD0346002B01D000F02DFB07F110
S3150802AB8038030C2219461A4819F04EFD0346002BC3
S3150802AB9001D000F021FB00237B600023BB60002369
S3150802ABA0FB6000233B6100237B614FF40053BB61CA
S3150802ABB00023FB6100233B6200237B624FF0007394
S3150802ABC0BB620023FB6200233B6300237B633B1DBE
S3150802ABD0194607481AF008FE0346002B01D000F072
S3150802ABE0FBFA034809F0C4FC00BF7037BD4680BDB6
S3150802ABF024050120002C014080B58EB000AF07F174
S3150802AC00280300221A605A609A60DA6007F11C0368
S3150802AC1000221A605A609A603B4600221A605A60FD
S3150802AC209A60DA601A615A619A61334B4FF0804230
S3150802AC301A60314B46F2A7125A602F4B00229A60CD
S3150802AC402D4B6322DA602C4B00221A612A4B002212
S3150802AC509A61294819F01EF80346002B01D000F024
S3150802AC60BBFA4FF48053BB6207F128031946224800
S3150802AC7019F0EEFD0346002B01D000F0ADFA1E488E
S3150802AC8019F00EF90346002B01D000F0A5FA0023AD
S3150802AC90FB6100237B6207F11C03194616481AF06A
S3150802ACA0D3FC0346002B01D000F096FA60233B60E2
S3150802ACB000237B600023BB6000233B613B460422E2
S3150802ACC019460D4819F0B0FC0346002B01D000F0D6
S3150802ACD083FA3B4608221946074819F0A5FC03469B
S3150802ACE0002B01D000F078FA034809F041FC00BFB6
S3150802ACF03837BD4680BD00BF7005012080B58EB0CD
S3150802AD0000AF07F1280300221A605A609A60DA60D7
S3150802AD1007F11C0300221A605A609A603B46002219
S3150802AD201A605A609A60DA601A615A619A613D4BF2
S3150802AD303D4A1A603B4B46F2A7125A60394B00222B
S3150802AD409A60384B6322DA60364B00221A61354B19
S3150802AD5000229A61334818F09DFF0346002B01D062
S3150802AD6000F03AFA4FF48053BB6207F128031946FA
S3150802AD702C4819F06DFD0346002B01D000F02CFA81
S3150802AD80284819F08DF80346002B01D000F024FA62
S3150802AD900023FB6100237B6207F11C031946214845
S3150802ADA01AF052FC0346002B01D000F015FA602374
S3150802ADB03B6000237B600023BB6000233B613B466C
S3150802ADC000221946174819F02FFC0346002B01D01A
S3150802ADD000F002FA3B4604221946124819F024FCEE
S3150802ADE00346002B01D000F0F7F93B460822194624
S3150802ADF00C4819F019FC0346002B01D000F0ECF9B7
S3150802AE003B460C221946074819F00EFC0346002B4E
S3150802AE1001D000F0E1F9034809F0AAFB00BF383770
S3150802AE20BD4680BDBC0501200004004080B500AFC8
S3150802AE300F4B104A1A600E4B40F6C3125A600C4B5F
S3150802AE4000229A600A4B6322DA60094B00221A61D1
S3150802AE50074B00225A61064B00229A61044818F0F1
S3150802AE6019FF0346002B01D000F0B6F900BF80BDDA
S3150802AE70080601200048014080B500AF224B234A4C
S3150802AE801A60214B4FF4E1325A601F4B00229A6036
S3150802AE901D4B0022DA601C4B00221A611A4B0C2247
S3150802AEA05A61194B00229A61174B0022DA61164B36
S3150802AEB000221A62144B00225A62134B00229A622B
S3150802AEC011481AF099FD0346002B01D000F084F9C7
S3150802AED000210D481CF009FE0346002B01D000F0A4
S3150802AEE07BF9002108481CF03EFE0346002B01D0E0
S3150802AEF000F072F904481CF0BFFD0346002B01D08E
S3150802AF0000F06AF900BF80BD5406012000380140EE
S3150802AF1080B58EB000AF07F1240300221A605A608A
S3150802AF209A60DA601A61964BD3F88C30944A43F0E9
S3150802AF301003C2F88C30924BD3F88C3003F010030E
S3150802AF403B623B6A8E4BD3F88C308D4A43F0200322
S3150802AF50C2F88C308A4BD3F88C3003F02003FB619D
S3150802AF60FB69874BD3F88C30854A43F08003C2F8D5
S3150802AF708C30834BD3F88C3003F08003BB61BB69FA
S3150802AF807F4BD3F88C307E4A43F00403C2F88C30E8
S3150802AF907B4BD3F88C3003F004037B617B69784BD7
S3150802AFA0D3F88C30764A43F00103C2F88C30744BDE
S3150802AFB0D3F88C3003F001033B613B69704BD3F83D
S3150802AFC08C306F4A43F00203C2F88C306C4BD3F8CC
S3150802AFD08C3003F00203FB60FB68694BD3F88C30B4
S3150802AFE0674A43F00803C2F88C30654BD3F88C30B5
S3150802AFF003F00803BB60BB68614BD3F88C30604A28
S3150802B00043F04003C2F88C305D4BD3F88C3003F022
S3150802B01040037B607B6800224FF40041594812F0D6
S3150802B02053FD00224FF48061574812F04DFD00226D
S3150802B0300121564812F048FD41F27C037B62002347
S3150802B040BB620023FB6207F1240319464F4812F03C
S3150802B05015FB0F237B620023BB620023FB6207F109
S3150802B060240319464A4812F009FB02237B62494B1C
S3150802B070BB620023FB6207F124031946464812F015
S3150802B080FDFA24237B620023BB620023FB6207F1DD
S3150802B09024031946404812F0F1FA21237B62002361
S3150802B0A0BB620023FB6207F1240319463B4812F0F0
S3150802B0B0E5FA4FF400437B620123BB620023FB627D
S3150802B0C000233B6307F1240319462E4812F0D6FAE9
S3150802B0D041F602737B620023BB620023FB6207F11F
S3150802B0E0240319462E4812F0C9FA01237B62294B1A
S3150802B0F0BB620023FB6207F124031946284812F0B3
S3150802B100BDFA4FF480637B620123BB620023FB62B4
S3150802B11000233B6307F1240319461B4812F0AEFAD3
S3150802B1204FF400437B620023BB620023FB6207F1F4
S3150802B13024031946144812F0A1FA01237B6201235B
S3150802B140BB620023FB6200233B6307F12403194613
S3150802B1500E4812F093FA002200210B2010F0AAFFE3
S3150802B1600B2010F0C1FF002200210C2010F0A2FFD4
S3150802B1700C2010F0B9FF00BF3837BD4680BD00BFAE
S3150802B180000C024400040242001802420010024265
S3150802B1900014024200002110000802420000024286
S3150802B1A0000C024280B582B000AF78607B681B68EB
S3150802B1B0074A934201D110F081FE7B681B68054A53
S3150802B1C0934201D1FDF7ACFD00BF0837BD4680BDED
S3150802B1D0001000400048014080B400AF72B600BFBC
S3150802B1E000BFFDE7B0B596B000AF786039600023BE
S3150802B1F07B6576E0774B784A4021786811F0B2FA97
S3150802B2000346002B03D0754810F058FC69E0FAF79C
S3150802B21077FA0346002B03D06F4B1B687B6502E067
S3150802B2206D4B1B687B65FAF785FA02467B6D93427E
S3150802B23004D168216848FAF729F952E022F0BCF9E4
S3150802B24002467B6D934241D022F00FFA02467B6D8D
S3150802B25093423BD022F050FA02467B6D934235D098
S3150802B26022F066FA02467B6D93422FD022F0CEF97F
S3150802B27002467B6D934229D022F0BAF902467B6DCB
S3150802B280934223D022F0A6F902467B6D93421DD043
S3150802B29022F0C6F902467B6D934217D022F052FA83
S3150802B2A002467B6D934211D022F00AFA02467B6D62
S3150802B2B093420BD022F054FA02467B6D934205D094
S3150802B2C022F0F0F902467B6D93420AD1424BDB68C3
S3150802B2D01846F9F77DFB03461A463E49786D29F06A
S3150802B2E0A5F94021786811F0ABFB0346002B81D102
S3150802B2F07868FAF75FF903461A46394B9A6078680E
S3150802B300FAF722F90346364A13607868FAF734F9E7
S3150802B3100346334A5360324B9B68002B12D0304B9C
S3150802B3201A682F4B5B6807F10C002E492AF082FE39
S3150802B33007F10C03184610F0C1FB294B9B68184607
S3150802B340FAF780F90C22264927482AF0F7FE03461F
S3150802B350002B36D0224B1B68DAB207F1500311468E
S3150802B360184621F022FC1E4B5B68DAB207F150033D
S3150802B3701146184621F034FC194B9B68DAB207F1DC
S3150802B38050031146184621F046FC07F10C0207F154
S3150802B39050031146184621F08CFF22F059F904464B
S3150802B3A007F10C03184621F01AFD054607F10C03AE
S3150802B3B0184621F020FD03461A462946204629F05A
S3150802B3C033FA094B064A07CA83E8070000BF58370B
S3150802B3D0BD46B0BD10070120E806012004D30508C2
S3150802B3E0E0B5002024D30508ECB5002080B58AB064
S3150802B3F002AF78600B467B8013463B800023BB6016
S3150802B4000023FB607B683B6101237B617B88BB6110
S3150802B4103B88FB6107F108031946074811F080F8D3
S3150802B42001230093012302220221034811F0D2F8D4
S3150802B43000BF2037BD4680BDAC04012080B58CB064
S3150802B44002AFF860B9607A604FF080433B6100232F
S3150802B4507B61FB68BB610123FB61BB683B627B685E
S3150802B4607B6207F110031946074811F059F80123C0
S3150802B4700093012302220221034811F0ABF800BF10
S3150802B4802837BD4680BD00BFAC04012080B500AF99
S3150802B490044811F0D0F800220121024811F0EEFA10
S3150802B4A000BF80BDAC04012080B500AFFAF728F9C9
S3150802B4B00346002B09D0FAF73DF903461A466FF000
S3150802B4C060410220FFF7BAFF09E0FAF733F90346AB
S3150802B4D09BB21A464FF6FF710220FFF787FFFFF766
S3150802B4E0D5FF00BF80BD000080B58EB000AFF86002
S3150802B4F0B9601346FB71FB79002B02D0FB79402B0E
S3150802B50001D900233FE007F114032422002118463B
S3150802B5102AF024FEFB687B61FAF7F2F80346002B51
S3150802B52003D04FF08043BB6101E00023BB610023D7
S3150802B530FB61FB799BB21846F9F7A0FA03463B6210
S3150802B54000237B624FF48013BB624FF40013FB6245
S3150802B55000233B6300237B634FF47A710C481EF089
S3150802B56061FD0346002B0AD107F11403BA6819468E
S3150802B5700848F9F7E5FB06481EF0AEFD02E0064864
S3150802B58010F09CFA012318463837BD4680BD00BF25
S3150802B59098910020AC04012048D3050880B483B0F2
S3150802B5A000AF78607B689B7818460C37BD465DF815
S3150802B5B0047B704780B483B000AF78600B46FB709B
S3150802B5C01346BB70BB78132B01D900230AE0FA781D
S3150802B5D0BB78796840F2BC4000FB02F20A44134485
S3150802B5E005331B7818460C37BD465DF8047B704751
S3150802B5F080B483B000AF78600B46FB70FB787A683C
S3150802B60040F2BC4101FB03F313440F331B7818467F
S3150802B6100C37BD465DF8047B7047000090B583B0D1
S3150802B62000AF78600B46FB70FC78FB7819467868A1
S3150802B630FFF7DEFF03461A4621460E4810F03EFA89
S3150802B640FB78796840F2BC4203FB02F20A440F32E5
S3150802B6501278511CCCB2796840F2BC4000FB03F365
S3150802B6600B440F3321461970134618460C37BD464C
S3150802B67090BD00BF68D3050880B483B000AF786078
S3150802B680084611461A460346FB700B46BB7013461C
S3150802B6907B70F978B8787A7813469B0013445B0076
S3150802B6A0322200FB02F21A4440F2BC4301FB03F3C6
S3150802B6B0134408337A681344083318460C37BD46D0
S3150802B6C05DF8047B704780B483B000AF78600B46A0
S3150802B6D0FB701346BB70FA78BB78796840F2BC40B7
S3150802B6E000FB02F20A44134403F57E731B781846DC
S3150802B6F00C37BD465DF8047B7047B0B483B000AF23
S3150802B70078600B46FB701346BB70FA78BB7878688C
S3150802B71040F2BC4102FB01F10144194401F57E7174
S3150802B7200978481CC5B2786840F2BC4404FB02F2A8
S3150802B7300244134403F57E732A461A700B461846CA
S3150802B7400C37BD46B0BC704780B483B000AF786092
S3150802B750084611461A460346FB700B46BB7013464B
S3150802B7607B70F878B9787B781A4652001A445300E7
S3150802B7701A460B461B015B1A5B001A4440F2BC438D
S3150802B78000FB03F3134403F584637A681344043312
S3150802B79018460C37BD465DF8047B704780B483B003
S3150802B7A000AF78600B46FB701346BB70FA78BB781D
S3150802B7B0796840F2BC4000FB02F20A44134403F2E1
S3150802B7C0BA431B7818460C37BD465DF8047B7047AA
S3150802B7D0B0B483B000AF78600B46FB701346BB70FB
S3150802B7E0FA78BB78786840F2BC4102FB01F1014461
S3150802B7F0194401F2BA410978481CC5B2786840F280
S3150802B800BC4404FB02F20244134403F2BA432A4636
S3150802B8101A700B4618460C37BD46B0BC704780B541
S3150802B82084B000AF0346FB800023FB730023BB8171
S3150802B8300023FB7314E026F09FFF0346184626F002
S3150802B840C1FF0246FB7B1946104620F0E3FF03467A
S3150802B850BB81BA89FB889A4206D0FB7B0133FB730C
S3150802B860FB7B072BE7D900E000BFFB7B18461037A6
S3150802B870BD4680BD80B485B000AF03460A46FB715B
S3150802B8801346BB710023FB73FA79BB79D31ADBB271
S3150802B890FB7397F90F30002B03DCFB7B0833DBB213
S3150802B8A0FB73FB7B18461437BD465DF8047B70476D
S3150802B8B080B485B000AF03460A46FB711346BB71D6
S3150802B8C00023FB73FA79BB791344DBB2FB7397F94E
S3150802B8D00F30082B03DDFB7B083BDBB2FB73FB7BDC
S3150802B8E018461437BD465DF8047B7047B0B598B064
S3150802B8F000AF07F1080383E803001346FB7143F61A
S3150802B9009823FB6543F69823BB650023A7F85630B0
S3150802B9104EF66023FB6592E05C4B1B78022B03D044
S3150802B9205A4B1B78002B75D126F026FF034618467C
S3150802B93027F0D5F80346184624F0D6F80346A7F8A2
S3150802B9405630B7F85630002B64D1504B00221A7085
S3150802B9500AF03AFA034618460AF066FD0346DBB2CF
S3150802B960BB7207F1140207F108031146184624F0C0
S3150802B9700CFA21F003FF044607F11403184621F0D6
S3150802B9802EFA054607F11403184621F034FA03463F
S3150802B9901A462946204628F047FF40F6B833BB65C3
S3150802B9A00DE03A4B1B78002B0DD1FB79184610F0A7
S3150802B9B09FF964201DF0EEFBBB6D643BBB65BB6D56
S3150802B9C0002BEED100E000BFBB6D002B1AD1304927
S3150802B9D002200AF0A1FF24F099FC012365226621C0
S3150802B9E024F010FD0AF0F0F90346662118460AF01B
S3150802B9F06DFE0AF0E9F90346652118460AF084FE47
S3150802BA0002233FE0214B1B78022B03D12149022056
S3150802BA100AF082FF1D4B1B78012B04D11E49022016
S3150802BA200AF07AFF0FE0FB79184610F061F94FF435
S3150802BA307A701DF0AFFBFB6DA3F57A73FB65FB6DA0
S3150802BA40002B7FF469AFFB6D002B1AD11349022034
S3150802BA500AF062FF24F05AFC01236722662124F0C9
S3150802BA60D1FC0AF0B1F90346662118460AF02EFE01
S3150802BA700AF0AAF90346672118460AF045FE022388
S3150802BA8000E0002318466037BD46B0BDB006022066
S3150802BA9098D30508B8D30508D8D30508F4D30508FA
S3150802BAA080B582B000AF0023FB710023BB7100236F
S3150802BAB0BB8002F003FC0346184602F001FE034669
S3150802BAC0BB71BB79062B02D10023FB7123E026F05A
S3150802BAD053FE0346184626F075FE0246BB79013B1D
S3150802BAE0DBB21946104620F095FE0346BB80BB889A
S3150802BAF0002B08D1BB791A46094902200AF00CFF25
S3150802BB000123FB7107E0BB791A46064902200AF0AF
S3150802BB1003FF0023FB71FB7918460837BD4680BD33
S3150802BB2010D4050824D40508F0B5AFB004AF03460F
S3150802BB303960FB71002387F8A7300023A7F8A430E1
S3150802BB40002387F89E304FF00003C7F89830002389
S3150802BB5087F89730002387F8963044F62063C7F8AB
S3150802BB60A03002F0ABFB0346184602F0A9FD0346D5
S3150802BB7087F8973097F89730002B00F0AF8097F840
S3150802BB809730082B00F2AA8097F89730062B04D133
S3150802BB904FF6FF73A7F8A43011E026F0EDFD034631
S3150802BBA0184626F00FFE024697F89730013BDBB29D
S3150802BBB01946104620F02EFE0346A7F8A430B7F819
S3150802BBC0A430002B0DD197F89730013BDAB23B68C7
S3150802BBD01A7097F897301A46C84902200AF09CFE4E
S3150802BBE07CE0012387F8A73074E097F8A72097F836
S3150802BBF0973011461846FFF73DFE034687F89630FA
S3150802BC0097F89630062B04D14FF6FF73A7F8A4309F
S3150802BC1011E026F0B1FD0346184626F0D3FD02468A
S3150802BC2097F89630013BDBB21946104620F0F2FD32
S3150802BC300346A7F8A430B7F8A430002B0DD197F81D
S3150802BC409630013BDAB23B681A7097F896301A4674
S3150802BC50AA4902200AF060FE40E097F8A72097F862
S3150802BC60973011461846FFF723FE034687F89630A3
S3150802BC7097F89630062B04D14FF6FF73A7F8A4302F
S3150802BC8011E026F079FD0346184626F09BFD02468A
S3150802BC9097F89630013BDBB21946104620F0BAFDFA
S3150802BCA00346A7F8A430B7F8A430002B0DD197F8AD
S3150802BCB09630013BDAB23B681A7097F896301A4604
S3150802BCC08E4902200AF028FE08E097F8A7300133C9
S3150802BCD087F8A73097F8A730042B86D9FB79184638
S3150802BCE010F006F83B681B7801331A46844902208D
S3150802BCF00AF012FE002387F89F303B681B78C3F1CF
S3150802BD000303DBB287F89F3097F99F30002B05DCD7
S3150802BD1097F89F300833DBB287F89F3007F10C0398
S3150802BD200121184620F0A9FD97F89F2007F10C0378
S3150802BD301146184620F0BCFD07F10C0300211846EF
S3150802BD4020F0D1FD07F1100207F10C03114618463F
S3150802BD5021F014F907F11003184621F040F80446B9
S3150802BD6007F11003184621F046F8034619462046FD
S3150802BD70F9F766FFFB7918460FF0BAFF1AE026F0C4
S3150802BD80FBFC0346184626F07CFD03461A4697F93D
S3150802BD909F300A339A4212D0FB7918460FF0A8FF51
S3150802BDA04FF47A701DF0F6F9D7F8A030A3F57A7336
S3150802BDB0C7F8A030D7F8A030002BE0D100E000BFCA
S3150802BDC0D7F8A030002B2BD14E4902200AF0A4FD49
S3150802BDD024F09CFA3B681B781A46920013449B008F
S3150802BDE0DBB20333DAB20123372124F00BFB09F065
S3150802BDF0EBFF0346372118460AF068FC09F0E4FF10
S3150802BE0002463B681B78194689000B449B00DBB245
S3150802BE100333DBB2194610460AF076FC0123AAE080
S3150802BE203B681B785E1C09F0CFFF02463B681B780D
S3150802BE300133DBB2194610460AF090F810EE103AB2
S3150802BE401846F4F7AFFC04460D4609F0BDFF024654
S3150802BE503B681B780133DBB2194610460AF0D6F85E
S3150802BE6003460293CDE900453246274902200AF0E5
S3150802BE7053FD3B681B780133DBB23B7207F1540270
S3150802BE8007F108031146184620F0EBFB21F08AFB5E
S3150802BE90044607F15403184620F088F9054607F1C7
S3150802BEA05403184620F08EF903461A4629462046B8
S3150802BEB028F0BAFC4FF416701DF06CF909F084FFED
S3150802BEC002463B681B780133DBB2194610460AF074
S3150802BED045F887ED260AD7ED267AB7EE007AF4EE0C
S3150802BEE0C77AF1EE10FA13D53B681B7801331A4666
S3150802BEF0064902200AF010FD12E000BF10D4050818
S3150802BF003CD4050868D4050890D40508B0D40508B9
S3150802BF103B681B7801331A46194902200AF0FCFCD1
S3150802BF203B681B785E1C09F04FFF02463B681B788C
S3150802BF300133DBB2194610460AF010F810EE103A31
S3150802BF401846F4F72FFC04460D4609F03DFF024653
S3150802BF503B681B780133DBB2194610460AF056F8DD
S3150802BF6003460293CDE900453246064902200AF005
S3150802BF70D3FC97F89E301846AC37BD46F0BD00BFD5
S3150802BF80C4D40508D4D405082DE9F043A3B006AFF6
S3150802BF900446084611461A462346FB8103467B7326
S3150802BFA00B463B731346FB72FF2387F86230002366
S3150802BFB087F86F3026F0E0FB0346184626F083FD25
S3150802BFC0786643F69823BB66002387F863303B7B83
S3150802BFD00C2B7BD107F158030422002118462AF0BC
S3150802BFE0BDF809F0F1FE034618460AF04BFA034675
S3150802BFF01A4607F158031146184621F039FFFA89FD
S3150802C00007F158031146184621F04DFF07F11402AD
S3150802C01007F158031146184622F000FB21F0ABFA45
S3150802C020044607F11403184621F04CFF054607F1AA
S3150802C0301403184621F052FF03461A46294620469B
S3150802C04028F0F2FB0023BB66786E21F088FD0346D2
S3150802C0501A46FB89934217D1786E21F09BFD034657
S3150802C060FE2B11D1FC89786E21F079FD03461D4617
S3150802C070786E21F08FFD034600932B462246C5496A
S3150802C08002200AF049FC21E0BB6E0133BB66BB6E97
S3150802C090B3F5966F12D3FC89786E21F060FD0346DC
S3150802C0A01D46786E21F076FD034600932B462246FE
S3150802C0B0B94902200AF030FC022314E2FB7A184638
S3150802C0C00FF016FE64201DF065F8BDE707F162025F
S3150802C0D0FB7A11461846FFF727FD034687F86330B1
S3150802C0E097F86330002B01D00123FCE13B7B0E2B32
S3150802C0F062D1AA4902200AF00FFC002387F86F30A2
S3150802C1001FE026F039FB0346184626F0D0FC024605
S3150802C11097F86F301946104623F010FF03461A4661
S3150802C120FB89934208D197F86F3001331A469C4926
S3150802C13002200AF0F1FB08E097F86F30013387F81E
S3150802C1406F3097F86F30022BDBD997F86F30022BD6
S3150802C1501AD9944902200AF0DFFB24F0D7F8012302
S3150802C1600122382124F04EF909F02EFE0346382121
S3150802C17018460AF0ABFA09F027FE034601211846CB
S3150802C1800AF0C2FA0223AEE197F86F300133032BA5
S3150802C1900ED0032B36DC012B02D0022B04D031E061
S3150802C1A0042387F85F302DE0032387F85F3029E000
S3150802C1B0022387F85F3025E03B7B0C2B07D17A49AF
S3150802C1C002200AF0A9FB052387F85F301AE07749AF
S3150802C1D002200AF0A1FB24F099F801230222382151
S3150802C1E024F010F909F0F0FD0346382118460AF042
S3150802C1F06DFA09F0E9FD0346022118460AF084FAA7
S3150802C200012370E1FB891A46694902200AF084FB78
S3150802C210684B00221A70062387F86030FB89A7F854
S3150802C2205C3026F0A9FA0346184626F0CBFA0346EE
S3150802C230C821184620F0C4FAFB7A1A4607F15C03AD
S3150802C24093E80300FFF752FB034687F8633097F833
S3150802C2506330002B02D097F8633044E1564B002234
S3150802C2601A704AF6C873BB6631E0534B1B78002B2B
S3150802C27023D0514B1B78022B04D1504902200AF0D5
S3150802C2804BFB27E04E4902200AF046FB24F03EF813
S3150802C29001236822662124F0B5F809F095FD0346C4
S3150802C2A0662118460AF012FA09F08EFD034668213D
S3150802C2B018460AF029FA022315E1FB7A18460FF006
S3150802C2C017FD64201CF066FFBB6E643BBB66BB6E43
S3150802C2D0002BCAD1BB6E002B1AD13A4902200AF0AA
S3150802C2E01BFB24F013F801236622662124F08AF840
S3150802C2F009F06AFD0346662118460AF0E7F909F0CD
S3150802C30063FD0346662118460AF0FEF90223EAE0AF
S3150802C31097F862305E1C09F057FD024697F86230BC
S3150802C3200133DBB21946104609F018FE10EE103A30
S3150802C3301846F4F737FA04460D4609F045FD024653
S3150802C34097F862300133DBB21946104609F05EFEF1
S3150802C35003460293CDE9004532461B4902200AF0FC
S3150802C360DBFA26F009FA0346184626F02BFA97F85E
S3150802C3706220FB89194620F05FFA09F025FD02467C
S3150802C380FB89194610460AF0D1F9002387F86F305F
S3150802C3902EE000BFF4D4050830D5050868D505088F
S3150802C3A07CD5050894D50508B8D50508C8D5050865
S3150802C3B0E8D50508B00602209C06022008D605081C
S3150802C3C020D6050838D6050854D6050826F0D4F925
S3150802C3D00346184626F0F6F9024697F86F301946CC
S3150802C3E0104620F017FA97F86F30013387F86F3046
S3150802C3F097F86F30072BE9D926F0BEF90346184697
S3150802C40026F0E0F903460021184620F003FA03460F
S3150802C410984626F0B1F90346184626F0D3F903469C
S3150802C4200121184620F0F6F90346994626F0A4F9A2
S3150802C4300346184626F0C6F903460221184620F096
S3150802C440E9F903461C4626F097F90346184626F0EC
S3150802C450B9F903460321184620F0DCF903461D46BE
S3150802C46026F08AF90346184626F0ACF90346042153
S3150802C470184620F0CFF903461E4626F07DF90346F4
S3150802C480184626F09FF903460521184620F0C2F9F8
S3150802C49003467B6026F070F90346184626F092F9A1
S3150802C4A003460621184620F0B5F903463B6026F0F6
S3150802C4B063F90346184626F085F903460721184606
S3150802C4C020F0A8F9034605933A6804927B68039319
S3150802C4D00296019500944B464246054902200AF007
S3150802C4E01BFA97F8633018467437BD46BDE8F083E1
S3150802C4F06CD605082DE9F043B7B006AF04460846E0
S3150802C50011461A462346FB8103467B730B463B7349
S3150802C5101346FB72FF2387F8B730002387F8BF302C
S3150802C52026F02AF90346184626F0CDFAC7F8B000CF
S3150802C53043F69823C7F8B830002387F8AF304FF090
S3150802C5400003C7F8A830FFF7ABFA0346002B01D160
S3150802C5500023FDE201F0B2FE0346184602F0B0F8E7
S3150802C560034687F8B7303B7B0C2B40F0868007F1F1
S3150802C5709C0304220021184629F0F0FD09F024FC48
S3150802C5800346184609F07EFF03461A4607F19C033E
S3150802C5901146184621F06CFCFA8907F19C031146EC
S3150802C5A0184621F080FC07F1580207F19C03114650
S3150802C5B0184622F033F820F0DEFF044607F1580346
S3150802C5C0184621F07FFC054607F15803184621F064
S3150802C5D085FC03461A462946204628F025F90023F3
S3150802C5E0C7F8B830D7F8B00021F0B9FA03461A46A8
S3150802C5F0FB8993421AD1D7F8B00021F0CBFA034649
S3150802C600FE2B13D1FC89D7F8B00021F0A8FA03460D
S3150802C6101D46D7F8B00021F0BDFA034600932B4613
S3150802C6202246BF4902200AF077F926E0D7F8B83041
S3150802C6300133C7F8B830D7F8B830B3F5966F14D3C4
S3150802C640FC89D7F8B00021F08AFA03461D46D7F8C6
S3150802C650B00021F09FFA034600932B462246B149C1
S3150802C66002200AF059F9022372E2FB7A18460FF001
S3150802C6703FFB64201CF08EFDB4E73B7B0E2B62D198
S3150802C680A94902200AF048F9002387F8BF301FE0BB
S3150802C69026F072F80346184626F009FA024697F873
S3150802C6A0BF301946104623F049FC03461A46FB8951
S3150802C6B0934208D197F8BF3001331A469B490220A4
S3150802C6C00AF02AF908E097F8BF30013387F8BF3035
S3150802C6D097F8BF30022BDBD997F8BF30022B1AD94D
S3150802C6E0934902200AF018F923F010FE01230122C9
S3150802C6F0382123F087FE09F067FB034638211846DE
S3150802C70009F0E4FF09F060FB03460121184609F027
S3150802C710FBFF02231CE297F8BF300133032B0ED02E
S3150802C720032B36DC012B02D0022B04D031E0042382
S3150802C73087F8A3302DE0032387F8A33029E00223E4
S3150802C74087F8A33025E03B7B0C2B07D179490220D9
S3150802C7500AF0E2F8052387F8A3301AE076490220A0
S3150802C7600AF0DAF823F0D2FD01230222382123F057
S3150802C77049FE09F029FB03463821184609F0A6FFA7
S3150802C78009F022FB03460221184609F0BDFF0123E0
S3150802C790DEE197F8B7303B7407F1140207F110038C
S3150802C7A0114618461FF05DFF20F0FCFE044607F10D
S3150802C7B0140318461FF0FAFC054607F11403184637
S3150802C7C01FF000FD03461A462946204628F02CF893
S3150802C7D04FF416701CF0DEFC09F0F6FA024697F8DA
S3150802C7E0B7301946104609F0B9FB87ED2A0AD7ED84
S3150802C7F02A7AB7EE007AF4EEC77AF1EE10FA07D57E
S3150802C80097F8B7301A464D4902200AF085F806E02D
S3150802C81097F8B7301A464A4902200AF07DF897F87F
S3150802C820B76009F0D1FA024697F8B73019461046AA
S3150802C83009F094FB10EE103A1846F3F7B3FF0446D4
S3150802C8400D4609F0C1FA024697F8B730194610465E
S3150802C85009F0DCFB03460293CDE900453246394925
S3150802C86002200AF059F8FB891A46374902200AF0CB
S3150802C87053F8364B00221A70062387F8A430FB8930
S3150802C880A7F8A03025F078FF0346184625F09AFF48
S3150802C8900346C82118461FF093FFFB7A1A4607F18A
S3150802C8A0A00393E80300FFF721F8034687F8AF30A1
S3150802C8B097F8AF30002B02D097F8AF3048E1244BF7
S3150802C8C000221A704AF6C873C7F8B83052E0204BED
S3150802C8D01B78002B42D01E4B1B78022B04D11D4914
S3150802C8E002200AF019F849E01B4902200AF014F856
S3150802C8F023F00CFD01236822662123F083FD09F04B
S3150802C90063FA03466621184609F0E0FE09F05CFA66
S3150802C91003466821184609F0F7FE022318E100BF0C
S3150802C920F4D4050830D5050868D505087CD5050868
S3150802C93094D50508B8D50508C8D50508B0D405089C
S3150802C940C4D40508D4D40508E8D50508B0060220DB
S3150802C9509C06022008D6050820D60508FB7A184642
S3150802C9600FF0C6F964201CF015FCD7F8B830643B02
S3150802C970C7F8B830D7F8B830002BA8D1D7F8B830EE
S3150802C980002B1AD17549022009F0C6FF23F0BEFC16
S3150802C99001236622662123F035FD09F015FA0346BE
S3150802C9A06621184609F092FE09F00EFA0346662138
S3150802C9B0184609F0A9FE0223CAE097F8B76009F0FB
S3150802C9C003FA024697F8B7301946104609F0C6FA2E
S3150802C9D010EE103A1846F3F7E5FE04460D4609F03E
S3150802C9E0F3F9024697F8B7301946104609F00EFBD6
S3150802C9F003460293CDE9004532465949022009F019
S3150802CA008BFF25F0B9FE0346184625F0DBFE97F89C
S3150802CA10B730013BDAB2FB8919461FF00DFF09F060
S3150802CA20D3F90246FB891946104609F07FFE002310
S3150802CA3087F8BF3011E025F09FFE0346184625F019
S3150802CA40C1FE024697F8BF30194610461FF0E2FEAD
S3150802CA5097F8BF30013387F8BF3097F8BF30072BF6
S3150802CA60E9D925F089FE0346184625F0ABFE0346AA
S3150802CA70002118461FF0CEFE0346984625F07CFE96
S3150802CA800346184625F09EFE0346012118461FF066
S3150802CA90C1FE0346994625F06FFE0346184625F061
S3150802CAA091FE0346022118461FF0B4FE03461C46B1
S3150802CAB025F062FE0346184625F084FE0346032146
S3150802CAC018461FF0A7FE03461D4625F055FE0346E7
S3150802CAD0184625F077FE0346042118461FF09AFEEB
S3150802CAE003461E4625F048FE0346184625F06AFE0A
S3150802CAF00346052118461FF08DFE03467B6025F086
S3150802CB003BFE0346184625F05DFE034606211846F7
S3150802CB101FF080FE03463B6025F02EFE03461846AC
S3150802CB2025F050FE0346072118461FF073FE0346FA
S3150802CB3005933A6804927B680393029601950094DA
S3150802CB404B4642460749022009F0E6FE97F8AF30FF
S3150802CB501846C437BD46BDE8F08300BF38D6050877
S3150802CB6054D605086CD6050880B500AF0D4B1B7860
S3150802CB70DBB2002B12D10B4B01221A704FF46D4215
S3150802CB800021094829F0EAFA1422084908481EF041
S3150802CB90D9FD2822074908481EF0D4FD024B18463B
S3150802CBA080BD00BFACF40120AC070120600701205C
S3150802CBB050070120840701207407012080B483B03E
S3150802CBC000AF78600B46FB70FB7841F2B07202FB4D
S3150802CBD003F37A68134418460C37BD465DF8047B9E
S3150802CBE0704780B584B000AF78600B467B8000231F
S3150802CBF0FB730023BB7300237B730023FB7312E0D2
S3150802CC00FB7B19467868FFF7D9FFB860BB681B88B3
S3150802CC107A889A4204D10123BB73FB7B7B7305E0B6
S3150802CC20FB7B0133FB73FB7B092BE9D9BB7B002B0F
S3150802CC3007D07B7B41F2B07202FB03F37A68134496
S3150802CC4000E0002318461037BD4680BD80B582B085
S3150802CC5000AF78600B46FB70FB78092B0CD8FB7883
S3150802CC6019467868FFF7AAFF034641F2B072002117
S3150802CC70184629F073FA00E000BF0837BD4680BDA2
S3150802CC8080B584B000AF78600B467B800023FB73C7
S3150802CC900023BB7300237B730023FB7312E0FB7B29
S3150802CCA019467868FFF78AFFB860BB681B887A88D6
S3150802CCB09A4204D10123BB73FB7B7B7305E0FB7BA2
S3150802CCC00133FB73FB7B092BE9D9BB7B002B0BD00A
S3150802CCD07B7B19467868FFF771FFB86041F2B0723C
S3150802CCE00021B86829F03AFA00BF1037BD4680BD60
S3150802CCF080B483B000AF78607B6803F56043B3F80D
S3150802CD00E03C18460C37BD465DF8047B704780B494
S3150802CD1083B000AF78600B46FB70FB787A6803F540
S3150802CD20EC43703332F8133018460C37BD465DF8BB
S3150802CD30047B704780B588B002AF78600B467B806B
S3150802CD4013467B700023FB750023BB7500237B7596
S3150802CD500023BB7400233B750023FB740023FB7579
S3150802CD602EE0FB7D19467868FFF728FFF860FB6816
S3150802CD701B887A889A4201D101237B75FB7D194665
S3150802CD807868FFF7C4FF03461A467B88934202D1A6
S3150802CD900123BB7517E0FB7D19467868FFF7B7FFD5
S3150802CDA00346002B09D1BB7C002B06D1FB7C002B4A
S3150802CDB003D1FB7D3B750123FB74FB7D0133FB75B8
S3150802CDC0FB7D092BCDD9BB7D012B02D07B7D002BA8
S3150802CDD009D17A88B97D7B7D00930B460E490220DC
S3150802CDE009F09AFD14E03B7D7A6803F5EC4370334B
S3150802CDF0798822F813107B88194608480EF05EFED9
S3150802CE003B7D7A68134403F56C43F6337A781A70D5
S3150802CE101837BD4680BD00BFA4D6050800D7050849
S3150802CE2080B483B000AF78607B6803F56043B3F8DB
S3150802CE30F43C18460C37BD465DF8047B704780B44F
S3150802CE4083B000AF78607B6803F560430022A3F8DD
S3150802CE50F42C00BF0C37BD465DF8047B704780B5DD
S3150802CE6084B000AF78600023FB817868FFF740FF43
S3150802CE700346FB817B6803F560431A46FB89A2F8E1
S3150802CE80F43C00BF1037BD4680BD000090B58FB098
S3150802CE9002AF78600B467B80002387F82F30002389
S3150802CEA087F82E3007F1180300221A605A609A6032
S3150802CEB0DA601A610023FB6007F1100300221A6088
S3150802CEC09A807B6803F56C43E03307F11800142255
S3150802CED0194629F0FAF97B6803F56C42F63207F12E
S3150802CEE00C031068516803C312891A803B7B1946E2
S3150802CEF07B7B1846BB7B1C46FB7B3A7C01920093E4
S3150802CF002346024645480EF0D9FD002387F82F30FE
S3150802CF101DE097F82F305B0030333B4433F8183C5A
S3150802CF207A889A420ED197F82F305B0030333B4409
S3150802CF30002223F8182C97F82F3030333B4400226E
S3150802CF4003F8242C97F82F30013387F82F3097F8F7
S3150802CF502F30092BDDD97B6803F56C43E0331422A5
S3150802CF600021184629F0FAF87B6803F56C43F63374
S3150802CF700A220021184629F0F1F8002387F82E30F4
S3150802CF80002387F82F3030E097F82F305B003033D4
S3150802CF903B4433F8183C002B22D097F82F3097F8E9
S3150802CFA02E105B0030333B4433F8180C7A6801F5CF
S3150802CFB0EC437033014622F8131097F82F2097F89E
S3150802CFC02E30591C87F82E10194602F130033B44BD
S3150802CFD013F8242C7B680B4403F56C43F6331A705A
S3150802CFE097F82F30013387F82F3097F82F30092B0F
S3150802CFF0CAD97B8819467868FFF742FE7868FFF730
S3150802D0000FFF03461A467B88934202D17868FFF7D8
S3150802D01016FF00BF3437BD4690BD00BF48D7050886
S3150802D02080B483B000AF78607B6803F5604393F8F9
S3150802D030F63C18460C37BD465DF8047B704780B44B
S3150802D04083B000AF78600B46FB70FB787A681344AE
S3150802D05003F56C43F6331B7818460C37BD465DF864
S3150802D060047B7047F0B595B00AAF7861396113460B
S3150802D070FB7300237B6200233B620023FB770023BA
S3150802D080BB771EF0A5F8B861FB7B19467869FFF7EE
S3150802D09095FD7862386921F016FB03461A4640F276
S3150802D0A0BC4302FB03F37A6A134404333B623869CE
S3150802D0B021F009FB03461946B8691EF0CAF8386911
S3150802D0C021F01CFB03461946B8691EF0D1F83869E7
S3150802D0D021F02FFB03461946B8691EF0E4F83869B1
S3150802D0E021F042FB0346FB77386921F058FB0346D9
S3150802D0F0BB7723F0F7F90246FB7F1946104623F061
S3150802D10009FA23F0EFF90246BB7F1946104623F0C7
S3150802D11010FAFB7F012B0ED123F0E4F90346002116
S3150802D120184623F015FA034602334FF4E472002137
S3150802D130184629F013F823F0D5F9034600211846B4
S3150802D14023F006FA0146FB7F5A1E1346DB009B1A9A
S3150802D150DB000B449C1C386921F03CFB0346382251
S3150802D1601946204629F0B1F8FA7FBB7F9A423FD189
S3150802D17023F0B8F97B6A0022002123F0C5FE7B6AF8
S3150802D180043340F2BC421946386A29F09EF87B6A93
S3150802D1901B889C467B6A5B799E467B6A9B791A4604
S3150802D1A07B6ADB7919467B6A1B7A18467B6A5B7A45
S3150802D1B01C467B6A9B7A1D467B6ADB7A1E467B6A1D
S3150802D1C01B7BBB607B6A5B7B7B607B6A9B7B089372
S3150802D1D07B680793BB6806930596049503940290A9
S3150802D1E001910092734662460349022009F094FBB4
S3150802D1F000BF2C37BD46F0BD7CD705082DE9F043A4
S3150802D2009BB00AAFF861B961002387F83F30002363
S3150802D21087F83E30002387F83D30002387F83C30F4
S3150802D220002387F83B3007F1200300221A605A6070
S3150802D2309A60DA601A61002387F83F3071E097F83E
S3150802D2403F301946F869FFF7B9FC7863B86921F0E7
S3150802D25055FA03461A467B6B1B889A425CD1012310
S3150802D26087F83E3097F83F3087F83D300021B86995
S3150802D27021F0BCFA034698460121B86921F0B6FAAC
S3150802D280034699460221B86921F0B0FA03461C46BC
S3150802D2900321B86921F0AAFA03461D460421B86992
S3150802D2A021F0A4FA03461E460521B86921F09EFA22
S3150802D2B003467B610621B86921F098FA03463B6169
S3150802D2C00721B86921F092FA0346FB600821B8697A
S3150802D2D021F08CFA0346BB600921B86921F086FA67
S3150802D2E003467B600A21B86921F080FA034608934F
S3150802D2F07A680792BA680692FA6805923A690492B7
S3150802D3007B6903930296019500944B4642469E49D1
S3150802D310022009F001FB08E097F83F30013387F84D
S3150802D3203F3097F83F30092B89D997F83E30002BC2
S3150802D33030D096480EF0C2FBB86921F0C4F903460C
S3150802D340042B1CD897F83D301A46B969F869FFF7D5
S3150802D35089FEB86921F0D2F903461C46B86921F05C
S3150802D360B2F903461D46B86921F0E3F9034600936C
S3150802D3702B4622468649022009F0CEFAFEE0B86913
S3150802D38021F0BCF903461A468249022009F0C4FA7A
S3150802D3900023F4E0002387F83F301DE097F83F307A
S3150802D3A01946F869FFF70AFC78637B6B1B88002B22
S3150802D3B00DD1012387F83C3097F83F3087F83B3088
S3150802D3C097F83F301946F869FFF740FC08E097F8E6
S3150802D3D03F30013387F83F3097F83F30092BDDD9C4
S3150802D3E097F83C30002B00F08A806B480EF066FBFB
S3150802D3F00021B86921F0FAF9034698460121B8696D
S3150802D40021F0F4F9034699460221B86921F0EEF9AA
S3150802D41003461C460321B86921F0E8F903461D466E
S3150802D4200421B86921F0E2F903461E460521B869C6
S3150802D43021F0DCF903467B610621B86921F0D6F9A9
S3150802D44003463B610721B86921F0D0F90346FB6020
S3150802D4500821B86921F0CAF90346BB600921B869EF
S3150802D46021F0C4F903467B600A21B86921F0BEF9A6
S3150802D47003461A467B6BDB7B099308927A68079206
S3150802D480BA680692FA6805923A6904927B69039326
S3150802D4900296019500944B4642464049022009F0FD
S3150802D4A03BFA97F83B301946F869FFF787FB78632A
S3150802D4B0B86921F023F903461A467B6B1A807B6BFF
S3150802D4C000229A7097F83B301A46B969F869FFF74D
S3150802D4D0C9FDB86921F0F7F803461C46B86921F078
S3150802D4E00DF903461D46B86921F023F90346009350
S3150802D4F02B4622462A49022009F00EFA3EE000236C
S3150802D50087F83F3016E097F83F301946F869FFF773
S3150802D51055FB786397F83F307A6B12885B0028339D
S3150802D52007F118010B4423F8202C97F83F300133F2
S3150802D53087F83F3097F83F30092BE4D93B8C9E4653
S3150802D5407B8C9846BB8C7B61FA8C398D788DBC8D29
S3150802D550FD8D3E8EB7F832C063460793069605954B
S3150802D56004940390029101927B69009343467246A2
S3150802D5700C49022009F0D0F9002300E001231846DD
S3150802D5804437BD46BDE8F083BCD70508F8D7050879
S3150802D59030D8050868D8050894D80508CCD80508EF
S3150802D5A00CD9050840D9050880B582B000AF786065
S3150802D5B00B46FB700A481EF0F1F80246FB789A42BF
S3150802D5C006D3FB781A46796805481EF061F902E027
S3150802D5D004480EF073FA00BF0837BD4680BD00BF87
S3150802D5E05007012090D9050880B582B000AF78604F
S3150802D5F00B46FB700A481EF0D1F80246FB789A429F
S3150802D60006D3FB781A46796805481EF041F902E006
S3150802D61004480EF053FA00BF0837BD4680BD00BF66
S3150802D62074070120BCD9050880B590B000AFF8632D
S3150802D63087ED0C0B87ED0A1B87ED082B87ED063B5A
S3150802D64087ED044B87ED025BB9637A603B60FB6B3F
S3150802D650BA6B1A66FB6B7A68DA67FB6B012283F888
S3150802D6607920F96BD7E90223C1E90E2397ED041B4A
S3150802D67097ED060BF86B00F0F9F8012197ED082BE8
S3150802D68097ED0A1B97ED0C0BF86B00F04BF839680F
S3150802D690F86B00F056F9F96B4FF000024FF00003F1
S3150802D6A0C1E91623F96B4FF000024FF00003C1E9F6
S3150802D6B01423F96B4FF000024FF00003C1E910235F
S3150802D6C0F96B4FF000024FF00003C1E9122300BFC5
S3150802D6D04037BD4680BD80B483B000AF78607968B4
S3150802D6E04FF000024FF00003C1E9162379684FF0A4
S3150802D6F000024FF00003C1E9142379684FF00002D3
S3150802D7004FF00003C1E9102379684FF000024FF089
S3150802D7100003C1E9122300BF0C37BD465DF8047B3E
S3150802D7207047000080B58AB000AFF86187ED040B38
S3150802D73087ED021B87ED002BB9614FF000024FF00F
S3150802D7400003D7E90401F3F7F7FA0346002B40F082
S3150802D75086804FF000024FF00003D7E90201F3F783
S3150802D760EBFA0346002B7AD14FF000024FF0000382
S3150802D770D7E90001F3F7E0FA0346002B6FD1BB693C
S3150802D780012B0CBF01230023DAB2FB6983F8782048
S3150802D790F969D7E90423C1E90023F969D7E902231C
S3150802D7A0C1E90223F969D7E90023C1E90423FB6920
S3150802D7B01B6E1846F2F7D4FF4FF000022A4BF3F716
S3150802D7C073F902460B46C7E90823F969D7E9042320
S3150802D7D0C1E90623D7E90823D7E90201F3F73AF89C
S3150802D7E002460B46F969C1E90823D7E90823D7E9AE
S3150802D7F00001F3F759F902460B46F969C1E90A230A
S3150802D800FB691B6B012B2BD1FB69D3E906234FF06E
S3150802D81000004FF00001F2F765FE02460B46F96971
S3150802D820C1E90623FB69D3E908234FF000004FF04C
S3150802D8300001F2F757FE02460B46F969C1E90823C9
S3150802D840FB69D3E90A234FF000004FF00001F2F713
S3150802D85049FE02460B46F969C1E90A2300E000BF00
S3150802D8602837BD4680BD00BF00408F4080B586B0D0
S3150802D87000AF786187ED020B87ED001BD7E900231D
S3150802D880D7E90201F3F76CFA0346002B55D17969F9
S3150802D890D7E90223C1E91A237969D7E90023C1E93D
S3150802D8A01C237B6993F87930002B47D07B69D3E92F
S3150802D8B012017B69D3E91C23F3F75CFA0346002BB2
S3150802D8C006D07B69D3E91C237969C1E9122310E0E2
S3150802D8D07B69D3E912017B69D3E91A23F3F72CFA98
S3150802D8E00346002B05D07B69D3E91A237969C1E976
S3150802D8F012237B69D3E914017B69D3E91C23F3F765
S3150802D90039FA0346002B06D07B69D3E91C237969C9
S3150802D910C1E9142312E07B69D3E914017B69D3E9CF
S3150802D9201A23F3F709FA0346002B07D07B69D3E9D2
S3150802D9301A237969C1E9142300E000BF1837BD46E6
S3150802D94080BD80B582B000AF786039607B6893F895
S3150802D9507930002B2ED07B681B6B3A689A4229D005
S3150802D9607B68D3E906234FF000004FF00001F2F777
S3150802D970B9FD02460B467968C1E906237B68D3E9F5
S3150802D98008234FF000004FF00001F2F7ABFD024604
S3150802D9900B467968C1E908237B68D3E90A234FF065
S3150802D9A000004FF00001F2F79DFD02460B4679682A
S3150802D9B0C1E90A237B683A681A6300BF0837BD467D
S3150802D9C080BDB0B58CB000AF78604FF000024FF062
S3150802D9D00003C7E908234FF000024FF00003C7E926
S3150802D9E006234FF000024FF00003C7E904234FF065
S3150802D9F000024FF00003C7E90A237B68DB6FFB606E
S3150802DA007B6893F8793083F00103DBB2002B01D0EF
S3150802DA100023F0E07B681B6EFA689A42C0F0EA803F
S3150802DA207B68D3E91023C7E908237B68D3E90E018B
S3150802DA30D7E90823F2F756FD02460B46C7E906233D
S3150802DA407B68D3E91623D7E90801F2F74BFD0246AC
S3150802DA500B46C7E904237B68D3E914457B68D3E9F7
S3150802DA600801D7E90623F2F7F5FE02460B462046D9
S3150802DA702946F2F739FD02460B467968C1E91423AD
S3150802DA807B6893F8783083F00103DBB2002B14D05D
S3150802DA907B68D3E914457B68D3E90601D7E90423F1
S3150802DAA0F2F7D8FE02460B4620462946F2F71AFD39
S3150802DAB002460B467968C1E914237B68D3E9140147
S3150802DAC07B68D3E91C23F3F755F90346002B06D0E6
S3150802DAD07B68D3E91C237968C1E9142310E07B68C3
S3150802DAE0D3E914017B68D3E91A23F3F725F9034628
S3150802DAF0002B05D07B68D3E91A237968C1E9142378
S3150802DB007B6893F87830002B0BD07B68D3E9062321
S3150802DB10D7E90601F2F79EFE02460B46C7E90A2333
S3150802DB2005E04FF000024FF00003C7E90A237B68BD
S3150802DB30D3E914457B68D3E90A01D7E90423F2F746
S3150802DB4089FE02460B4620462946F2F7CBFC0246D8
S3150802DB500B46D7E90A01F2F7C7FC02460B46C7E9A4
S3150802DB600A237B68D3E91C23D7E90A01F3F702F9EA
S3150802DB700346002B05D07B68D3E91C23C7E90A2391
S3150802DB800EE07B68D3E91A23D7E90A01F3F7D4F83A
S3150802DB900346002B04D07B68D3E91A23C7E90A2374
S3150802DBA07968D7E90A23C1E912237968D7E90823EC
S3150802DBB0C1E916237B68D3E90E014FF000024FF044
S3150802DBC00003F3F7AFF80346002B11D04FF000021B
S3150802DBD04FF00003D7E90601F3F7A4F80346002B32
S3150802DBE006D079684FF000024FF00003C1E912230C
S3150802DBF0012300E0002318463037BD46B0BD80B485
S3150802DC0083B000AF78607B68D3E90E2343EC172B09
S3150802DC10B0EE470AF0EE670A0C37BD465DF8047B9C
S3150802DC20704780B485B000AFF86087ED000BF968DD
S3150802DC30D7E90023C1E90E2300BF1437BD465DF8B4
S3150802DC40047B704780B485B000AFF86087ED000B9F
S3150802DC50F968D7E90023C1E9102300BF1437BD4686
S3150802DC605DF8047B704780B483B000AF78607B6848
S3150802DC70D3E9122343EC172BB0EE470AF0EE670AF4
S3150802DC800C37BD465DF8047B7047000080B500AFCF
S3150802DC90074B1B78DBB2002B07D1054B01221A7002
S3150802DCA002220021034828F059FA024B184680BD81
S3150802DCB0B6F40120B4F4012080B483B000AF7860D2
S3150802DCC07B681B7818460C37BD465DF8047B70479F
S3150802DCD080B483B000AF78600B46FB70FB78002BEC
S3150802DCE005D1074B00221A70064B00221A607B6880
S3150802DCF0FA781A7000BF0C37BD465DF8047B704788
S3150802DD00ADF40120B0F4012080B483B000AF78608E
S3150802DD107B685B7818460C37BD465DF8047B70470E
S3150802DD2080B483B000AF78600B46FB707B68FA78E4
S3150802DD305A7000BF0C37BD465DF8047B7047000079
S3150802DD4080B500AF4F4B1B78002B02D0012B28D091
S3150802DD5056E0FAF75BFC034600211846FAF7AFFFCE
S3150802DD600346012B16D1FAF751FC03460121184640
S3150802DD70FAF7A5FF0346022B0CD1434B00221A6081
S3150802DD80424B00221A603F4B1B780133DAB23D4BF5
S3150802DD901A7035E03E4B1B6863225A63FAF722FF74
S3150802DDA02EE03A4B1B680133384A1360374B1B681F
S3150802DDB0312B1ED9344B00221A60344B00221A60CA
S3150802DDC0304B1B780133DAB22E4B1A70FFF75EFF1F
S3150802DDD0034601211846FFF77BFFFFF757FF034665
S3150802DDE000211846FFF79CFFFAF70AFFFAF71EFF0B
S3150802DDF005E0274B1B6863225A63FAF7F3FE00BF56
S3150802DE00214B1B680133204A13601F4B1B6841F2E2
S3150802DE106F72934234D9FAF7F3FEFAF707FFFAF765
S3150802DE20F5FB034600211846FAF749FF0346012B7C
S3150802DE3018D1FAF7EBFB034601211846FAF73FFF1A
S3150802DE400346012B0ED1FFF721FF03460721184689
S3150802DE50FFF73EFF22F05AFA01230D22382122F05B
S3150802DE60D1FA0DE0FFF712FF034606211846FFF71F
S3150802DE702FFF22F04BFA01230D22382122F0C2FA93
S3150802DE8000BF80BDADF40120B0F40120B8F4012032
S3150802DE90BC05012080B500AFFFF7F8FE0346184619
S3150802DEA0FFF732FF0346002B14D1C84B00221A6033
S3150802DEB0C74B00221A60FAF7A3FEFFF7E7FE0346EE
S3150802DEC01846FFF7F9FE0346032B00F0C880FAF757
S3150802DED0ADFEC4E0FFF7DAFE03461846FFF714FF65
S3150802DEE00346012B0ED1FFF7D1FE03460021184641
S3150802DEF0FFF7EEFEFFF7CAFE034600211846FFF7B4
S3150802DF000FFF9AE1FFF7C2FE03461846FFF7FCFE2B
S3150802DF100346022B4ED1FFF7B9FE034604211846E3
S3150802DF20FFF7D6FEFAF772FB034600211846FAF700
S3150802DF30C6FE0346012B36D1FAF768FB03460121D2
S3150802DF401846FAF7BCFE0346022B2CD19F4B1B68D8
S3150802DF5001339E4A13609D4B1B68312B1CD99D4980
S3150802DF60022008F0D9FC994B00221A60984B00222D
S3150802DF701A60FAF745FEFAF759FEFFF787FE0346D7
S3150802DF8000211846FFF7CCFEFFF780FE0346022162
S3150802DF901846FFF79DFE62E08F4B1B6863225A63A1
S3150802DFA0FAF720FE5BE08C4B1B6863225A63FAF78A
S3150802DFB019FE54E0FFF76AFE03461846FFF7A4FE69
S3150802DFC00346032B4BD1FFF761FE0346042118468D
S3150802DFD0FFF77EFEFAF71AFB034600211846FAF700
S3150802DFE06EFE0346022B34D1FAF710FB03460121D3
S3150802DFF01846FAF764FE0346012B2AD1734B1B68AF
S3150802E0000133724A1360714B1B68312B1AD9734953
S3150802E010022008F081FC6D4B00221A606C4B00222C
S3150802E0201A60FAF7EDFDFFF731FE0346002118469E
S3150802E030FFF776FEFFF72AFE034603211846FFF787
S3150802E04047FE0CE0644B1B6863229A63FAF7BCFD31
S3150802E05005E0614B1B6863229A63FAF7B5FDFFF781
S3150802E06015FE03461846FFF74FFE0346002B00F03F
S3150802E070E480574B1B680133554A1360544B1B689F
S3150802E08041F26F72934240F2D880FAF7B9FDFAF775
S3150802E090CDFDFFF7FBFD03461846FFF735FE03469F
S3150802E0A0022B55D1FAF7B2FA034600211846FAF7B7
S3150802E0B006FE0346012B2AD1FAF7A8FA03460121DE
S3150802E0C01846FAF7FCFD0346012B20D1FFF7DEFDC1
S3150802E0D0034607211846FFF7FBFD4149022008F0CF
S3150802E0E01BFC22F013F901230D22382122F08AF9AA
S3150802E0F007F06AFE03463821184608F0E7FA07F0E1
S3150802E10063FE03460D21184608F0FEFA8EE0FFF775
S3150802E110BDFD034606211846FFF7DAFD31490220FE
S3150802E12008F0FAFB22F0F2F801230D22382122F038
S3150802E13069F907F049FE03463821184608F0C6FA77
S3150802E14007F042FE03460D21184608F0DDFA6DE097
S3150802E150FFF79CFD03461846FFF7D6FD0346032B39
S3150802E16064D1FAF753FA034600211846FAF7A7FDCF
S3150802E1700346012B3AD1FAF749FA03460121184612
S3150802E180FAF79DFD0346012B30D1FFF77FFD0346C3
S3150802E19008211846FFF79CFD1349022008F0BCFB2C
S3150802E1A022F0B4F801230C22382122F02BF907F0C9
S3150802E1B00BFE03463821184608F088FA07F004FED3
S3150802E1C003460C21184608F09FFA2FE0BCF40120FA
S3150802E1D0C0F40120E0D90508BC050120F4D90508D8
S3150802E1E008DA050820DA050838DA0508FFF74EFDC9
S3150802E1F0034609211846FFF76BFD1049022008F06D
S3150802E2008BFB22F083F801230C22382122F0FAF83C
S3150802E21007F0DAFD03463821184608F057FA07F0E0
S3150802E220D3FD03460C21184608F06EFAFFF72EFDB9
S3150802E230034600211846FFF773FD80BD50DA05082C
S3150802E24080B500AF1C4B1B78002B33D107F0BCFD01
S3150802E2500346184607F048FE0346002B04D0FAF791
S3150802E260CFFCFAF7E3FC26E0FFF710FD0346184653
S3150802E270FFF722FD0346002B02D1FFF761FD1AE0E4
S3150802E280FFF704FD03461846FFF716FD0346042B5F
S3150802E2900DD9FFF7FBFC03461846FFF70DFD0346AB
S3150802E2A00A2B04D8FAF7ACFCFAF7C0FC03E0FFF72E
S3150802E2B0F1FD00E000BF80BD4A90002080B500AFA6
S3150802E2C0074B1B78DBB2002B07D1054B01221A70CC
S3150802E2D018220021034827F041FF024B184680BD49
S3150802E2E0AAF50120C8F4012080B483B000AF786093
S3150802E2F07B685B6818460C37BD465DF8047B704739
S3150802E30080B485B000AF78607B685B68FB60FB68A9
S3150802E3100133FB607B68FA685A6000BF1437BD4652
S3150802E3205DF8047B704780B485B000AF78607B687F
S3150802E3305B68FB60FB68013BFB607B68FA685A60B6
S3150802E34000BF1437BD465DF8047B704780B483B0BE
S3150802E35000AF786039607B683A685A6000BF0C374C
S3150802E360BD465DF8047B704780B483B000AF786021
S3150802E3707B689B6818460C37BD465DF8047B704778
S3150802E38080B483B000AF786039607B683A689A6077
S3150802E39000BF0C37BD465DF8047B704780B483B076
S3150802E3A000AF78607B681B7B18460C37BD465DF864
S3150802E3B0047B704780B483B000AF78600B46FB706D
S3150802E3C07B68FA781A7300BF0C37BD465DF8047B82
S3150802E3D0704780B483B000AF78607B685B7B184671
S3150802E3E00C37BD465DF8047B704780B582B000AF36
S3150802E3F078600B46FB707B68FA785A730221786854
S3150802E40000F02FFA00BF0837BD4680BD80B483B03E
S3150802E41000AF78607B689B7B18460C37BD465DF873
S3150802E420047B704780B483B000AF78600B46FB70FC
S3150802E4307B68FA789A7300BF0C37BD465DF8047B91
S3150802E440704780B582B000AF0023FB710023BB7111
S3150802E45000237B7100233B71FAF7D8F803460021A3
S3150802E4601846FAF732F90346012B01D10123FB714B
S3150802E470FAF7CCF8034601211846FAF726F90346B5
S3150802E480012B01D10223BB71FAF7C0F80346022118
S3150802E4901846FAF71AF90346012B01D104237B71B0
S3150802E4A0FAF7B4F8034603211846FAF70EF90346B3
S3150802E4B0012B01D108233B71FA79BB791343DAB2EE
S3150802E4C07B791343DAB23B791343DBB21846083732
S3150802E4D0BD4680BD80B485B000AF78600B46FB7040
S3150802E4E00023FB73FB780E2B38D801A252F823F0CF
S3150802E4F02DE502085DE5020857E502085DE5020812
S3150802E50051E502085DE502084BE502085DE50208E9
S3150802E51045E502085DE502083FE502085DE50208F1
S3150802E52039E502085DE5020833E502080123FB73B3
S3150802E53015E00823FB7312E00723FB730FE006239B
S3150802E540FB730CE00523FB7309E00423FB7306E067
S3150802E5500323FB7303E00223FB7300E000BF7B681F
S3150802E560FA7B9A7400BF1437BD465DF8047B704780
S3150802E57080B485B000AF78600B46FB700023FB734E
S3150802E580FB780E2B38D801A252F823F0C9E5020807
S3150802E590F9E50208F3E50208F9E50208EDE50208DD
S3150802E5A0F9E50208E7E50208F9E50208E1E50208E5
S3150802E5B0F9E50208DBE50208F9E50208D5E50208ED
S3150802E5C0F9E50208CFE502080623FB7315E00523E1
S3150802E5D0FB7312E00423FB730FE00323FB730CE0C7
S3150802E5E00223FB7309E00123FB7306E00823FB738E
S3150802E5F003E00723FB7300E000BF7B68FA7BDA744B
S3150802E60000BF1437BD465DF8047B704780B483B0FB
S3150802E61000AF78607B681B7D18460C37BD465DF8EF
S3150802E620047B704780B485B000AF78600B46FB70F8
S3150802E6300023FB73FB780E2B38D801A252F823F07D
S3150802E6407DE60208ADE60208A7E60208ADE602087C
S3150802E650A1E60208ADE602089BE60208ADE6020854
S3150802E66095E60208ADE602088FE60208ADE602085C
S3150802E67089E60208ADE6020883E602080523FB736B
S3150802E68015E00423FB7312E00323FB730FE0022356
S3150802E690FB730CE00123FB7309E00823FB7306E016
S3150802E6A00723FB7303E00623FB7300E000BF7B68C6
S3150802E6B0FA7B1A7500BF1437BD465DF8047B7047AE
S3150802E6C080B483B000AF78607B685B7D18460C37F0
S3150802E6D0BD465DF8047B704780B485B000AF7860AC
S3150802E6E00B46FB700023FB73FB780E2B38D801A26E
S3150802E6F052F823F031E7020861E702085BE70208ED
S3150802E70061E7020855E7020861E702084FE70208CF
S3150802E71061E7020849E7020861E7020843E70208D7
S3150802E72061E702083DE7020861E7020837E70208DF
S3150802E7300323FB7315E00223FB7312E00123FB7329
S3150802E7400FE00823FB730CE00723FB7309E006239B
S3150802E750FB7306E00523FB7303E00423FB7300E067
S3150802E76000BF7B68FA7B5A7500BF1437BD465DF851
S3150802E770047B704780B582B000AF78600B46FB70A9
S3150802E780FB7819467868FFF7A5FEFB78194678687C
S3150802E790FFF7EEFEFB7819467868FFF743FFFB782A
S3150802E7A019467868FFF798FF00BF0837BD4680BD4F
S3150802E7B080B483B000AF78607B68DB7B18460C3781
S3150802E7C0BD465DF8047B704780B483B000AF7860BD
S3150802E7D07B680022DA7300BF0C37BD465DF8047BFE
S3150802E7E0704780B483B000AF78607B681B7C18469C
S3150802E7F00C37BD465DF8047B704780B483B000AF22
S3150802E80078607B6800221A7400BF0C37BD465DF833
S3150802E810047B704780B483B000AF78607B685B7C0A
S3150802E82018460C37BD465DF8047B704780B483B042
S3150802E83000AF78600B46FB707B68FA785A7400BFA3
S3150802E8400C37BD465DF8047B704780B483B000AFD1
S3150802E85078607B681B7818460C37BD465DF8047BE2
S3150802E860704780B483B000AF78600B46FB707B6854
S3150802E870FA781A7000BF0C37BD465DF8047B7047FC
S3150802E88080B584B000AF03460A46FB711346BB71D6
S3150802E8900023FB73FB79072B4AD801A252F823F00F
S3150802E8A0C1E80208CFE80208DDE80208EBE8020838
S3150802E8B0F9E8020807E9020815E9020823E9020845
S3150802E8C0BB79184600F03AF80346FB7330E0BB7989
S3150802E8D0184600F0DBF80346FB7329E0BB791846B5
S3150802E8E000F032F90346FB7322E0BB79184600F0C2
S3150802E8F089F90346FB731BE0BB79184600F0E0F979
S3150802E9000346FB7314E0BB79184600F037FA034650
S3150802E910FB730DE0BB79184600F08EFA0346FB73CB
S3150802E92006E0BB79184600F0E5FA0346FB7300BF1A
S3150802E930FB7B18461037BD4680BD00BF80B483B046
S3150802E94000AF0346FB71FB790F2B43D801A252F89D
S3150802E95023F000BF95E9020899E902089DE9020831
S3150802E960A1E90208A5E90208A9E90208ADE902082F
S3150802E970B1E90208B5E90208B9E90208BDE90208DF
S3150802E980C1E90208C5E90208C9E90208CDE902088F
S3150802E990D1E9020807231EE011231CE006231AE028
S3150802E9A0102318E0052316E00F2314E0042312E0CF
S3150802E9B00E2310E008230EE00D230CE009230AE0DB
S3150802E9C00C2308E0032306E00B2304E0022302E0FB
S3150802E9D00A2300E0002318460C37BD465DF8047B7F
S3150802E9E0704700BF80B483B000AF0346FB71FB7962
S3150802E9F0023B0F2B42D801A252F823F075EA02080D
S3150802EA006DEA020855EA02084DEA020845EA0208D2
S3150802EA103DEA02085DEA020865EA020879EA02089E
S3150802EA2071EA020869EA020861EA020859EA020872
S3150802EA3051EA020849EA020841EA020800231FE0ED
S3150802EA4001231DE002231BE0032319E0042317E038
S3150802EA50052315E0062313E0072311E008230FE038
S3150802EA6009230DE00A230BE00B2309E00C2307E038
S3150802EA700D2305E00E2303E00F2301E000BF002368
S3150802EA8018460C37BD465DF8047B704780B483B0E0
S3150802EA9000AF0346FB71FB79023B0C2B24D801A27B
S3150802EAA052F823F0DDEA0208E9EA0208E9EA02086E
S3150802EAB0E9EA0208E1EA0208E9EA0208E9EA0208DA
S3150802EAC0E9EA0208E5EA0208E9EA0208E9EA0208C6
S3150802EAD0E9EA0208D9EA0208072306E0052304E060
S3150802EAE0082302E0032300E0002318460C37BD463C
S3150802EAF05DF8047B704700BF80B483B000AF03465D
S3150802EB00FB71FB79033B052B16D801A252F823F0B9
S3150802EB1035EB020839EB02082DEB020839EB02083D
S3150802EB2029EB020831EB02080E2307E0022305E06F
S3150802EB30062303E00A2301E000BF002318460C3728
S3150802EB40BD465DF8047B704780B483B000AF0346C8
S3150802EB50FB71FB790C2B25D801A252F823F000BFD2
S3150802EB6099EB0208A5EB0208A5EB0208A5EB020839
S3150802EB709DEB0208A5EB0208A5EB0208A5EB020825
S3150802EB80A1EB0208A5EB0208A5EB0208A5EB020811
S3150802EB9095EB0208072306E0052304E0082302E0B2
S3150802EBA0032300E0002318460C37BD465DF8047BB4
S3150802EBB0704700BF80B483B000AF0346FB71FB7990
S3150802EBC0033B052B16D801A252F823F0F1EB0208F3
S3150802EBD0F5EB0208E9EB0208F5EB0208E5EB020899
S3150802EBE0EDEB02080C2307E0002305E0042303E00B
S3150802EBF0082301E000BF002318460C37BD465DF81E
S3150802EC00047B704780B483B000AF0346FB71FB797F
S3150802EC10023B0C2B24D801A252F823F059EC020825
S3150802EC2061EC020861EC020861EC02085DEC02087C
S3150802EC3061EC020861EC020861EC020851EC020878
S3150802EC4061EC020861EC020861EC020855EC020864
S3150802EC50072306E0052304E0082302E0032300E075
S3150802EC60002318460C37BD465DF8047B704700BF83
S3150802EC7080B483B000AF0346FB71FB79033B052BD7
S3150802EC8016D801A252F823F0ADEC0208B1EC02083C
S3150802EC90A5EC0208B1EC0208A1EC0208A9EC0208EC
S3150802ECA00A2307E00E2305E0022303E0062301E018
S3150802ECB000BF002318460C37BD465DF8047B704733
S3150802ECC080B483B000AF0346FB71FB790C2B25D8C1
S3150802ECD001A252F823F000BF15ED02081DED020845
S3150802ECE01DED02081DED020819ED02081DED0208C8
S3150802ECF01DED02081DED02080DED02081DED0208C4
S3150802ED001DED02081DED020811ED0208072306E0B3
S3150802ED10052304E0082302E0032300E00023184643
S3150802ED200C37BD465DF8047B704700BF80B483B0DC
S3150802ED3000AF0346FB71FB79033B052B16D801A2EC
S3150802ED4052F823F069ED02086DED020861ED02083A
S3150802ED506DED02085DED020865ED0208082307E07D
S3150802ED600C2305E0002303E0042301E000BF00238F
S3150802ED7018460C37BD465DF8047B704780B483B0ED
S3150802ED8000AF0346FB71FB79023B0C2B24D801A288
S3150802ED9052F823F0D5ED0208D9ED0208D9ED02089A
S3150802EDA0D9ED0208C9ED0208D9ED0208D9ED020823
S3150802EDB0D9ED0208CDED0208D9ED0208D9ED02080F
S3150802EDC0D9ED0208D1ED0208072306E0052304E07F
S3150802EDD0082302E0032300E0002318460C37BD4649
S3150802EDE05DF8047B704700BF80B483B000AF03466A
S3150802EDF0FB71FB79033B052B16D801A252F823F0C7
S3150802EE0025EE020829EE02081DEE020829EE02087E
S3150802EE1019EE020821EE0208062307E00A2305E096
S3150802EE200E2303E0022301E000BF002318460C3735
S3150802EE30BD465DF8047B704780B483B000AF0346D5
S3150802EE40FB71FB790C2B25D801A252F823F000BFDF
S3150802EE5091EE020895EE020895EE020895EE020872
S3150802EE6085EE020895EE020895EE020895EE02086E
S3150802EE7089EE020895EE020895EE020895EE02085A
S3150802EE808DEE0208072306E0052304E0082302E0C4
S3150802EE90032300E0002318460C37BD465DF8047BC1
S3150802EEA0704700BF80B483B000AF0346FB71FB799D
S3150802EEB0033B052B16D801A252F823F0E1EE02080D
S3150802EEC0E5EE0208D9EE0208E5EE0208D5EE0208DA
S3150802EED0DDEE0208042307E0082305E00C2303E01D
S3150802EEE0002301E000BF002318460C37BD465DF833
S3150802EEF0047B704780B483B000AF0346FB71FB798D
S3150802EF00023B0C2B24D801A252F823F041EF020847
S3150802EF1051EF020851EF020851EF020845EF0208C5
S3150802EF2051EF020851EF020851EF020849EF0208B1
S3150802EF3051EF020851EF020851EF02084DEF02089D
S3150802EF40072306E0052304E0082302E0032300E082
S3150802EF50002318460C37BD465DF8047B704700BF90
S3150802EF6080B483B000AF0346FB71FB79033B052BE4
S3150802EF7016D801A252F823F09DEF0208A1EF020863
S3150802EF8095EF0208A1EF020891EF020899EF02082D
S3150802EF90022307E0062305E00A2303E00E2301E025
S3150802EFA000BF002318460C37BD465DF8047B704740
S3150802EFB080B582B000AF78607B68012B06D1FFF777
S3150802EFC07DF903461846FFF7AEF909E07B68B3F107
S3150802EFD0FF3F05D1FFF772F903461846FFF790F986
S3150802EFE000BF0837BD4680BD80B500AF1A4B1B6807
S3150802EFF080220021184627F0B1F8174B1868174BDC
S3150802F00093ED007B164B93ED006B164B93ED002B9D
S3150802F010154B93ED005B154B1968002364229FED8F
S3150802F0200A4B9FED0B3BB0EE461AF0EE661AB0EEAF
S3150802F030470AF0EE670AFEF7F7FAF9F715FD00BF79
S3150802F04080BD00BFAFF300800000000000005940F9
S3150802F0500000000000000000F4120020E0F4012085
S3150802F060E8120020E8F40120F0F40120F012002052
S3150802F07080B500AF0C4B1B689FED090B1846FEF7CF
S3150802F080D0FD094B1B681846FEF725FBFFF716F954
S3150802F090034600211846FFF759F900BF80BD00BF95
S3150802F0A00000000000000000F412002080B483B0C3
S3150802F0B000AF0346FB71FB790F2B43D801A252F826
S3150802F0C023F000BF05F1020809F102080DF1020852
S3150802F0D011F1020815F1020819F102081DF10208D8
S3150802F0E021F1020825F1020829F102082DF1020888
S3150802F0F031F1020835F1020839F102083DF1020838
S3150802F10041F1020801231EE002231CE003231AE050
S3150802F110042318E0052316E0062314E0072312E069
S3150802F120082310E009230EE00A230CE00B230AE069
S3150802F1300C2308E00D2306E00E2304E00F2302E069
S3150802F140102300E0002318460C37BD465DF8047B01
S3150802F150704700BF80B586B000AF0346FB710B4609
S3150802F160BB7113467B710023FB750023BB75002315
S3150802F1703B610023FB607B79FF2B07D0BA797B7949
S3150802F1809A4203D0FA797B799A4249D1FB79BB75BF
S3150802F1900023FB7512E0BA7DBB799A4212D0BB7D79
S3150802F1A00F2B02D90123BB7502E0BB7D0133BB7568
S3150802F1B03B6901333B61FB7D0133FB75FB7D0F2BFD
S3150802F1C0E9D900E000BFFB79BB750023FB7512E0A5
S3150802F1D0BA7DBB799A4212D0BB7D012B02D110238C
S3150802F1E0BB7502E0BB7D013BBB75FB680133FB6067
S3150802F1F0FB7D0133FB75FB7D0F2BE9D900E000BFD0
S3150802F2003A69FB689A4202D13B695B4270E03A6905
S3150802F210FB689A4201DDFB686AE03B695B4267E08C
S3150802F220FB79BB750023FB7519E07A79BB7D9A4297
S3150802F23002D1FF233B6117E0BA7DBB799A4212D00D
S3150802F240BB7D0F2B02D90123BB7502E0BB7D0133BF
S3150802F250BB753B6901333B61FB7D0133FB75FB7D66
S3150802F2600F2BE2D900E000BFFB79BB750023FB75C3
S3150802F27019E07A79BB7D9A4202D1FF23FB6017E037
S3150802F280BA7DBB799A4212D0BB7D012B02D11023DB
S3150802F290BB7502E0BB7D013BBB75FB680133FB60B6
S3150802F2A0FB7D0133FB75FB7D0F2BE2D900E000BF26
S3150802F2B03A69FB689A4208D13B69FF2B05D0FB687D
S3150802F2C0FF2B02D03B695B4212E03A69FB689A421D
S3150802F2D004DDFB68FF2B01D0FB6809E03B69FF2BC5
S3150802F2E002D03B695B4203E003480CF0E7FB0023CC
S3150802F2F018461837BD4680BD68DA050880B584B059
S3150802F30000AF03460A46FB711346BB710023FB6036
S3150802F310FB791846FFF7CAFE0346FB72FEF7CEFFD5
S3150802F32003461846FFF73AF803461846FFF7BEFEA5
S3150802F3300346BB72FB79102B0AD8FEF7BFFF0346BA
S3150802F3401846FFF72BF803461A46FB79934201D172
S3150802F350002320E0BB791846FFF7A8FE03461A46A3
S3150802F360F97ABB7A1846FFF7F5FEF860FB68002BB8
S3150802F37001D100230FE00A4B1B78022B06D1FA684B
S3150802F38013469B0013445A01134404E0FB684FF4E6
S3150802F3909B7202FB03F318461037BD4680BD00BFB9
S3150802F3A0C4F4012080B586B000AF03460A46FB7155
S3150802F3B01346BB7100237B61FB791846FFF776FE7D
S3150802F3C00346FB74FEF77AFF03461846FEF7E6FF86
S3150802F3D003461846FFF76AFE0346BB74BB7918460E
S3150802F3E0FFF764FE03461A46F97CBB7C1846FFF70C
S3150802F3F0B1FEF860FB68002B01D100233FE2AE4B59
S3150802F4001B78022B07D1FA6813469B0013445A014C
S3150802F41013447B6105E0FB684FF49B7202FB03F31E
S3150802F4207B61A54B1B78022B40F08E817B69002BF2
S3150802F43040F3B080FB68012B0FD106F0C5FC0346EA
S3150802F4400121184607F082F80346002B02D09B4892
S3150802F4500CF034FB7B695E3B11E2FB68022B10D190
S3150802F46006F0B2FC03460121184607F06FF8034678
S3150802F470002B02D092480CF021FB7B69A3F5877317
S3150802F480FDE1FB68032B10D106F09EFC0346012121
S3150802F490184607F05BF80346002B02D089480CF0A1
S3150802F4A00DFB7B69A3F5AF73E9E1FB68042B10D169
S3150802F4B006F08AFC03460121184607F047F8034678
S3150802F4C0002B02D080480CF0F9FA7B69A3F5B973D0
S3150802F4D0D5E1FB68052B10D106F076FC034601211F
S3150802F4E0184607F033F80346002B02D077480CF08B
S3150802F4F0E5FA7B69A3F5BE73C1E1FB68062B10D159
S3150802F50006F062FC03460121184607F01FF8034677
S3150802F510002B02D06E480CF0D1FA7B69A3F5BE73B4
S3150802F520ADE1FB68072B10D106F04EFC034601211C
S3150802F530184607F00BF80346002B02D065480CF074
S3150802F540BDFA7B69A3F5C87399E1FB68082B10D14C
S3150802F55006F03AFC03460121184606F0F7FF034671
S3150802F560002B02D05C480CF0A9FA7B69A3F5CD738F
S3150802F57085E106F029FC03460121184606F0E6FF56
S3150802F5800346002B02D055480CF098FA7B69A3F57E
S3150802F590D27374E1FB68B3F1FF3F0FD106F014FC96
S3150802F5A003460121184606F0D1FF0346002B02D076
S3150802F5B04B480CF083FA7B695E3360E1FB6813F112
S3150802F5C0020F10D106F000FC03460121184606F088
S3150802F5D0BDFF0346002B02D042480CF06FFA7B6946
S3150802F5E003F587734BE1FB6813F1030F10D106F09D
S3150802F5F0EBFB03460121184606F0A8FF0346002B3B
S3150802F60002D039480CF05AFA7B6903F5AF7336E132
S3150802F610FB6813F1040F10D106F0D6FB034601214D
S3150802F620184606F093FF0346002B02D02F480CF02B
S3150802F63045FA7B6903F5B97321E1FB6813F1050FF6
S3150802F64010D106F0C1FB03460121184606F07EFFDB
S3150802F6500346002B02D026480CF030FA7B6903F5E4
S3150802F660BE730CE1FB6813F1060F10D106F0ACFB72
S3150802F67003460121184606F069FF0346002B02D00D
S3150802F6801C480CF01BFA7B6903F5BE73F7E0FB68AE
S3150802F69013F1070F32D106F097FB034601211846EC
S3150802F6A006F054FF0346002B02D013480CF006FA64
S3150802F6B07B6903F5C873E2E0C4F401209CDA050805
S3150802F6C0D4DA05080CDB050844DB05087CDB0508EB
S3150802F6D0B4DB0508ECDB050824DC05085CDC050858
S3150802F6E094DC0508CCDC050804DD05083CDD0508C4
S3150802F6F074DD0508ACDD0508E4DD0508FB6813F1D1
S3150802F700080F10D106F060FB03460121184606F0E1
S3150802F7101DFF0346002B02D05B480CF0CFF97B692C
S3150802F72003F5CD73ABE006F04FFB034601211846FD
S3150802F73006F00CFF0346002B02D054480CF0BEF923
S3150802F7407B6903F5D2739AE07B69002B4ADDFB6875
S3150802F750012B0FD106F038FB03460121184606F0A5
S3150802F760F5FE0346002B02D049480CF0A7F97B693F
S3150802F770643B84E0FB68022B0FD106F025FB0346A7
S3150802F7800121184606F0E2FE0346002B02D0414844
S3150802F7900CF094F97B69FF3B71E0FB68032B10D1EF
S3150802F7A006F012FB03460121184606F0CFFE034671
S3150802F7B0002B02D038480CF081F97B69A3F5AA73AD
S3150802F7C05DE006F001FB03460121184606F0BEFE7F
S3150802F7D00346002B02D031480CF070F97B69A3F579
S3150802F7E0AA734CE0FB68B3F1FF3F0FD106F0ECFABF
S3150802F7F003460121184606F0A9FE0346002B02D04D
S3150802F80027480CF05BF97B69643338E0FB6813F12F
S3150802F810020F0FD106F0D8FA03460121184606F060
S3150802F82095FE0346002B02D01E480CF047F97B6969
S3150802F830FF3324E0FB6813F1030F10D106F0C4FA74
S3150802F84003460121184606F081FE0346002B02D024
S3150802F85015480CF033F97B6903F5AA730FE006F035
S3150802F860B3FA03460121184606F070FE0346002B3A
S3150802F87002D006480CF022F97B6903F5AA731846EA
S3150802F8801837BD4680BD00BF1CDE050854DE0508D4
S3150802F8909CDA0508D4DA05080CDB05085CDC0508E1
S3150802F8A094DC0508CCDC050804DD050880B500AF44
S3150802F8B02A4B00221A702A4B00221A70294B002260
S3150802F8C01A70294B00221A70284B00221A70284BEC
S3150802F8D000221A70274B00221A60274B00221A6050
S3150802F8E0264B00221A60264B00221A70F8F78EFE63
S3150802F8F003461846F8F7C2FE03461A46214B1A7003
S3150802F900F8F784FE034600211846F8F7DEFE03469A
S3150802F9101A461D4B1A70F8F779FE03460121184656
S3150802F920F8F7D3FE03461A46184B1A70F8F76EFE16
S3150802F930034602211846F8F7C8FE03461A46144B30
S3150802F9401A70F8F763FE034603211846F8F7BDFE58
S3150802F95003461A460F4B1A7000BF80BD7CF501207C
S3150802F9607DF501207EF501207FF5012080F5012035
S3150802F97081F5012084F5012088F501208CF5012006
S3150802F98090F5012091F5012092F5012093F50120C9
S3150802F99094F5012095F5012080B500AF274B00228A
S3150802F9A01A70274B00221A70264B00221A70264B11
S3150802F9B000221A70254B00221A60254B00221A6073
S3150802F9C0244B00221A60244B00221A70F8F71EFEF6
S3150802F9D003461846F8F752FE03461A461F4B1A7094
S3150802F9E0F8F714FE034600211846F8F76EFE03469A
S3150802F9F01A461B4B1A70F8F709FE034601211846E8
S3150802FA00F8F763FE03461A46164B1A70F8F7FEFD18
S3150802FA10034602211846F8F758FE03461A46124BC1
S3150802FA201A70F8F7F3FD034603211846F8F74DFE58
S3150802FA3003461A460D4B1A7000BF80BD7EF501209B
S3150802FA407FF5012080F5012081F5012084F501204A
S3150802FA5088F501208CF5012090F5012091F5012009
S3150802FA6092F5012093F5012094F5012095F50120E0
S3150802FA70B0B500AFF6F724F90346002B16D020F0EE
S3150802FA8045FC0546F6F728F903461A46920013443A
S3150802FA909B00DCB2F6F72CF903462344DBB2143B8F
S3150802FAA0DAB201233721284620F0ACFC324B1B7808
S3150802FAB0002B0BD031480CF001F822F05DFE03460C
S3150802FAC00D21184622F0FDFE012353E02C4B1B782C
S3150802FAD0002B0BD02B480BF0F1FF22F04DFE03460C
S3150802FAE00E21184622F0EDFE012343E0264B1B7831
S3150802FAF0002B0BD025480BF0E1FF22F03DFE034612
S3150802FB000C21184622F0DDFE012333E0204B1B7838
S3150802FB10002B0BD01F480BF0D1FF22F02DFE034617
S3150802FB200F21184622F0CDFE012323E01A4B1B783B
S3150802FB30002B0BD019480BF0C1FF22F01DFE03461D
S3150802FB401021184622F0BDFE012313E0144B1B7840
S3150802FB50002B0BD013480BF0B1FF22F00DFE034623
S3150802FB601121184622F0ADFE012303E00E480BF0E0
S3150802FB70A5FF00231846B0BD7CF501208CDE0508DA
S3150802FB807DF50120C8DE05087EF5012014DF05088B
S3150802FB907FF5012054DF050880F501209CDF050862
S3150802FBA081F50120ECDF050830E0050880B485B050
S3150802FBB000AFBA607B600346FB730B46BB73FA7BE6
S3150802FBC0BB7B9A4213D07B6883EAE372A2EBE372A9
S3150802FBD0BB68002BB8BF5B4264339A4203DD0A4B0B
S3150802FBE001221A7009E0094B01221A7005E0074B37
S3150802FBF000221A70044B00221A7000BF1437BD4641
S3150802FC005DF8047B704700BF7DF501207CF5012075
S3150802FC10B0B582B000AF78603960294B1B78022BE9
S3150802FC2022D13B68002BB8BF5B421846F0F7A8FD05
S3150802FC3004460D467B68002BB8BF5B421846F0F7B0
S3150802FC409FFD1DA3D3E90023F0F74EFC02460B469F
S3150802FC5020462946F1F78EF80346002B00D125E007
S3150802FC60184B01221A7021E03B68002BB8BF5B4291
S3150802FC701846F0F785FD04460D467B68002BB8BF8B
S3150802FC805B421846F0F77CFD4FF000020E4BF0F788
S3150802FC902BFC02460B4620462946F1F76BF803462B
S3150802FCA0002B00D102E0074B01221A7000BF083769
S3150802FCB0BD46B0BDAFF3008000000000000C7240E4
S3150802FCC0C4F401207EF5012000F4804080B582B09C
S3150802FCD000AF7860704B1B78012B00F0D9806F4B10
S3150802FCE01B78012B00F0D4806B4B1B78012B00F09C
S3150802FCF0CF806B4B1B78012B00F0CA80694B1B78AF
S3150802FD00012B00F0C580684B1B687A689A4205D0B9
S3150802FD10654A7B681360654B00221A60634B1B6851
S3150802FD200133624A1360614B1B6843F2AF62934226
S3150802FD3026D9F8F76BFC034600211846F8F7F6FCB5
S3150802FD400346012B0DD0F8F761FC0346022118463B
S3150802FD50F8F7ECFC0346012B03D0514B01221A702B
S3150802FD600EE0534B1B78012B03D14B4B01221A7021
S3150802FD7006E04F4B1B78002B02D14A4B01221A7020
S3150802FD80F8F744FC03461846F8F778FC03461A4681
S3150802FD90484B1B789A4233D1F8F738FC03460021C0
S3150802FDA01846F8F792FC03461A46434B1B789A42C2
S3150802FDB026D1F8F72BFC034601211846F8F785FCED
S3150802FDC003461A463D4B1B789A4219D1F8F71EFC90
S3150802FDD0034602211846F8F778FC03461A46384BBA
S3150802FDE01B789A420CD1F8F711FC034603211846F0
S3150802FDF0F8F76BFC03461A46324B1B789A4238D000
S3150802FE00F8F704FC03461846F8F738FC03461A4680
S3150802FE10284B1A70F8F7FAFB034600211846F8F73A
S3150802FE2054FC03461A46244B1A70F8F7EFFB0346AE
S3150802FE3001211846F8F749FC03461A461F4B1A7061
S3150802FE40F8F7E4FB034602211846F8F73EFC034698
S3150802FE501A461B4B1A70F8F7D9FB034603211846B4
S3150802FE60F8F733FC03461A46164B1A70164B00224D
S3150802FE701A60154B1B680133134A1360124B1B6831
S3150802FE8043F2C722934204D9094B01221A7000E0B1
S3150802FE9000BF0837BD4680BD7FF501207EF50120EB
S3150802FEA080F5012081F5012084F5012088F50120DD
S3150802FEB090F5012091F5012092F5012093F5012094
S3150802FEC094F5012095F501208CF5012080B582B0C4
S3150802FED000AF0346FB71144B01221A70FEF7EEF9C6
S3150802FEE0034600211846FEF7BCFC104B00221A7086
S3150802FEF00F4B00221A800F4B00221A70FEF7DEF90A
S3150802FF0003461846FEF760FCFEF7D8F9034618467C
S3150802FF10FEF773FCFB79002B01D0FFF7C7FC00BF85
S3150802FF200837BD4680BD00BF97F5012098F5012028
S3150802FF309AF5012096F5012098B500AFB64B1A78C6
S3150802FF40B64B1B789A4205D0B34B1A78B34B1A7044
S3150802FF50FFF722FDB04B1B78022B11D0AE4B1B7854
S3150802FF60062B0DD0AC4B1B780A2B09D0FEF7A6F947
S3150802FF7003461846FEF7B8F903461846FFF7A6FEE3
S3150802FF80A54B1B78002B06D0A34B1B78012B02D05E
S3150802FF90A34B00221A70A04B1B780A2B00F275831A
S3150802FFA001A252F823F000BFD5FF02080D0003088C
S3150802FFB01F0103086B010308AB0103084902030882
S3150802FFC0DB020308B1030308F10303083B04030831
S3150802FFD039050308934B00221A60934B00221A60D4
S3150802FFE0924B05221A70914B1B781846F8F7FCFBC0
S3150802FFF08B4B01221A70FEF761F903460021184657
S31508030000FEF7A4F9844B01221A7047E3884B1B6851
S31508030010632B7BD9F8F780FC844B1B781846F8F7D3
S31508030020E3FB804B1B6801337E4A13607D4B1B68D9
S31508030030B3F5C87F3BD37E4B00221A60794B002267
S315080300401A60FEF73BF9034600211846FEF77EF9C8
S31508030050764B1B780133DAB2744B1A70734B1B78E1
S315080300600C2B24D9F8F78AFC0020F8F7BDFB6C4B58
S3150803007000221A706D4B03221A70FEF71FF9024607
S315080300806A4B1B7819461046FEF7D0FBFEF716F99E
S3150803009003461846FEF728F90246644B1B7865495A
S315080300A0022006F039FC5C4B02221A70F6E2FEF7D0
S315080300B005F903461846FEF717F90346002BB8BF9A
S315080300C05B42112B40F3E382F8F758FC0020F8F75C
S315080300D08BFB534B00221A70FEF7F0F80246534B7C
S315080300E01B7819461046FEF7A1FBFEF7E7F8034609
S315080300F01846FEF7F9F802464C4B1B784E49022080
S3150803010006F00AFC444B02221A70C7E2484B1B68E6
S315080301100133474A13600020F8F766FBB7E2474BFB
S315080301201B8801339AB2454B1A80444B1B88B3F597
S31508030130FA7FC0F0AE82414B00221A80364B032267
S315080301401A70FEF7BBF80346F0211846FEF732F994
S315080301503B4B1B6801219FED2A2B9FED2B1B9FED24
S31508030160280B1846FDF7DEFA93E2F8F74FFA03462B
S315080301701846F8F783FA0346012B03D1264B0422C4
S315080301801A7005E02D4B00221A80234B05221A709C
S315080301902C4B00221A802A4B1B689FED1D0B184611
S315080301A0FDF73FFDF8F7B8FB78E2F8F72FFA0346B1
S315080301B01846F8F763FA0346022B40F06C82FEF7FB
S315080301C07DF803461846FEF78FF80346322B0ADCFA
S315080301D0FEF774F803461846FEF786F8034613F146
S315080301E0320F80F25882154B00221A800A4B1B786D
S315080301F00133DAB2084B1A704DE200BFAFF3008041
S315080302000000000000000000000000000000044099
S31508030210000000000000244098F50120ABF50120FA
S31508030220A9F501209CF50120A4F50120A8F50120D4
S31508030230A0F5012070E005089CE00508ACF501204F
S31508030240F41200209AF50120F8F7E0F90346184658
S31508030250F8F714FA0346012B32D1F8F78FFBAE4BA6
S315080302601B689FEDA70B1846FDF7DBFCAA4B1B681B
S315080302701846FDF730FA05F0A7FD0346012118468F
S3150803028006F064F90346002B0DD0FEF717F803466C
S315080302901846FEF729F803461946A0480BF00EFC44
S315080302A09F480BF00BFCFEF709F803460021184696
S315080302B0FEF74CF89B4B00221A809B4B06221A70BA
S315080302C0FDF7FCFF03461846FEF70EF803461946E4
S315080302D04FF49B70FFF79CFCE0E1924B1B880133BC
S315080302E09AB2904B1A808F4B1B88B3F5FA7F5BD370
S315080302F08C4B00221A808D4B00221A80F8F79AFB42
S31508030300FDF7DCFF0446FEF79CF80346194620462C
S31508030310FEF750F8FDF7D2FF0446FDF7CFFF034675
S315080303201846FEF73BF8034619462046FEF75DF8DE
S31508030330FDF7C4FF0346FF211846FEF773F8FDF7DA
S31508030340BDFF0446FDF7BAFF03461846FEF726F82F
S31508030350034619462046FEF70DFAFDF7AFFF034697
S315080303601846FEF71BF80346194671480BF0A6FB19
S315080303706B480BF0A3FB6B4B00221A80FDF79EFF1D
S315080303800346F0211846FEF715F8634B1B6801214F
S315080303909FED5B2B9FED5C1B9FED590B1846FDF7F5
S315080303A0C1F9614B07221A70604B00221A8075E166
S315080303B0F8F72CF903461846F8F760F90346012BB4
S315080303C003D1594B08221A7005E0564B00221A80AE
S315080303D0554B09221A70554B00221A804E4B1B683F
S315080303E09FED4B0B1846FDF71CFCF8F795FA55E1FC
S315080303F0F8F70CF903461846F8F740F90346022BB3
S3150803040040F04B81FDF75AFF03461846FDF76CFF8C
S315080304100346322B0ADCFDF751FF03461846FDF760
S3150803042063FF034613F1320F80F237813D4B0022F7
S315080304301A803D4B09221A702FE1F8F7E7F80346AD
S315080304401846F8F71BF90346012B4BD1F8F796FA2A
S31508030450314B1B689FED2A0B1846FDF7E2FB2E4B23
S315080304601B681846FDF737F905F0AEFC034601216C
S31508030470184606F06BF80346002B0DD0FDF71EFF52
S3150803048003461846FDF730FF0346194623480BF083
S3150803049015FB23480BF012FBFDF710FF034618461E
S315080304A0FDF722FF0346722B0CDDFDF707FF034614
S315080304B01846FDF719FF0346D72B03DC1D4B02220B
S315080304C01A7002E01B4B01221A70FDF7F7FE03466A
S315080304D000211846FDF73AFF124B00221A80124BE9
S315080304E00A221A70FDF7EAFE03461846FDF7FCFED4
S315080304F0034619464FF49B70FFF78AFBCEE000BF0D
S315080305000000000000000000000000000000044096
S315080305100000000000002440F4120020C0E0050893
S31508030520D4E00508ACF5012098F501209AF50120D9
S31508030530D8E00508C4F401207F4B1B8801339AB21F
S315080305407D4B1A807C4B1B88B3F5FA7FC0F09980E4
S31508030550794B00221A80794B00221A80FDF7AEFEEA
S315080305600446FDF76EFF034619462046FDF722FFAC
S31508030570FDF7A4FE0446FDF7A1FE03461846FDF75C
S315080305800DFF034619462046FDF72FFFFDF796FE96
S315080305900346FF211846FDF745FFFDF78FFE044680
S315080305A0FDF78CFE03461846FDF7F8FE0346194683
S315080305B02046FEF7DFF8FDF781FE03461846FDF7EA
S315080305C0EDFE034619465E480BF078FA5D480BF0D4
S315080305D075FAFDF773FE03461846FDF7DFFE034675
S315080305E003F00103DBB2012B18D1574B08221A700B
S315080305F0564B1B6801219FED462B9FED471B9FED2D
S31508030600440B1846FDF78EF8504B1B689FED440BB9
S315080306101846FDF706FBF8F77FF932E04C4B1B78D3
S31508030620022B0FD1494B1B6801219FED392B9FEDF7
S315080306303E1B9FED370B1846FDF774F845480BF03C
S315080306403DFA0EE0414B1B6801219FED312B9FEDCF
S31508030650381B9FED2F0B1846FDF764F83E480BF041
S315080306602DFAFDF72BFE03461846FDF797FE0346BC
S315080306701846374B1B781A46012106F0F5FD012368
S3150803068042E02E4B00221A8008E000BF06E000BFB6
S3150803069004E000BF02E000BF00E000BF274B1B8851
S315080306A001339AB2254B1A80244B1B8847F22F52E3
S315080306B0934228D9F8F7BEF9244B1B689FED140B10
S315080306C01846FDF7AEFAFFF7D3F90346002B06D112
S315080306D022F052F803460A21184622F0F2F80022BD
S315080306E00221FF2006F0C0FD184B1B681846FCF7CD
S315080306F0F2FFFDF7E3FD034600211846FDF726FE44
S315080307004FF0FF3300E00023184698BDAFF300808F
S315080307100000000000000000000000000000044084
S315080307200000000000002440B81E85EB51B8FA3FCC
S31508030730CDCCCCCCCCCC1640ACF501209AF5012017
S31508030740D8E00508D4E0050898F50120F41200203E
S31508030750C4F40120F8E0050820E1050800000000BC
S3150803076090B583B000AF0023FB71D74B1A78D74BEC
S315080307701B789A4205D0D44B1A78D44B1A70FFF7D4
S315080307800BF9D14B1B78002B2FD0CF4B1B78142B8F
S315080307902BD0CD4B1B781E2B27D0FDF78FFD034699
S315080307A01846FDF7A1FD03461846FFF78FFAC64B11
S315080307B01B78632B0DD8C64B1C68FDF77FFD0346D4
S315080307C01846FDF791FD034619462046FFF720FA1A
S315080307D00BE0FDF773FD03461846FDF785FD034653
S315080307E019464FF49B70FFF713FAB74B1B78712B17
S315080307F003F2308301A252F823F000BFC5090308A8
S315080308001110030801120308B9140308553E030817
S31508030810553E0308553E0308553E0308553E03084F
S31508030820553E0308553E0308DD1603087D180308DD
S315080308302F1B0308553E0308553E0308553E030878
S31508030840553E0308553E0308553E0308611D030834
S31508030850F5220308C1250308553E0308553E030838
S31508030860553E0308553E0308553E0308553E0308FF
S31508030870553E03084F28030839290308D12B0308D3
S31508030880553E0308553E0308553E0308553E0308DF
S31508030890553E0308553E0308553E0308553E0308CF
S315080308A0553E0308553E0308553E0308553E0308BF
S315080308B0553E0308553E0308553E0308553E0308AF
S315080308C0553E0308553E0308553E0308553E03089F
S315080308D0553E0308553E0308553E0308553E03088F
S315080308E0553E0308553E0308553E0308553E03087F
S315080308F0553E0308553E0308553E0308553E03086F
S31508030900553E0308553E0308553E0308553E03085E
S31508030910553E0308553E0308553E0308553E03084E
S31508030920553E0308553E0308553E0308553E03083E
S31508030930553E0308553E0308553E0308553E03082E
S31508030940553E0308553E0308553E0308553E03081E
S31508030950553E0308553E0308553E0308553E03080E
S31508030960553E0308553E0308553E0308553E0308FE
S31508030970553E0308553E0308553E0308553E0308EE
S31508030980553E0308553E0308553E03083B2E030808
S315080309905F3003086B32030855340308553E0308D2
S315080309A0553E0308553E0308553E0308553E0308BE
S315080309B0553E030859360308833803084B3A030898
S315080309C0753C0308434B00221A60434B00221A80E6
S315080309D0424B00221A80424B00221A60414B0022E6
